:100000000C94F0040C940F050C940F050C940F0540
:100010000C940F050C940F050C940F050C940F0510
:100020000C940F050C940F050C940F050C940F0500
:100030000C940F050C940F050C940F050C9494A8C8
:100040000C940F050C940F050C940F050C940F05E0
:100050000C940F050C940F050C940F050C940F05D0
:100060000C940F050C94B68D0C94E48D0C940F0534
:100070000C940F050C940F050C940F050C940F05B0
:100080000C940F050C940F050C940F050C940F05A0
:100090000C94B20F0C940F050C94DE0F0C940F050A
:1000A0000C940F050C940F050C940F050C940F0580
:1000B0000C940F050C940F050C940F050C940F0570
:1000C0000C940F050C940F050C940F050C940F0560
:1000D0000C940F050C940F050C940F050C940F0550
:1000E0000C940F050C94C3100C94CD100C94B91003
:1000F0000C9463100C948E100C94D7100C94381040
:100100000C94EB100C9496150C94A9150C940F05F7
:100110000C940F050C940F050C94F5100C94E11041
:100120006E616E00696E6600202073747430383A18
:1001300030343A3030202E2E2E2E20536574207409
:10014000696D65202848483A4D4D3A535320666FF3
:10015000726D61742900202073747531323735391E
:100160003930383538202E2E205365742074696D4F
:10017000652F646174652028556E69782074696DF7
:100180006520666F726D6174290D0A00202065205C
:100190002E2E2E2E2E2E2E2E2E2E2E2E2E2E204576
:1001A0007261736520454550524F4D2C206C6F6134
:1001B000642064656661756C7420636F6E66696740
:1001C00075726174696F6E0D0A0047656E657261C4
:1001D0006C20436F6E6669673A0D0A0020206D201F
:1001E000706F6C6C203630202E2E2E2E2E2E20532B
:1001F000657420696E74657276616C2062657477CF
:1002000065656E20636865636B696E6720666F72F3
:1002100020757064617465730D0A00202020202011
:1002200020202020202020616E6420656E647320D1
:1002300061742030373A35393A35390D0A002020BB
:100240002020202020202020202020696E64657836
:1002500020322E20507269636520697320302E345D
:10026000352C207374617274732061742030303ABD
:1002700030303A30300D0A0020202020202020206D
:10028000202020204164642F4F7665727772697454
:100290006520656E74727920746F2070726963696D
:1002A0006E67207461626C652C20656E7472790DC6
:1002B0000A002020702061646420322030303A30FF
:1002C000303A30302030373A35393A353920302E0F
:1002D00034350D0A002020702064656C2032202EF9
:1002E0002044656C65746520656E747279203220D7
:1002F00066726F6D207072696365207461626C65EF
:100300000D0A00202070207072696E74202E20501B
:1003100072696E742070726963696E6720696E66B7
:100320006F0D0A0050726963696E67206F72204D0D
:10033000657465722053747566663A0D0A00202054
:10034000736D63202E2E2E2E2E20536574206D6F1C
:10035000646520746F20636F6F7264696E61746F7F
:10036000720D0A002020736D72202E2E2E2E2E204C
:10037000536574206D6F646520746F20726F75749F
:1003800065722F656E646E6F64650D0A00202073C0
:10039000633135202E2E2E2E205365742063686124
:1003A0006E6E656C20746F2069653A2031350D0AD8
:1003B000002020737042414444202E2E2053657447
:1003C0002050414E494420746F2069653A203078AE
:1003D000424141440D0A003830322E31352E34204E
:1003E000436F6D6D616E64733A0D0A002020697071
:1003F000202E2E2E2E2E2E205072696E74206675A1
:100400006C6C204950204D656E750D0A00495020D6
:10041000436F6D6D616E64733A0D0A002020642095
:100420002E2E2E2E2E2E2E2044756D70207261647D
:10043000696F207265676973746572730D0A0020B5
:100440002069202E2E2E2E2E2E2E20496E666F0D08
:100450000A00446562756767696E673A0D0A005560
:100460006E6B6E6F776E206D6574657220636F6D55
:100470006D616E640D0A00556E6B6E6F776E206D48
:100480006574657220636F6D6D616E640D0A00495D
:100490006E76616C696420636F6D6D616E64206659
:1004A0006F7220636F6F7264696E61746F720D0A90
:1004B00000556E6B6E6F776E2070726963696E6740
:1004C00020636F6D6D616E640D0A00556E6B6E6F0B
:1004D000776E2070726963696E6720636F6D6D61FE
:1004E0006E640D0A000D0A4572726F7220616464B9
:1004F000696E6720656E7472790D0A00556E6B6EB9
:100500006F776E20277365742720636F6D6D616E42
:10051000643F0D0A00496E76616C69642074696DF0
:1005200065206F7065726174696F6E0D0A006E6F81
:1005300064652074797065206368616E6765642EF8
:10054000205265626F6F74206E6F77202E2E2E0DF5
:100550000A006E6F64652074797065206368616E4F
:100560006765642E205265626F6F74206E6F77200E
:100570002E2E2E0D0A002C207265736574206E6F6E
:10058000646520746F2074616B65206566666563C1
:10059000742E0D0A0053657474696E672063686178
:1005A0006E6E656C20746F20000D0A53657474695B
:1005B0006E672050414E494420746F20000D0A5A46
:1005C00049503E00454550524F4D20496E76616C72
:1005D00069642E204C6F6164696E67206465666192
:1005E000756C74730D0A00454550524F4D2056618D
:1005F0006C69640D0A0003020201010000FFFEFDA8
:10060000FCFBF9F7F4EF992425219020682B0000DA
:100610000000B43200005C2F8D2E00000437000073
:100620008738193300001C242C240000F2230B24EB
:1006300000000000D42300000000000032238423C7
:100640000000722322235423000013236323010498
:100650000101010201010101010101010101040186
:10066000080201010101020101020102010102016E
:100670000202010101012201110104010401010131
:1006800001080202000110010808485454502F319B
:100690002E3120323030204F4B0D0A436F6E74657F
:1006A0006E742D547970653A206170706C69636165
:1006B00074696F6E2F6578690D0A0D0A003C3F78EA
:1006C0006D6C2076657273696F6E3D92312E30923B
:1006D00020656E636F64696E673D925554462D3890
:1006E000923F3E0D0A003C54696D6520786D6C6E3A
:1006F000733D92687474707B737D3A2F2F726566B8
:100700002F766572923E0D0A3C556E6978546D3EA7
:10071000003C2F556E6978546D3E0D0A3C2F54698C
:100720006D653E0D0A003C54617269666650726FD9
:1007300066696C6520786D6C6E733D926874747038
:100740007B737D3A2F2F7265662F766572923E0D10
:100750000A003C54544920687265663D222F70722D
:100760002F302F7466662F0022202F3E0D0A003C8A
:100770002F54617269666650726F66696C65203EBF
:100780000D0A003C54544920786D6C6E733D92689C
:100790007474707B737D3A2F2F7265662F76657245
:1007A000923E0D0A3C737461727454696D653E002B
:1007B0003C2F737461727454696D653E0D0A3C651B
:1007C0006E6454696D653E003C2F656E6454696DBE
:1007D000653E0D0A3C4368617267653E3C66697818
:1007E00065643E3C76616C3E003C2F76616C3E0D4C
:1007F0000A3C6375723E5553443C2F6375723E0D3F
:100800000A3C2F66697865643E0D0A3C2F43686197
:100810007267653E0D0A3C2F5454493E0D0A003C58
:1008200041637469766554617269666620786D6C9F
:100830006E733D92687474707B737D3A2F2F72656E
:10084000662F766572923E003C2F4163746976652F
:100850005461726966663E000D0A00202020202047
:100860002020207C00202020202A2020207C0049DD
:100870006E646578207C20416374697665207C20F5
:100880002020537461727420207C20202020456E2B
:10089000642020207C2056616C7565200D0A00497B
:1008A0004E46494E4954594E414ECDCCCC3D0AD7C7
:1008B000233C17B7D13877CC2B329595E6241FB15E
:1008C0004F0A000020410000C84200401C4620BCE6
:1008D000BE4CCA1B0E5AAEC59D7400407A10F35A26
:1008E00000A0724E18090010A5D4E80000E8764870
:1008F000170000E40B54020000CA9A3B000000E11C
:10090000F505000080969800000040420F000000AE
:10091000A08601000000102700000000E80300008E
:1009200000006400000000000A0000000000010058
:10093000000000002C76D888DC674F0823DFC1DF79
:10094000AE59E1B1B796E5E3E453C63AE65199767C
:1009500096E8E6C28426EB898C9B62ED407C6FFCB6
:10096000EFBC9C9F40F2BAA56FA5F490055A2AF7F8
:100970005C936B6CF9676DC11BFCE0E40D47FEF501
:1009800020E6B500D0ED902E030094357705008069
:10099000841E080000204E0A000000C80C333333C8
:1009A000330F986E12831141EF8D2114893BE65568
:1009B00016CFFEE6DB18D1844B381BF77C1D901D4B
:1009C000A4BBE424203284725E228100C9F124ECAD
:1009D000A1E53D276364696E6F70737578585B009D
:1009E00011241FBECFEFD1E4DEBFCDBF15E1A0E0E3
:1009F000B2E0E4E1F1E801E00BBF02C007900D9224
:100A0000AA3FB107D9F719E3AAEFB5E101C01D92DA
:100A1000A537B107E1F70E94900C0C94C0680C94C4
:100A200000000895089508956F927F928F929F928B
:100A3000AF92BF92CF92DF92EF92FF920F931F93EC
:100A4000DF93CF93CDB7DEB7EC970FB6F894DEBF48
:100A50000FBECDBF80E00E94B29300D000D000D086
:100A6000EDB7FEB731964E010894811C911CADB7CD
:100A7000BEB712969C928E92119780E092E093837B
:100A800082838091990790919A07958384830E942D
:100A90006DBCEDB7FEB736960FB6F894FEBF0FBE2D
:100AA000EDBF82E0B4010E94208E80E197E20E94B7
:100AB00001128091B61B882319F42EE032E002C0A7
:100AC00022E132E000D000D000D0EDB7FEB7319681
:100AD0008E010F5F1F4FADB7BEB712961C930E93DA
:100AE000119785E192E093838283358324830E946A
:100AF0006DBCEDB7FEB736960FB6F894FEBF0FBECD
:100B0000EDBF83E0B4010E94208EC80162E272E072
:100B10000E940CBBD8010D900020E9F77D010894DC
:100B2000E108F10880E197E20E940112CC24DD2463
:100B300029E2622E22E0722E58018E01095F1F4FBA
:100B400000D000D000D0EDB7FEB73196ADB7BEB73C
:100B50001296FC92EE92119773826282D601AE5D7C
:100B6000B64D8C91848315820E946DBCE2E0F0E06A
:100B7000EE0EFF1E8DB79EB706960FB6F8949EBF79
:100B80000FBE8DBF97E0C91661F4D7011C9284E0B7
:100B9000B4010E94208EC5016EE272E00E940CBB7F
:100BA00078010894C11CD11CB0E1CB16D10441F6E8
:100BB000F701108285E0B4010E94208E8E010F5F44
:100BC0001F4FC80165E372E00E940CBBD8010D9075
:100BD0000020E9F77D010894E108F10892E3C92EAD
:100BE00099E2D92E870189E2A82E82E0B82E00D0A2
:100BF00000D000D0EDB7FEB73196ADB7BEB71296B4
:100C00001C930E931197B382A282D6018D916D0130
:100C1000848315820E946DBC0E5F1F4FEDB7FEB737
:100C200036960FB6F894FEBF0FBEEDBFFAE3CF16AF
:100C3000F9E2DF06E1F6D70150961C9280E197E2D7
:100C40000E94011286E0B4010E94208E83E040E4FD
:100C500052E46FE070E020E030E008E416E0EE24BB
:100C6000FF240E941514EC960FB6F894DEBF0FBE59
:100C7000CDBFCF91DF911F910F91FF90EF90DF904B
:100C8000CF90BF90AF909F908F907F906F9008957E
:100C9000EF92FF920F931F93DF93CF93CDB7DEB701
:100CA000EC970FB6F894DEBF0FBECDBF80E00E9478
:100CB000409181E00E94409182E00E94409180E05A
:100CC0000E944F902DB73EB7285030400FB6F89491
:100CD0003EBF0FBE2DBFEDB7FEB731968E010F5F41
:100CE0001F4FADB7BEB712961C930E9311972CE30E
:100CF00032E03383228364837583868397830E94E3
:100D00006DBC2DB73EB7285F3F4F0FB6F8943EBF7E
:100D10000FBE2DBF87E0B8010E94208E81E00E94A7
:100D20004F90ADB7BEB718970FB6F894BEBF0FBEC1
:100D3000ADBFEDB7FEB7319612961C930E93119787
:100D400026E432E03383228364837583868397832A
:100D50000E946DBC2DB73EB7285F3F4F0FB6F89489
:100D60003EBF0FBE2DBF88E0B8010E94208E82E0FA
:100D70000E944F90ADB7BEB718970FB6F894BEBF9C
:100D80000FBEADBFEDB7FEB7319612961C930E9312
:100D9000119720E532E03383228364837583868351
:100DA00097830E946DBC2DB73EB7285F3F4F0FB6AB
:100DB000F8943EBF0FBE2DBF89E0B8010E94208E7F
:100DC00083E040E452E46FE070E020E030E004E1D2
:100DD00015E0EE24FF240E941514EC960FB6F8944B
:100DE000DEBF0FBECDBFCF91DF911F910F91FF905E
:100DF000EF900895AF92BF92CF92DF92EF92FF9261
:100E00000F931F93CF93DF938AE592E00E9438BC43
:100E1000C8E1D6E048E7E42E43E0F42E37E6A32EFF
:100E200032E0B32EE881F981108100D000D000D0EB
:100E3000EDB7FEB73196ADB7BEB71296BC92AE9283
:100E40001197F382E282148315820E94FCBB07E0B3
:100E50008DB79EB706960FB6F8949EBF0FBE8DBF96
:100E6000C12EDD24C601002E02C0959587950A94F7
:100E7000E2F780FD03C080E390E002C081E390E0F0
:100E800060916F39709170390E94D0BB015050F75A
:100E900085E792E00E9438BC2296A0E1B0E0EA0E1D
:100EA000FB1EB6E0CC36DB0709F0BCCF85E792E04D
:100EB0000E9438BCDF91CF911F910F91FF90EF906E
:100EC000DF90CF90BF90AF9008953F924F925F9286
:100ED0006F927F928F929F92AF92BF92CF92DF924A
:100EE000EF92FF920F931F93DF93CF93CDB7DEB7AF
:100EF0006F970FB6F894DEBF0FBECDBF8091FA1585
:100F00009091FB1501979093FB158093FA1501962C
:100F10009F70892B11F46A9A629A789480E090E02D
:100F20000E94AC0E182F8F3F09F4E2C48B3121F0E0
:100F30008091FC158823D1F180914B38882329F0CA
:100F400080E090E00E94D39ED3C48091FC1588235A
:100F500011F481E005C0813031F41B3521F582E0C8
:100F60008093FC15C5C48230F1F41092FC15113445
:100F700009F0BEC400D000D086E792E0ADB7BEB79E
:100F800012969C938E9311978DEF95E114969C93F6
:100F90008E9313970E94FCBB1092C5160F900F9072
:100FA0000F900F90A5C41092FC15A2C48091C51695
:100FB000883C50F460916F3970917039812F992776
:100FC00087FD90950E94D0BB8091C516883C08F0A3
:100FD0008FC41D3019F01A3009F075C4E82FF0E005
:100FE000EA53F94E1082982F9F5F9093C516809117
:100FF0004B38882349F086EC96E10E94D39E1092EC
:10100000C6161092C5168ACF8091C6168C3609F482
:101010006DC28D3684F4843609F40DC1853624F40E
:101020008C3409F050C374C2853609F485C2893600
:1010300009F049C313C0823709F455C283373CF421
:101040008D3609F40AC3803709F03DC37BC283376C
:1010500009F4F4C0843709F036C3AEC08091C716D6
:10106000803729F486EC96E10E94569F15C400D083
:1010700089E792E0EDB7FEB7928381830E94FCBBC3
:101080008DB79EB708970FB6F8949EBF0FBE8DBF61
:10109000EDB7FEB7319680E892E0ADB7BEB71296D5
:1010A0009C938E93119780915F2690916026A091DA
:1010B0006126B091622682839383A483B583809155
:1010C0005B2690915C26A0915D26B0915E2686837A
:1010D0009783A087B1870E94FCBB0F900F900F9061
:1010E0000F90EDB7FEB731968AE992E0ADB7BEB783
:1010F00012969C938E931197809198078283138206
:101100008091990790919A07958384830E94FCBBF4
:10111000EDB7FEB736960FB6F894FEBF0FBEEDBF23
:101120008091760390917703892B51F400D086EB60
:1011300092E0ADB7BEB712969C938E93119707C0FD
:1011400000D08AEC92E0EDB7FEB7928381830E94D3
:10115000FCBB0F900F90CE010196BE016E5F7F4FDA
:10116000AE014D5F5F4F0E9456A88DB79EB708979E
:101170000FB6F8949EBF0FBE8DBFEDB7FEB7319688
:1011800082EE92E0ADB7BEB712969C938E93119704
:101190008981828313828A81848315828B818683ED
:1011A00017820E94FCBBEDB7FEB738960FB6F894D5
:1011B000FEBF0FBEEDBF70C32091990730919A0713
:1011C000FE0135968BE0DF011D928A95E9F782E0FA
:1011D0008D833F832E83933048F486EC96E16AEF4B
:1011E00072E00E940CBB85E08093C5168091760367
:1011F000909177034091C516BE016B5F7F4F892B9D
:1012000051F485E090E099878887415082E027EC8F
:1012100036E100E205C0415082E027EC36E103E20E
:10122000EE24E394E5E0CE2EAA24A39488248394AC
:101230000E943E3B31C30E94FA062EC38091C7161E
:101240008D3609F48FC08E363CF4833609F441C0E4
:101250008B3609F038C16BC0833709F4C8C08437B6
:1012600009F4FDC0803709F02EC188EC96E10E9498
:101270008B8A9C838B8300D089EA95E0EDB7FEB71B
:10128000928381830E940EBC00D08FEF92E0ADB7B5
:10129000BEB712969C938E9311978B819C81149666
:1012A0009C938E9313970E94FCBB0F900F900F900E
:1012B0000F908E010D5F1F4F80E5B8010E94BF3B6C
:1012C00080E50E94793A8EE090E062E070E0A8014B
:1012D000C3C01B8288EC96E10E9476B98B8380E1C3
:1012E00090E061E070E0AE014D5F5F4F0E9404113D
:1012F00000D085E995E0EDB7FEB7928381830E9427
:101300000EBC00D0EDB7FEB7319686E093E0ADB7E6
:10131000BEB712969C938E9311978B818283138212
:101320000E94FCBB0F900F9086E795E0BDC108ECD2
:1013300016E160E1E62EF12CEC0EFD1EC8010E94C4
:101340002B8AD7018D937D010E5F1F4FB6E1083EBA
:101350001B07A1F784E190E060E170E0AE01405F1F
:101360005F4F7AC08091C816823771F481E090E0B7
:10137000909377038093760300D082E595E0EDB7F4
:10138000FEB7928381830FC08336C1F41092770336
:101390001092760300D08EE295E0ADB7BEB71296FC
:1013A0009C938E9311970E940EBC0F900F9081E139
:1013B00090E062E070E046E753E04EC008EC16E1D2
:1013C00052E3E52E59E2F52EC8010E942B8AF7015F
:1013D00081937F010E5F1F4FF6E1083D1F07A1F7C4
:1013E00084E290E068E070E042E359E235C0809129
:1013F000C816813321F581E08093B61B8DE566EB3D
:101400007BE10E94BF3B87E766EB7BE10E94BF3B2D
:1014100080E866EB7BE10E94BF3B82E866EB7BE104
:101420000E94BF3B0E94F03B0E94F03B81E862E2D9
:1014300079E20E94BF3B83E862E379E205C0109243
:10144000B61B8DE566EB7BE10E94BF3B83E190E03C
:1014500061E070E046EB5BE10E9404111DC28091E7
:10146000C8168437C9F40E9405A85B016C0120E806
:1014700031E541E050E00E9445B57B018C0189ECEB
:1014800096E10E94CCA86A0D7B1D8C1D9D1D6E19D6
:101490007F09800B910B10C0853789F489EC96E1A8
:1014A00060E070E04AE050E00E9460B861157105AC
:1014B0008105910509F4F0C10E94F9A7EDC100D0A2
:1014C00085E195E0F9C000D08CEF94E0EDB7FEB770
:1014D000928381830E940EBC0F900F9080E090E079
:1014E0000E941405D9C10E944806D6C14EB1209170
:1014F000C716332727FD30952053304081E090E018
:1015000002C0880F991F2A95E2F78C71842B12C0B4
:101510004EB12091C716332727FD30952053304018
:1015200081E090E002C0880F991F2A95E2F78C7144
:10153000809584238EB9B0C180ED90E06FEF0E945A
:10154000F9BFAAC188EC96E169E073E00E94C4BAD1
:10155000FC01009709F47DC08081843649F0803712
:1015600021F0813609F071C01DC00E9486A994C186
:1015700080E090E069E073E00E94C4BA0E9476B90E
:10158000182F0E942EA700D000D0EDB7FEB73196DD
:101590008DE093E0ADB7BEB712969C938E931197F2
:1015A000128340C080E090E069E073E00E94C4BA1A
:1015B0000E9476B9382E80E090E069E073E00E94E6
:1015C000C4BA0E94CCA82B013C0180E090E069E005
:1015D00073E00E94C4BA0E94CCA84B015C0180E079
:1015E00090E069E073E00E94C4BA60E070E00E949D
:1015F000F2B66B017C01832DB301A2019501840138
:101600000E943FA78823E9F400D000D0EDB7FEB7D1
:10161000319680E293E0ADB7BEB712969C938E935D
:101620001197328213820E94FCBB0F900F900F9093
:101630000F900E941DA7AC018EE490E062E870E07C
:101640000BCF00D085EE94E02FC000D08BEC94E05F
:1016500033C000D081EB94E027C080917603909155
:101660007703892B21F400D08FE894E025C088EC23
:1016700096E169E073E00E94C4BAFC010097C9F0EA
:101680008081893609F408C1803759F480E090E000
:1016900069E073E00E94C4BA0E9476B90E9415A75F
:1016A000FBC000D087E794E0EDB7FEB7928381835B
:1016B000EFC000D08FE594E0ADB7BEB712969C9313
:1016C0008E931197E5C000D082E594E0EDB7FEB7A8
:1016D000928381830E940EBCEFE3F4E0ADB7BEB706
:1016E0001296FC93EE9311970E940EBCECE1F4E08D
:1016F000ADB7BEB71296FC93EE9311970E940EBC45
:10170000EDE0F4E0ADB7BEB71296FC93EE931197FF
:101710000E940EBCECEEF3E0ADB7BEB71296FC93A0
:10172000EE9311970E940EBCE7EDF3E0ADB7BEB7A4
:101730001296FC93EE9311970E940EBCE1EBF3E03E
:10174000ADB7BEB71296FC93EE9311970E940EBCF4
:10175000EDE8F3E0ADB7BEB71296FC93EE931197A8
:101760000E940EBCE4E6F3E0ADB7BEB71296FC9360
:10177000EE9311970E940EBCEEE3F3E0ADB7BEB757
:101780001296FC93EE9311970E940EBCE4E2F3E0F4
:10179000ADB7BEB71296FC93EE9311970E940EBCA4
:1017A000E3E0F3E0ADB7BEB71296FC93EE9311976A
:1017B0000E940EBCE5EDF2E0ADB7BEB71296FC9309
:1017C000EE9311970E940EBCE2EBF2E0ADB7BEB70C
:1017D0001296FC93EE9311970E940EBCE8E7F2E09C
:1017E000ADB7BEB71296FC93EE9311970E940EBC54
:1017F000EEE3F2E0ADB7BEB71296FC93EE9311970D
:101800000E940EBCEBE1F2E0ADB7BEB71296FC93BE
:10181000EE9311970E940EBC0F900F90809176036B
:1018200090917703892B69F000D0ECEDF1E0ADB732
:10183000BEB71296FC93EE9311970E940EBC0F90C8
:101840000F9000D0EAECF1E0ADB7BEB71296FC9372
:10185000EE9311970E940EBCECE8F1E0ADB7BEB775
:101860001296FC93EE9311970E940EBCE6E5F1E010
:10187000ADB7BEB71296FC93EE9311970E940EBCC3
:10188000E8E2F1E0ADB7BEB71296FC93EE93119784
:101890000E940EBC0F900F901092C6161092C516A3
:1018A00080914B38882309F039CB00D0E3E3F3E093
:1018B000ADB7BEB71296FC93EE9311970E94FCBB96
:1018C0000F900F902BCB183051F4882309F426CBBE
:1018D000E82FF0E0EA53F94E1082815006C0E82F5D
:1018E000F0E0EA53F94E10838F5F8093C51616CB54
:1018F0006F960FB6F894DEBF0FBECDBFCF91DF91CC
:101900001F910F91FF90EF90DF90CF90BF90AF901D
:101910009F908F907F906F905F904F903F90089531
:10192000CF92DF92EF92FF920F931F93DF93CF93AB
:10193000CDB7DEB728970FB6F894DEBF0FBECDBF88
:101940000E94063C882311F00E94FF100E94BE15E1
:10195000789481E00E941D10882311F00E94FF10EE
:101960000E94B18C8AB1806D8AB98BB1806C8BB9C1
:101970005C988CE364E070E04AE353E00E94128DCF
:1019800080E395E70E94011280E395E70E9401122F
:1019900080E395E70E9401120E94358F8EED9EE054
:1019A00065EC7EE00E9484BB00D000D000D0EDB793
:1019B000FEB731968FE393E0ADB7BEB712969C9316
:1019C0008E93119781E693E0938382838DE693E073
:1019D000958384830E94FCBBEDB7FEB736960FB6A5
:1019E000F894FEBF0FBEEDBF80ED90E00E94F1BF06
:1019F000893A09F084C000D087EE95E0ADB7BEB754
:101A000012969C938E9311970E940EBC0F900F908C
:101A100080E090E060E170E041E050E028E937E0EC
:101A20000E94361180E090E061E170E042E050E019
:101A300026E733E00E94361180E090E06EE070E02F
:101A400042E050E029E937E00E94361180E090E062
:101A500068E070E046E050E024E636E20E9436118D
:101A600080E090E063E170E041E050E026EB3BE194
:101A70000E94361180E090E064E170E040E150E0C7
:101A800022E239E20E94361180E090E064E270E0E8
:101A900048E050E022E339E20E94361180E090E015
:101AA0006CE470E042E050E024EB3BE10E94361130
:101AB00080E090E06CE370E040E150E028E438E042
:101AC0000E94361180E090E06CE270E040E150E06E
:101AD00028E538E00E9436118091760390917703D3
:101AE000892B09F00EC10E941DA79C0180E090E0A7
:101AF0006EE470E042E850E00E94361102C100D06E
:101B000084EC95E0EDB7FEB7928381830E940EBC12
:101B100098E1909398070F900F9080916326882307
:101B200099F49093642680EF809365268FE98093E3
:101B3000662685EE809367260E94E2B6809368262B
:101B40000E94E2B6809369268E010F5F1F4F88E0E6
:101B5000D8011D928A95E9F781E0898382E08A8322
:101B600083E08B8384E08C8385E08D8386E08E83A5
:101B700087E08F8381E090E060E070E048E050E033
:101B800098010E94361180E090E068E070E0A801C2
:101B90000E94041180E190E061E070E048E957E0C4
:101BA0000E94041180E090E061E170E042E050E0CA
:101BB00026E733E00E9436118091760390917703F7
:101BC000029730F081E090E0909377038093760362
:101BD0008EE090E062E070E049E957E00E94041175
:101BE0008CE490E062E070E044EB5BE10E94041161
:101BF00088E090E066E070E044E656E20E9404115E
:101C00008CE390E060E170E048E458E00E94041149
:101C10008CE290E060E170E048E558E00E94041139
:101C200083E190E061E070E046EB5BE10E9404112B
:101C30008091760390917703892B09F054C080E05E
:101C400040E050E060E070E008E710E020E030E0C5
:101C50000F2EF0E0CF2EF0E0DF2EF0ECEF2EFFE3C2
:101C6000FF2EF02D0E943FA781E049E750E060E0A1
:101C700070E000EF10E020E030E00F2EFDECCF2E02
:101C8000FCECDF2EFCE4EF2EFEE3FF2EF02D0E9495
:101C90003FA782E041EF50E060E070E008E611E02D
:101CA00020E030E00F2EFDECCF2EFCECDF2EFCE42C
:101CB000EF2EFDE3FF2EF02D0E943FA783E049E6C3
:101CC00051E060E070E00FE711E521E030E00F2E19
:101CD000F0E0CF2EF0E0DF2EF0E0EF2EFFE3FF2E5E
:101CE000F02D0E943FA70E941DA7AC018EE490E05A
:101CF00062E870E00E94041180ED90E069EA0E94C1
:101D0000F9BF0E940A8A81E00E94993A8091760385
:101D100090917703892B21F484E696E20E946F89E3
:101D200000D08DEB95E0EDB7FEB7928381830E94E2
:101D30000EBC8EB18C618EB98DB18C618DB90F9056
:101D40000F900E946EAD0E94F03B0E9465070E94BA
:101D5000358F0E94DDABF7CFDF93CF930F92CDB7D6
:101D6000DEB781E0BE016F5F7F4F41E00E940B1044
:101D7000813019F02FEF3FEF03C08981282F30E029
:101D8000C9010F90CF91DF9108950F931F93DF93B7
:101D9000CF930F92CDB7DEB78E010F5F1F4F81E05B
:101DA000B80141E00E940B108823C9F3898190E0BB
:101DB0000F90CF91DF911F910F9108950F931F9373
:101DC000DF93CF930F92CDB7DEB789838A3071F45A
:101DD0008DE089838E010F5F1F4F81E0B80141E0E4
:101DE0000E9414108823C9F38AE089838E010F5F53
:101DF0001F4F81E0B80141E00E9414108823C9F30D
:101E000080E090E00F90CF91DF911F910F910895A6
:101E10009B01AC016050774F824C9F4FF2E0660F00
:101E2000771F881F991FFA95D1F7E3E0220F331F20
:101E3000441F551FEA95D1F70E9445B52150304007
:101E40003093CD002093CC0082E08093C80086E0E0
:101E50008093CA0088ED8093C9000895DC018091C9
:101E6000C9008F7B8093C9002091B0268091B12654
:101E7000821730F0275F922F981B892F295005C0B9
:101E80002150922F981B892F2F5F482F681708F435
:101E9000462F342F12C09091B126E92FF0E0E4567E
:101EA000F94D8C918083993019F41092B12603C0BA
:101EB0009F5F9093B12631501196332361F7809143
:101EC000B426882351F4E22FF0E0E456F94D8081E6
:101ED0008093CE0081E08093B4268091C900806415
:101EE0008093C900842F0895DC012091B526222318
:101EF00011F480E008958091C9008F778093C90024
:101F00002A3058F08091B3268093B2268AE08093DD
:101F1000B5266A3020F02AE003C0261708F0262FE5
:101F2000322F17C0E091B226F0E0E456F94D8285D9
:101F30008C939091B2269F5F9093B2268091B526A4
:101F400081508093B5269A3011F41092B2261196E2
:101F50003150332339F78091C90080688093C900DC
:101F6000822F08951F920F920FB60F920BB60F9209
:101F700011248F939F93EF93FF939091B3268091B9
:101F8000B5268F5F8093B5268091CE00E92FF0E0D3
:101F9000E456F94D8287993019F41092B32603C0A4
:101FA0009F5F9093B326FF91EF919F918F910F9038
:101FB0000BBE0F900FBE0F901F9018951F920F929F
:101FC0000FB60F920BB60F9211248F93EF93FF93DE
:101FD0008091B026893019F41092B02603C08F5F2B
:101FE0008093B026E091B0268091B126E81739F0B1
:101FF000F0E0E456F94D80818093CE0002C010924B
:10200000B426FF91EF918F910F900BBE0F900FBEF2
:102010000F901F901895813011F080E00895CB014A
:10202000642F0E94740F0895813011F080E00895AC
:10203000CB01642F0E942E0F0895813011F085E8A6
:10204000089560E076E980E090E00E94080F80E06B
:10205000089590938F1780938E17089590939117FA
:1020600080939017089590939317809392170895F3
:102070001F920F920FB60F920BB60F9211242F934F
:102080003F934F935F936F937F938F939F93AF9300
:10209000BF93EF93FF93E0918E17F0918F170995FF
:1020A000FF91EF91BF91AF919F918F917F916F9130
:1020B0005F914F913F912F910F900BBE0F900FBEEC
:1020C0000F901F9018951F920F920FB60F920BB69C
:1020D0000F9211242F933F934F935F936F937F93AE
:1020E0008F939F93AF93BF93EF93FF93E0919017DC
:1020F000F09191170995FF91EF91BF91AF919F9149
:102100008F917F916F915F914F913F912F910F90A0
:102110000BBE0F900FBE0F901F9018951F920F923D
:102120000FB60F920BB60F9211242F933F934F933C
:102130005F936F937F938F939F93AF93BF93EF932F
:10214000FF93E0919217F09193170995FF91EF910A
:10215000BF91AF919F918F917F916F915F914F91BF
:102160003F912F910F900BBE0F900FBE0F901F90BD
:1021700018951F920F920FB60F9211240F900FBE59
:102180000F901F9018951F920F920FB60F92112467
:102190000F900FBE0F901F9018951F920F920FB6C1
:1021A0000F9211240F900FBE0F901F9018951F9241
:1021B0000F920FB60F9211240F900FBE0F901F9029
:1021C00018951F920F920FB60F9211240F900FBE09
:1021D0000F901F9018951F920F920FB60F92112417
:1021E0000F900FBE0F901F9018951F920F920FB671
:1021F0000F9211240F900FBE0F901F9018958FEF24
:102200009FEF0E940112FBCFCF92DF92EF92FF92DD
:102210000F931F93CF93DF938C017B016A01CB0156
:10222000800F911F8150904110F085E816C0C0E0EA
:10223000D0E00FC0C8010E94F1BFF601EC0FFD1FF6
:102240006081861719F0C8010E94F9BF0F5F1F4F08
:102250002196CE15DF0570F380E0DF91CF911F91BD
:102260000F91FF90EF90DF90CF900895CF92DF9283
:10227000EF92FF920F931F93CF93DF938B017A011D
:1022800069018130910531F4862F642FA9010E94E4
:10229000C3151DC0892B11F088EE19C0CA01860F25
:1022A000971F8150904110F085E811C0C0E0D0E048
:1022B0000AC0CE01800F911F0E94F1BFF601EC0F02
:1022C000FD1F80832196CE15DF0598F380E0DF9116
:1022D000CF911F910F91FF90EF90DF90CF900895D5
:1022E0000E94DF1308950E947B110E94C0150E9476
:1022F0009C1180E008959FB7F894E0E0F0E089E059
:102300008093570084919FBF8F70823011F090E0CE
:1023100001C09FE080E80FB6F8948093610090932D
:1023200061000FBE80E1809335018093340180937A
:1023300033018093320108951092941710929517EB
:102340008FEF809396178093971780939817EAEBF7
:10235000F6E29FEF948311821082399687E2EC3582
:10236000F807C1F780E28093B60088EA8093DC002A
:102370008FE08093F4009093F3009093F200909399
:10238000F10082E08093E0008091DF008260809322
:10239000DF0008950895FC018091DE0080FDFCCFF0
:1023A0002091E100822F2091E200922F2091E30002
:1023B000A22F2091E400B22F24E0880F991FAA1FBA
:1023C000BB1F2A95D1F780839183A283B38308959D
:1023D000FC012091E900822F2091EA00922F2091A8
:1023E000EB00A22F2091EC00B22F34E0880F991F50
:1023F000AA1FBB1F3A95D1F780839183A283B38331
:102400000895AC018436910518F060E070E01EC0BC
:102410007FB7F89461E01AC057FD02C09A0102C06C
:102420002FEF3FE7C901880F991F909581959F4F26
:102430009093250180932401FABBE0932101D09B66
:10244000FECF421B530B1092210102C0F1E0E2E0EB
:102450004115510509F761117FBF089520E090E013
:10246000FC01B3E0EE0FFF1FBA95E1F7E80FF91F8B
:10247000EA54F94D84819581892B09F021E0822F5E
:102480000895EF92FF920F931F938091961790E01B
:10249000FC0113E0EE0FFF1F1A95E1F7E80FF91F9B
:1024A000EA54F94DE080F180028113818091941704
:1024B000882309F449C01093F8000093F700F092C4
:1024C000F600E092F5008091DF0080FD08C081E019
:1024D0008093E0008091DF0081608093DF00209195
:1024E000E100822F2091E200922F2091E300A22FA1
:1024F0002091E400B22F9C01AD012F5F3F4F4F4F61
:102500005F4FDA01C9018E259F25A027B127807072
:102510009070A070B87F0097A105B10531F4E21664
:10252000F30604071507B0F018C08FEF9FEFAFEF69
:10253000B7E0E822F9220A231B2357702E153F0526
:102540004007510738F009C08091DF008E7F8093EB
:10255000DF0003C081E0809395171F910F91FF90DA
:10256000EF9008951F931FB7F894809195178823D3
:1025700009F44CC01092951730919417332309F445
:1025800045C0809197178F3F59F4809198178F3FDE
:1025900039F480919617809398178093971712C0FB
:1025A000209196178091981790E0FC0153E0EE0F70
:1025B000FF1F5A95E1F7E80FF91FEA54F94D2087FC
:1025C000209398178091961790E0FC0143E0EE0F5E
:1025D000FF1F4A95E1F7E80FF91FEA54F94D80858E
:1025E000809396178091981790E0FC0123E0EE0FFE
:1025F000FF1F2A95E1F7E80FF91FEA54F94D8FEF15
:1026000080873150309394170E9441121FBF1F9151
:102610000895FF920F931F93182F823110F08AE8CC
:10262000C5C0FFB6F8940E94B2120091941700231F
:1026300009F4C0C040919617242F842F302F121711
:10264000F1F5212F30E0141781F4F901A3E0EE0F2A
:10265000FF1FAA95E1F7E20FF31FEA54F94D8085B9
:10266000809396170E94411218C090E0DC01E3E0CD
:10267000AA0FBB1FEA95E1F7A80FB91FAA54B94DDD
:10268000F90173E0EE0FFF1F7A95E1F7E20FF31FF8
:10269000EA54F94D808518968C93812F90E0FC01C7
:1026A00063E0EE0FFF1F6A95E1F7E80FF91FEA54A8
:1026B000F94D8FEF808701500093941762C0822FED
:1026C00090E0FC0153E0EE0FFF1F5A95E1F7E80F91
:1026D000F91FEA54F94D50853150822F09F46AC030
:1026E000252FADCF1217D1F5209198171317B1F4FC
:1026F000121721F48FEF809398170DC0812F90E06F
:10270000FC0143E0EE0FFF1F4A95E1F7E80FF91FC8
:10271000EA54F94D80858093971733C0842F90E059
:10272000DC0133E0AA0FBB1F3A95E1F7A80FB91FF0
:10273000AA54B94D812F90E0FC0103E0EE0FFF1F7A
:102740000A95E1F7E80FF91FEA54F94D80851896CC
:102750008C931217B1F44093981713C0822F90E016
:10276000FC0173E0EE0FFF1F7A95E1F7E80FF91F08
:10277000EA54F94D422F20852F3F09F0B3CF80E076
:102780000FC0812F90E0FC0163E0EE0FFF1F6A9500
:10279000E1F7E80FF91FEA54F94D1582148281E040
:1027A000FFBE882311F489E801C080E01F910F91DA
:1027B000FF90089530919717232F432FDDCF1F935C
:1027C0000E94B2121FEF25C06FB7F894822F90E0DD
:1027D000FC01B3E0EE0FFF1FBA95E1F7E80FF91F18
:1027E000EA54F94D2085448155818681978110876F
:1027F00015821482178216822F3F09F43FEF6FBFB4
:102800004115510551F03093981720939717FA010D
:10281000099530919817209197172F3FA9F630937B
:102820009817209397171F9108952F923F924F92D8
:102830005F926F927F928F929F92AF92BF92CF9250
:10284000DF92EF92FF920F931F93DF93CF9300D00D
:1028500000D00F92CDB7DEB7582E1801FB82EA8266
:1028600001E1081710F48AE820C12114310409F4A9
:1028700019C190E09D838C83FC01A3E0EE0FFF1F44
:10288000AA95E1F7E80FF91FEA54F94D8481958183
:10289000892B11F088E809C1E4E076956795579592
:1028A0004795EA95D1F72115310529F021303105F9
:1028B00009F0F8C026C0DB01CA010897A109B109D7
:1028C000885F9F4FAF4FB74008F0EEC02091E10006
:1028D000822F2091E200922F2091E300A22F2091DD
:1028E000E400B22F7A018B01E80EF91E0A1F1B1FAC
:1028F0008FEF9FEFAFEFBFE0E822F9220A231B23FF
:1029000020C02091E100822F2091E200922F20919F
:10291000E300A22F2091E400B22F8A019B01081B43
:10292000190B2A0B3B0BD901C801BF700897A109ED
:10293000B109885F9F4FAF4FB74008F0B5C07A012B
:102940008B012FB72983F8946FEF862E6FEF962EA9
:102950006FEFA62E6FE0B62E8E209F20A022B12210
:102960000E94B212609096173FEF631671F040908C
:102970009417C62CD62C77248FEF9FEFAFEFB7E0DC
:10298000E822F9220A231B2367C050929617EC8194
:10299000FD8153E0EE0FFF1F5A95E1F7AC81BD8139
:1029A000EA0FFB1FEA54F94D60865AC0BFEFDB16F1
:1029B00009F44DC06D2D70E0FB0143E0EE0FFF1FE9
:1029C0004A95E1F7E60FF71FEA54F94D208131816E
:1029D00042815381D501C40182279327A427B527BB
:1029E00080709070A070B87F0097A105B10539F490
:1029F000281539054A055B0508F46FC007C05770F4
:102A0000E216F3060407150708F467C0EC81FD81A0
:102A100033E0EE0FFF1F3A95E1F70C811D81E00FC7
:102A2000F11FEA54F94DD0866D1419F4509296179F
:102A300017C08C2D90E0FC0123E0EE0FFF1F2A95BC
:102A4000E1F7E80FF91FEA54F94D508609C08FEFFE
:102A5000DC2C7394CD2CD82E741408F4A7CF49C065
:102A6000EC81FD8193E0EE0FFF1F9A95E1F72C8139
:102A70003D81E20FF31FEA54F94D80829182A282D8
:102A8000B382358224828A819B8197838683809159
:102A900094178F5F809394170E94411299819FBF72
:102AA00080E003C088EE01C08BE80F900F900F907C
:102AB0000F900F90CF91DF911F910F91FF90EF90AA
:102AC000DF90CF90BF90AF909F908F907F906F904E
:102AD0005F904F903F902F900895FB0183E0EE0FA1
:102AE000FF1F8A95E1F7E60FF71FEA54F94D80853D
:102AF000B0CF8C2D90E0FC0103E0EE0FFF1F0A9594
:102B0000E1F7E80FF91FEA54F94D5086EC81FD8199
:102B100013E0EE0FFF1F1A95E1F7AC81BD81EA0FBC
:102B2000FB1FEA54F94D8FEF80879ACF1F920F92C7
:102B30000FB60F9211248F9380919417882319F068
:102B400081E0809395178F910F900FBE0F901F908B
:102B500018951F920F920FB60F9211248F938FEF3B
:102B60008093E4008093E3008093E2008093E1008F
:102B70008F910F900FBE0F901F90189581E00895D0
:102B8000A59A9D9A0895DF93CF93CDB7DEB7C05431
:102B9000D0400FB6F894DEBF0FBECDBFA82FB62F22
:102BA000749A759A6C9A6D9A5E9A5F9A569A579A29
:102BB000A2989A9AA5989D9A84B1876084B983E572
:102BC0008CBDFE0131966E2F93E09E01205C3F4F3D
:102BD0008E2F861BA598000000000000000000005A
:102BE00000000000000000000000000000000000E5
:102BF0000000000000009EBD0DB407FEFDCF8F77E2
:102C00008EBD0DB407FEFDCF1EBC0DB407FEFDCF7B
:102C10008EB5A59A8083E217F30711F03196D8CFCD
:102C20001CBCFE01319620E030E0BE016F5B7F4F9F
:102C300081912827022E2295207F2025032E322FD6
:102C400022952F700226269532272327220F220F46
:102C5000220F2025E617F70759F7232B11F085E8F7
:102C60000CC09E012F5F3F4F2A0F311DCA01B901D1
:102C70004B2F50E00E94D6BA80E0C05CDF4F0FB609
:102C8000F894DEBF0FBECDBFCF91DF910895BC0198
:102C9000009721F08FE59BE10E947E1608958FE555
:102CA0009BE160E070E00E941B1708950F931F9353
:102CB000CF93DF938FE59BE166E00E947616C7E431
:102CC000DBE109E917E1198308838FE59BE1BE0188
:102CD0000E947E16249603561F4F8BE1CF35D807EE
:102CE00091F7DF91CF911F910F910895FC0111820F
:102CF000108213821282158264830895CF93DF932A
:102D0000DC01EB012FB7F89415969C91159714965A
:102D10008C911497981711F48CE819C0992321F419
:102D200011967C936E9306C01296ED91FC911397C9
:102D3000738362831396DC93CE9312971B821A825D
:102D400015968C9115978F5F15968C9380E02FBF09
:102D5000DF91CF9108959F92AF92BF92CF92DF9271
:102D6000EF92FF920F931F93CF93DF938C015B0140
:102D70006A019FB6F894DC0115968C91882319F4AA
:102D8000C0E0D0E04AC0F801C081D18141155105B1
:102D9000B1F07E0111C0D60112966D917C9113970E
:102DA000ED91FC91888199810995882359F47E01E0
:102DB0008A819B819C01E901209769F72EC02097A9
:102DC00061F17E01AB2849F5F801808191812A816A
:102DD0003B81C817D90719F43183208305C0D70177
:102DE00013963C932E931297F80182819381C81712
:102DF000D90711F4F382E282D80115968C911597C8
:102E0000815015968C9315978D919C911197892BD4
:102E100021F413961C921E9212979FBECE01DF9151
:102E2000CF911F910F91FF90EF90DF90CF90BF90C7
:102E3000AF909F900895AB0160E070E00E94AB16E8
:102E40000895AB0161E070E00E94AB160895CF9346
:102E5000DF93EC010BC0CE0160E070E00E941B1715
:102E6000009711F41D8205C00E9447168D818823AA
:102E700091F7DF91CF9108950F931F93DF93CF9335
:102E8000CDB7DEB728970FB6F894DEBF0FBECDBF23
:102E9000809141018F71883029F581E080934F0145
:102EA00089E080934201CE0101960E94CB118E01F0
:102EB0000B5F1F4F80914F0180FD14C0C8010E941D
:102EC000CB118D819E81AF81B88529813A814B815B
:102ED0005C81821B930BA40BB50B8D3D9105A10565
:102EE000B10540F328960FB6F894DEBF0FBECDBFF4
:102EF000CF91DF911F910F910895CF93DF93EC0154
:102F00008091792790917A270F9709F033C08091AB
:102F100039018D7F8093390194E6809141018F7151
:102F20008830C9F0915031F48091390182608093EA
:102F30003901EDCF0000000000000000000000009B
:102F40000000000000000000000000000000000081
:102F500000000000E2CFC830D10519F0C330D10520
:102F600049F488E090E090937A278093792728E0CD
:102F700030E0E1C18091410190E08F7190709093B9
:102F80007A2780937927C830D10509F44FC0C9301A
:102F9000D10560F4C430D10509F49AC0C630D1051A
:102FA00009F4A3C0239709F0B9C157C0CF30D105A8
:102FB00079F0C031D10520F4299709F0AFC164C080
:102FC000C631D10509F4CBC0699709F0A7C136C154
:102FD00083E0809342010E94E2B680936D0180916C
:102FE0006E019770887F982B90936E01000000000F
:102FF00000000000000000000000000000000000D1
:103000000000000000000000000000008091390175
:1030100082608093390183E290E00E940112D09394
:103020007A27C09379272FE030E085C1089709F40B
:1030300075C188E08093420100000000000000009C
:103040000000000000000000000000000000000080
:10305000000000000000000061C1089709F45EC193
:1030600083E08093420100000000000000000000A7
:103070000000000000000000000000000000000050
:103080000000000000004AC18830910539F1893004
:10309000910520F4069709F041C106C086319105DB
:1030A00019F0499709F03AC189E080934201000084
:1030B0000000000000000000000000000000000010
:1030C000000000000000000000000000000026C119
:1030D0008830910519F0099721F420C10E943C170E
:1030E0001DC184E08093420119C18930910569F0C6
:1030F0008A30910520F4089709F010C11AC0863172
:10310000910519F0499709F009C186E080934201C1
:1031100000000000000000000000000000000000AF
:10312000000000000000000000000000000000009F
:10313000F5C00E943C1786E0809342010000000029
:10314000000000000000000000000000000000007F
:10315000000000000000000000000000DFC0883018
:10316000910509F18930910520F4069709F0D6C040
:1031700030C08930910519F0499709F0CFC086E138
:1031800080934201000000000000000000000000E9
:10319000000000000000000000000000000000002F
:1031A00000000000BBC00E943C1786E180934201F2
:1031B000000000000000000000000000000000000F
:1031C00000000000000000000000000000000000FF
:1031D000A5C089E0809342010000000000000000CB
:1031E00000000000000000000000000000000000DF
:1031F000000000000000000080914101282F30E015
:103200002F71307030937A27209379272930310538
:1032100009F091C086E180934201000000000000A7
:10322000000000000000000000000000000000009E
:103230000000000000000000000070C08830910510
:1032400009F457C08930910520F4069709F066C04B
:103250001BC08930910521F0469709F05FC014C06A
:1032600089E180934201000000000000000000009E
:10327000000000000000000000000000000000004E
:103280000000000000004AC089E080934201000075
:10329000000000000000000000000000000000002E
:1032A000000000000000000000000000000080910D
:1032B0004101282F30E02F71307030937A2720930E
:1032C00079272930310509F036C089E18093420120
:1032D00000000000000000000000000000000000EE
:1032E00000000000000000000000000000000000DE
:1032F00015C00E943C1789E1809342010000000044
:1033000000000000000000000000000000000000BD
:10331000000000000000000000000000809141015A
:10332000282F30E02F7130702F313105B9F3209301
:10333000792730937A27C901DF91CF910895809141
:10334000651B9091661B892BA9F48DE90E944F168D
:103350009093661B8093651B892B61F08091692790
:10336000882341F080918327882321F486E190E02F
:103370000E947D1780916F27882351F08AE697E29B
:1033800060E070E00E941B17009711F00E94D119B5
:1033900080918327882321F0823011F40E941C1B26
:1033A0000895EF92FF920F931F93CF93DF937C01C9
:1033B000DC010D911C91D8011696ED91FC911797A7
:1033C000808180937C27C82FD0E02196CE0FDF1F0D
:1033D000988129812D3310F02CE303C0222309F4B6
:1033E00021E092959695969593708FEF989FC001E6
:1033F000112430E0FC01E29FC001E39F900DF29F99
:10340000900D112464EB70E00E941EB56F3F7105B2
:1034100011F008F06FEF6883D8011296FC92EE92DB
:103420001197C8010E948D24DF91CF911F910F91B8
:10343000FF90EF900895CF92DF92EF92FF920F935B
:103440001F93CF93DF93E091651BF091661BC081C2
:10345000D181C0904701D0907B01D7FC34C082E07D
:10346000D80E0DE910E00D191109EEEFDE0E0C0F6C
:103470001D1FED2CFF2497012F5F3F4FC80160E80F
:1034800071E0A9010E94D6BAF801D292FF83EE83BF
:10349000EE0EFF1EF701C2826091651B7091661BE4
:1034A0008AE697E20E947E168DE90E944F1690935D
:1034B000661B8093651B892B31F489E08093420160
:1034C00081E080936927DF91CF911F910F91FF9049
:1034D000EF90DF90CF900895809183278823F1F0BB
:1034E000809142018295869587708093671B109228
:1034F000681B82E0809383278091651B9091661BF7
:10350000892B41F489E090E00E947D1781E080934F
:103510006927089586E190E00E947D170895FF9243
:103520000F931F93CF93DF93EC018B01442349F05A
:1035300090916C01809178278295807F9F70892B74
:1035400003C080916C018F7080936C010230110573
:1035500098F4442369F090916C0180917027880F52
:103560008E70917F892B80936C0110926F0117C030
:1035700080916C018E6011C0809174278295807F4C
:1035800090917727892B80936F0190916C018091A6
:103590007027880F8E70917F892B80936C0189E151
:1035A00090E00E947D174997D1F7FFB6F89401305B
:1035B000110559F480917C27833118F080E492E062
:1035C00002C080E890E00E9401128091390182607F
:1035D00080933901809139018D7F80933901288151
:1035E00030E02150304080E891E0BE01A9010E9406
:1035F000D6BA81E080938327FFBEDF91CF911F91E0
:103600000F91FF900895FC0180918327882311F08A
:1036100086E80895F0937627E09375278681978151
:1036200090937E2780937D27009711F488EE08956C
:103630000E948F1A80E00895109283278091671B63
:103640009091681B83309105B9F08430910528F47E
:10365000009731F00197E1F409C00597C9F412C051
:10366000609175277091762780E017C0609175276B
:103670007091762787E811C0609175277091762741
:1036800081EE0BC0609175277091762789EE05C099
:10369000609175277091762785E80E941535089509
:1036A000282F85FD03C0982F9F7304C0982F9195F4
:1036B0009F719195E6EFF5E08491891734F03F967C
:1036C0008491981714F0822F0CC0803E3CF0803219
:1036D0003CF487FF06C08F71806203C080E201C0A6
:1036E0008FE18068089584E08093702723E0209321
:1036F00077278FEF9FEF90936527809364279093B0
:103700006827809367278BE0809372271092632746
:1037100080E098EFAFEFB7E080937F27909380270A
:10372000A0938127B09382278AE091E0909362274B
:10373000809361278AE080937B2782E080937127C2
:1037400085E0809374272093782783E80E94501B9C
:103750008093582781E080936627109273270895FD
:1037600085FD03C0982F9F7304C0982F91959F717A
:103770009195E6EFF5E080E02491921724F0291767
:103780003CF4815008958F5F31968031A9F780E035
:1037900008958091642790916527809362019093AA
:1037A0006301E9E5F7E2A4E6B1E081918D9387E258
:1037B000E136F807D1F780916727909168278093C9
:1037C00060019093610190914801809166278295F4
:1037D000880F80769F79892B8093480190916F01A3
:1037E000809177278F70907F892B80936F019091C4
:1037F0006E0180917327880F880F880F8870977FDC
:10380000892B80936E0190916F018091742782952E
:10381000807F9F70892B80936F01909148018091E8
:1038200072278F71907E892B809348018091582751
:103830000E94B01B909145018F70907F892B8093DF
:1038400045010895CF93DF93EB018E3431F0893534
:1038500041F4888180937827EFC088818093702716
:10386000EBC02091792730917A272F30310511F460
:1038700081E8E3C08B3009F4CDC08C3070F4823025
:1038800009F487C0833018F48823B1F115C0833060
:1038900009F490C0843081F466C0833511F1843519
:1038A00028F48F3459F0803539F410C0873509F485
:1038B00064C0803F09F48BC084EFBFC098819093AF
:1038C000772780916F019F70807F5FC08881998189
:1038D000809364279093652780936201909363019E
:1038E000ABC08881998180936727909368278093E4
:1038F000600190936101A0C080918327882309F023
:1039000097C080E098EFAFEFB7E0088004C0B695AD
:10391000A795979587950A94D2F781709070892B17
:1039200009F488C02830310519F428E030E008C0D7
:1039300088E090E00E947D170897D1F726E130E0FB
:10394000988190937227809148019F71807E982B77
:10395000909348012830310509F46EC086E190E06B
:103960000E947D1769C080918327882309F060C079
:103970008881882309F460C05DC098819093742782
:1039800080916F019295907F8F70982B90936F012B
:1039900053C08881809358270E94501B80935827DA
:1039A0000E94B01B909145018F70907F892B80936E
:1039B000450142C088818093662790914801829595
:1039C000880F80769F79892B8093480135C0888144
:1039D00080935927898180935A278A8180935B2716
:1039E0008B8180935C278C8180935D278D81809370
:1039F0005E278E8180935F278F8180936027E9E522
:103A0000F7E2A4E6B1E081918D9387E2E136F80711
:103A1000D1F712C088818093732790916E01880F2F
:103A2000880F880F8870977F892B80936E0104C060
:103A300086E803C088EE01C080E0DF91CF91089551
:103A4000DF93CF930F92CDB7DEB781E090E065E1D1
:103A500070E041E050E09E012F5F3F4F0E94361121
:103A6000809139018D7F8093390180EF90E00E9431
:103A70000112809139018E7F8093390181E090E0BD
:103A80000E9401128091390181608093390120E008
:103A900030E0809141012F5F3F4F93E0293E39078D
:103AA00011F485E815C090E08F7190708830910511
:103AB00081F790937A27809379279981992339F018
:103AC000809152019F70807F982B9093520180E0EB
:103AD0000F90CF91DF9108950E94E2B680936D011F
:103AE000EEE6F1E080819770887F982B908380E0EC
:103AF0000E94031F0E94F11E0895882311F00E9466
:103B0000731B0E94201D882311F085E80895809181
:103B10006E01806280936E018CE480934E010E945E
:103B20006C1D80916F27882359F40EC08AE697E2B6
:103B300060E070E00E941B17009711F00E9447168A
:103B400080916F27882391F70E94C91B10928327C9
:103B50001092692788E080934F0180E480934F01A1
:103B600084E080934F010E940E3C80E008950F9303
:103B70001F93CF93DF930E947311882309F00CC128
:103B800080913901816080933901809139018D7F65
:103B9000809339018CE791E00E94011280913901F4
:103BA0008E7F8093390181E090E00E940112809124
:103BB000390181608093390188E08093420120E0DF
:103BC00080914101215009F4E7C090E08F7190701D
:103BD00088309105A9F790937A278093792780916F
:103BE0005C01833809F0D8C0DDC080916E0180622D
:103BF00080936E018CE480934E0186E090E00E94F9
:103C00007D1710924E01C0E0D0E010E08091460197
:103C1000CC0FDD1FCC0FDD1F90E08076907025E08B
:103C2000969587952A95E1F7C82BD92B1F5F1830F9
:103C300069F783E090E00E947D1780914F01109317
:103C40004F0180E480934F018CE480934E01CE01BC
:103C50000E94E7B60E946C1D09C0C9E5D7E20E9428
:103C6000E2B6899387E2C136D807C9F78091592710
:103C700030915A2740915B2760915C2770915D27B6
:103C8000F0915E27B0915F2750916027082F015077
:103C900091E0081708F090E0832F815021E083170E
:103CA00008F020E0192F180F91E0181708F090E0A5
:103CB000292B842F815031E0841708F030E0A22FA7
:103CC000A80F91E0A81708F090E0392B862F8150BB
:103CD00021E0861708F020E0E32FE80F91E0E817D5
:103CE00008F090E0292B872F815031E0871708F0EA
:103CF00030E0622F680F91E0681708F090E0392BF0
:103D00008F2F815021E08F1708F020E0432F480FBC
:103D100091E0481708F090E0292B8B2F815091E01B
:103D20008B1708F090E0322F380F21E0381708F099
:103D300020E0922B5195591779F43F3F69F44F3F9A
:103D400059F46F3F49F4EF3F39F4AF3F29F41F3F77
:103D500019F40E3F08F081CF89EE9EE10E942E10EB
:103D600081EE9EE10E9429100E9456168DE90E9464
:103D70004F169093661B8093651B8AE697E265E079
:103D80000E9476160E94731B0E94C91B1092832703
:103D90001092692780E001C085E8DF91CF911F91E3
:103DA0000F91089580E090E060E070E048E050E01E
:103DB00029E537E20E9436110E94201D882361F711
:103DC00014CF1F931FB7F8940E946C1A1FBF1F9146
:103DD00008951F931FB7F8940E941B1A1FBF1F91CD
:103DE00008958091792790917A270F9711F082E8B2
:103DF000089588E090E00E947D17089711F085E80B
:103E0000089580E00895882311F088EE0895809148
:103E1000792790917A270F9711F481E8089580917E
:103E20008327882391F41092692788E090E00E940C
:103E30007D170897D1F78FE090E00E947D170F97CC
:103E400021F40E940E3C80E0089586E80895982FA2
:103E500080918327882311F086E80895983041F4F3
:103E600088E090E00E947D171092692788E008950D
:103E70008091651B9091661B892B31F086E190E063
:103E80000E947D1786E0089581E08093692786E08F
:103E90000895CF93DF93DC019C9111962C9111979B
:103EA00080918427882321F4CD010E9447161AC0EF
:103EB000E92FF22F9F012F5F3F4F47E458E288E040
:103EC000EA010990AE01E90109929E018150C1F712
:103ED00080915928818783E180838DEA98E2BD0132
:103EE0000E947E16DF91CF910895DC01ED91FC9147
:103EF000119784E180836383528341838DEA98E242
:103F0000BD010E947E1608950F931F93DF93CF93F8
:103F100000D0CDB7DEB7A091E727B091E827ED91AB
:103F2000FC91119784E180838BEE83830FEF1FEF69
:103F3000128301838DEA98E2BD010E947E161092E1
:103F4000D5271A83098380E5BE016F5F7F4F0E94EA
:103F5000402F10931E2800931D2810922C28109299
:103F60002D2810922E2810922F281092302810926F
:103F7000312810923228109233280E948A2D0F90F7
:103F80000F90CF91DF911F910F910895EF92FF92C3
:103F90000F931F93E0902828F090292880E061E09B
:103FA00040E020E030E000E010E00E94B7278823E6
:103FB000A9F4A091E727B091E827ED91FC91119722
:103FC00084E1808381EE83838FEF9FEF92838183EF
:103FD0008DEA98E2BD010E947E1619C0A70160E03B
:103FE00070E084E0440F551F661F771F8A95D1F754
:103FF00080E020E030E004E81FE1EE24FF240E948E
:104000001514882321F080E090E00E94841F1F9106
:104010000F91FF90EF900895FF920F931F93DF93FE
:10402000CF9300D0CDB7DEB7F0905B280E94471643
:10403000FF20B1F583E569E578E20E94402F2091E9
:10404000592830915A288091472880932C288091B4
:10405000482880932D288091492880932E2880918C
:104060004A2880932F2880914B2880933028809174
:104070004C288093312880914D288093322880915C
:104080004E288093332881E0809363281092D527AF
:104090008091E127833031F582E08093E12722C0CF
:1040A0001092D5270FEF1FEF1A83098380E5BE0119
:1040B0006F5F7F4F0E94402F10931E2800931D2892
:1040C00010922C2810922D2810922E2810922F2812
:1040D00010923028109231281092322810923328F2
:1040E0002FEF3FEFE091E727F091E827A081B18122
:1040F00084E18C931396FC92139712963C932E9323
:1041000011978DEA98E2BF010E947E160E948A2DC7
:104110000F900F90CF91DF911F910F91FF90089515
:10412000CF92DF92EF92FF920F931F93DF93CF9383
:10413000CDB7DEB72C970FB6F894DEBF0FBECDBF5C
:10414000D82EC92E082F192FDE011196F801808173
:1041500091819C01F9018CE001900D928150E1F771
:10416000D801ED90FC90809163288250823020F03D
:10417000C8010E9447165AC082E0F7018083D70128
:10418000A956BF4FFD0181938A859B8512969C930A
:104190008E9311978C8582839D0128503040D901E0
:1041A000E9E5F7E288E001900D928150E1F7F9012D
:1041B00038979F01AE014E5F5F4F88E0DA010D90A6
:1041C000AD01D9010D929D018150C1F78091642705
:1041D00090916527929382938091E22782938F5FDB
:1041E0008093E22783E69CEC929382938BE1829307
:1041F000D7011796FC93EE93169786E897E2B801DD
:104200000E947E168C3829F481EFB8010E94952D0A
:104210000DC08D2D9C2D0E94F62C81E00E942E1247
:10422000882311F40E94212AF70114822C960FB6DC
:10423000F894DEBF0FBECDBFCF91DF911F910F91DC
:10424000FF90EF90DF90CF900895EF92FF920F9341
:104250001F93DF93CF93CDB7DEB72F970FB6F894A8
:10426000DEBF0FBECDBFAC018C01DE011196FC019B
:10427000808191819C01F9018FE001900D92815024
:10428000E1F74093E7275093E8278C81823019F4B7
:104290008F8198851AC08F8180932C288885809380
:1042A0002D28898580932E288A8580932F288B85B9
:1042B000809330288C85809331288D858093322897
:1042C0008E85809333288EEF9FEF90931E288093E6
:1042D0001D2880E5BE016B5F7F4F0E94402F8091BB
:1042E000AB28813011F40E94652DD801ED90FC902F
:1042F00081E0F701808312830183E756FF4F8083BB
:104300008F8581839F0128503040D901E9E5F7E28C
:1043100088E001900D928150E1F7F9018FEF9FEF56
:10432000929382938C81823051F480911D289091D8
:104330001E289293829345E123E238EC11C0F901E3
:104340003A979F014CE258E288E0DA010D90AD0106
:10435000D9010D929D018150C1F74BE123E23CEC64
:104360008091642790916527929382938091E227B0
:1043700082938F5F8093E227329322934293D701F7
:104380001796FC93EE93169780E0BE016E5F7F4F09
:104390000E94402F84E0BE016D5F7F4F0E94402F3E
:1043A000882361F4C70162E070E041E00E94031BD2
:1043B000882321F481E08093642812C0D801ED9114
:1043C000FC9184E1808381EE83838FEF9FEF928362
:1043D00081838DEA98E2B8010E947E160E948A2DA0
:1043E0002F960FB6F894DEBF0FBECDBFCF91DF91F1
:1043F0001F910F91FF90EF900895DC011696ED91BB
:10440000FC91179782818695869583708330A9F4F5
:104410008091691B90916A1B089790936A1B809307
:10442000691BDC01369688E001900D928150E1F71E
:1044300080916B1B8F5F80936B1B80E00895FC0164
:10444000A681B78112968C91129786958695837076
:104450008230A1F4E091691BF0916A1B3297F093CE
:104460006A1BE093691B16968D919C911797918317
:10447000808380916B1B8F5F80936B1B80E008951E
:10448000AF92BF92CF92DF92EF92FF920F931F9362
:10449000DF93CF9300D000D0CDB7DEB7FB01A08073
:1044A000B180D50112967C936E9311978AE08C931C
:1044B0007BE9C72ED12CCA0CDB1C8091E327882313
:1044C00019F46DE0E62E0EC0482F50E0C41AD50A4C
:1044D0005DE0E52EE80E29EE37E2C601B90150E0B5
:1044E0000E94D6BAD0926A1BC092691B10926B1BB5
:1044F0008FE192E29A83898386E897E28E010F5FCB
:104500001F4FB8010E942117F0906B1B10926B1B7C
:104510008DEF91E29A83898386E897E2B8010E9441
:10452000211780916B1BE091691BF0916A1B3197F9
:1045300090E09C0144E0220F331F4A95E1F72F29B8
:104540002083880F991F880F991F8F0D911D880F49
:10455000991F80936B1B4E2D480FE82FF0E0E095DC
:10456000F095EC0DFD1D129280916328833019F4B3
:104570002FEF3FE402C02FEF3FE0809184278111AD
:104580003068DF013E932E938091672790916827D2
:104590002FEF8E3F920789F43A974A5F9F0169E5B2
:1045A00077E288E0DB010D90BD01D9010D929D01FC
:1045B0008150C1F720E030EC05C0FD019293829359
:1045C00020E030E880916427909165279293829350
:1045D0008091E02782938F5F8093E027329322932C
:1045E0004293D5011796FC93EE931697C50162E0AE
:1045F00070E040E00E94031B81E0809364280F90EC
:104600000F900F900F90CF91DF911F910F91FF901E
:10461000EF90DF90CF90BF90AF900895BC0180E005
:104620000E94402208950F931F938C01DC01ED91AD
:10463000FC9181810E946F3FC8010E9447161F9123
:104640000F9108950F931F938C01DC01ED91FC9164
:10465000818162810E94BD42C8010E9447161F915C
:104660000F910895AF92BF92CF92DF92EF920F9386
:104670001F935C01DC01ED91FC9104811581268181
:104680003781818162814381E08439966F010E9484
:10469000A243C5010E9447161F910F91EF90DF9032
:1046A000CF90BF90AF9008950F931F938C01DC01C2
:1046B000ED91FC9181810E949842C8010E944716A9
:1046C0001F910F9108950F931F938C01DC01ED91C1
:1046D000FC9181810E94423FC8010E9447161F91B0
:1046E0000F9108950F931F938C01DC01ED91FC91C4
:1046F000818162813396AF010E941B43C8010E94F1
:1047000047161F910F9108950F931F93DF93CF9337
:10471000CDB7DEB766970FB6F894DEBF0FBECDBF3C
:104720008C01DC01ED91FC91818192819B838A83D4
:10473000838189839E012C5F3F4FAF014C5F5F4FA8
:1047400088E0DA010D90AD01D9010D929D018150F3
:10475000C1F7818192819E878D8784858C879E0198
:10476000215F3F4FAF01435F5F4F88E0DA010D905B
:10477000AD01D9010D929D018150C1F7CE01019685
:10478000BE01645F7F4F45890E946D3FC8010E9452
:10479000471666960FB6F894DEBF0FBECDBFCF9119
:1047A000DF911F910F910895CF92DF92EF92FF92C8
:1047B0000F936C01DC01ED91FC91BF016E5F7F4FA7
:1047C00024893589E788F08C8181438906890E9494
:1047D000403FC6010E9447160F91FF90EF90DF9077
:1047E000CF900895EF92FF920F937C01DC01ED9141
:1047F000FC91218132814381548165817681878159
:10480000908501850E943744C7010E9447160F9189
:10481000FF90EF9008950F931F938C01DC01ED91B1
:10482000FC918181928163810E948142C8010E9432
:1048300047161F910F9108950F931F938C01DC0170
:10484000ED91FC91818162810E94443FC8010E94E8
:1048500047161F910F9108956F927F928F92AF929A
:10486000CF92EF920F93DF93CF93CDB7DEB76697DA
:104870000FB6F894DEBF0FBECDBF3C01DC01ED9159
:10488000FC9181818983828193819B838A839E01AC
:104890002C5F3F4FAF014C5F5F4F88E0DA010D9016
:1048A000AD01D9010D929D018150C1F784858C879E
:1048B000858596859E878D879E01215F3F4FAF013D
:1048C000415F5F4F88E0DA010D90AD01D9010D9293
:1048D0009D018150C1F7258D368DCE010196BE0117
:1048E000645F7F4F448D0789E08CC18CA28C838CE0
:1048F0000E94F444C3010E94471666960FB6F894CE
:10490000DEBF0FBECDBFCF91DF910F91EF90CF9063
:10491000AF908F907F906F900895FC01108261811D
:1049200072816115710521F082E298E20E947E1683
:104930000895AF92BF92CF92DF92EF92FF920F93C2
:104940001F93DF93CF930F92CDB7DEB77C01FC01AD
:10495000A080B180F501A681B7813C9130933728C2
:10496000FD01E30FF11D8181809357281196CD90B1
:10497000DC901297D0923528C092342813968C91EF
:10498000139780933828AD014C5F5F4F7D2D729552
:104990007695769573706D2D66956695637019F4AE
:1049A000FA0120E049C014968D919C91159790933F
:1049B0003B2880933A28FD0136966230E1F410924C
:1049C0003C2810923D2810923E2810923F281092C9
:1049D000402810924128109242281092432816969F
:1049E0008D919C91179790933D2880933C28FD01D1
:1049F000389624E021C0633011F022E01DC01696E5
:104A00008C91169780933C28818180933D288281E8
:104A100080933E28838180933F288481809340281F
:104A20008581809341288681809342288781809365
:104A30004328FD013E962AE0772309F447C0C6FCCF
:104A400008C08191919190934628809345282E5FCC
:104A500008C080913A2890913B28909346288093F3
:104A600045287230C1F410924728109248281092BD
:104A7000492810924A2810924B2810924C281092E4
:104A80004D2810924E2880819181909348288093E0
:104A900047282E5F1BC07330C9F48081809347285C
:104AA00081818093482882818093492883818093E3
:104AB0004A28848180934B28858180934C28868165
:104AC00080934D28878180934E28285F3550321B74
:104AD0003093582870934428609339288A01020F34
:104AE000111D8C2D877080933628833021F4F801B6
:104AF0008081809356281982C3FE0DC0F50166811E
:104B000077816F5F7F4F84E398E2A8019E012F5F5A
:104B10003F4F0E941CA230913628313009F461C009
:104B2000313020F0333009F04DC16FC02981F801D8
:104B3000E20FF11D8081918190935A28809359282A
:104B4000822F8E5F8983F801E80FF11D80818093A9
:104B50005B282D5F29832350877019F02C5F280F65
:104B600029838981F801E80FF11D908190935C28D9
:104B7000482F4F5F4983292F2770892F90E0807736
:104B8000907034E0959587953A95E1F7382F222378
:104B900011F48823A1F0C801840F911D90935E2821
:104BA00080935D28222319F0220F240F29833323B9
:104BB00031F0330F330F330F8981380F39838091F0
:104BC00058289981981750F4891B80935F28090F02
:104BD000111D1093612800936028F8C010925F287F
:104BE000F5C080915828882369F0863718F086E749
:104BF000809358288981080F111D10935A2800931B
:104C00005928E4C010925828E1C081E0898320919E
:104C10005628243009F4DAC0253030F4213059F018
:104C2000223009F0CFC00DC0273009F4CFC02830A2
:104C300009F0C8C012C0F80181818093592882E030
:104C40002EC0F8018181928190935A28809359282F
:104C50003983838180935B28B9C0F8018181928177
:104C600090935A2880935928398383819481909313
:104C70005C2880935B2885E08983858180935D280B
:104C800086E089838681978190935F2880935E2850
:104C90002983D4FE9BC080858093602889E0898326
:104CA00095C080913628833061F4809156288430F5
:104CB00011F0873031F482E298E2B7010E947E164B
:104CC0008BC08091D527813009F467C0813020F0F6
:104CD000843008F077C03AC08091DF27882341F5FF
:104CE00090916328933090F0933009F06BC08091DD
:104CF0003628813009F462C0833009F063C08091A6
:104D000056288430B9F1873079F543C08091362830
:104D1000813009F453C0833009F054C08091562883
:104D2000843041F1873001F5923009F04BC031C039
:104D3000823019F0843009F045C0809136288823EC
:104D400009F040C0C7010E94823346C00E94E83289
:104D500080913628813091F18330A1F580915628D9
:104D6000843041F0873089F0813061F5C7010E94BD
:104D7000491F32C080918B27882321F0C7010E94F0
:104D80007A282AC00E945E271DC080916328823045
:104D9000C9F4C7010E940E231FC0809136288330BA
:104DA00059F480915628823069F480E00E940913FA
:104DB000C7010E940C2010C0813021F4C7010E945D
:104DC0003D2A0AC0C7010E94471606C08091642888
:104DD000882309F066CF75CF0F90CF91DF911F9197
:104DE0000F91FF90EF90DF90CF90BF90AF9008951C
:104DF000CF93DF93DB01EC01EE81FF818281869509
:104E000086958370823011F040E009C040E02D911A
:104E10003C91868197812817390709F441E0842F56
:104E2000DF91CF910895CF93DF93DB01EC01EE8109
:104E3000FF818281869586958370833011F020E012
:104E40002FC020E09C918681981751F511969C9176
:104E500011978781981721F512969C91129780855A
:104E60009817F1F413969C91139781859817C1F4C4
:104E700014969C9114978285981791F415969C919D
:104E800015978385981761F416969C9116978485DB
:104E9000981731F417969C918585981709F421E0AD
:104EA000822FDF91CF910895FB0140E02081318175
:104EB0002817390709F441E0842F08950F931F93B1
:104EC000CF93DF938DE90E944F168C01009709F470
:104ED00049C0DC014D915C918CE0FA018083128322
:104EE0000183E556FF4F80914428833069F4389759
:104EF000EF01A7E4B8E288E00D9009928150E1F754
:104F00006FE021E03CE009C080914728909148285B
:104F10009293829369E021E038E080914528909156
:104F20004628929382938091E22782938F5F8093A9
:104F3000E227329322936293DA011796FC93EE9361
:104F40001697F8018081918161E070E040E00E9455
:104F5000031B882321F481E08093642803C0C801E7
:104F60000E944716DF91CF911F910F9108956F9284
:104F70007F929F92AF92BF92CF92DF92EF92FF9279
:104F80000F931F93CF93DF93D82E962EC42E5901E3
:104F900038018DE90E944F167C01009709F49BC0EF
:104FA000DC010D911C91DD2021F084E0F80180836B
:104FB00003C08BE0D8018C93F801F282E182E656BF
:104FC000FF4F84E080832091672730916827C901D3
:104FD0000296029710F0992069F03897EF01A9E541
:104FE000B7E288E00D9009928150E1F762E183E237
:104FF00090EC05C0329322936CE083E290E8CC20E1
:1050000061F020916427309165276216730629F0BC
:105010006E5F3293229370E002C0806471E022E000
:10502000C21641F4AC015860D5018D919C919293C8
:10503000829328C0B3E0CB1661F4AC015C60389772
:105040006A5FEF01D50188E00D9009928150E1F788
:1050500019C020911D2830911E284FEF2E3F340794
:1050600029F0AC015860329322930CC0AC015C6013
:1050700038976A5FEF01ACE2B8E288E00D900992E0
:105080008150E1F73297772339F08091642790912E
:1050900065279183808302C0718260828091E227BC
:1050A00082938F5F8093E227529342936293D80159
:1050B0001796FC93EE931697C80162E070E041E00A
:1050C0000E94031B882321F481E08093642804C09C
:1050D000C7010E94471680E0DF91CF911F910F9189
:1050E000FF90EF90DF90CF90BF90AF909F907F9018
:1050F0006F900895DF92EF92FF920F931F93DF93CB
:10510000CF9300D000D0CDB7DEB7109262280E94B6
:10511000471680916328823008F4BDC080914428EE
:10512000823021F0833009F0B6C003C088EF96E2E8
:1051300002C083E197E29A83898387E498E29C83A3
:105140008B8386E897E2BE016F5F7F4F0E94211735
:10515000BC01009789F0DC014D915C91DA01169653
:10516000ED91FC9117972091452830914628848134
:1051700095812817390719F00E945E278CC081E0BD
:10518000FA01848380914428823021F0833009F031
:105190006DC023C02091472830914828A2EBB7E288
:1051A00014968C911497882391F0ED91FC911197AE
:1051B0000190F081E02D8481882349F40680F781F5
:1051C000E02D868197812817390709F441C015968B
:1051D000E7E2A53DBE0721F749C0D0904728E090FF
:1051E0004828F090492800914A2810914B28309186
:1051F0004C2820914D2890914E28A2EBB7E21496AE
:105200008C911497882369F1ED91FC91119701908D
:10521000F081E02D8481882321F50680F781E02D3F
:1052200086818D15F1F487818E15D9F480858F15CF
:10523000C1F481858017A9F48285811791F4838553
:10524000831779F48485821761F48585891749F479
:10525000DA011696ED91FC91179781818061818327
:1052600005C01596E7E2A53DBE0749F6DA0114969A
:105270001C92149712967C936E931197CA0161E069
:1052800070E040E00E94031B882329F481E08093B2
:105290006428809362280F900F900F900F90CF9109
:1052A000DF911F910F91FF90EF90DF900895DC0147
:1052B000ED91FC911197E081E43278F4F0E0EE0F8B
:1052C000FF1FEA5FF94F259134912115310519F03F
:1052D000F901099508950E94471608951F9380913A
:1052E0006428882381F48091DE27882361F089ED8A
:1052F00097E260E070E00E941B17009721F00E9487
:10530000572911E001C010E080912728882359F027
:1053100082E298E260E070E00E941B17009719F0AB
:105320000E94572911E0812F1F910895DC01ED9112
:10533000FC91119780E18083418362838DEA98E23A
:10534000BD010E947E1608957F928F929F92AF9228
:10535000BF92CF92DF92EF92FF920F931F93DF9352
:10536000CF9300D000D0CDB7DEB702EB17E294E5C3
:10537000892E97E2992E5E010894A11CB11C80E150
:10538000782ED80114968C9114978823C9F112961F
:105390008D919C911397019713969C938E931297DE
:1053A000892B71F514961C921497ED90FC90F701DF
:1053B000C080D1809A828982FC82EB8286E897E263
:1053C000B5010E941B17D6018C91823019F08D30E7
:1053D000A1F405C080EFB7010E94952D0EC0F60123
:1053E0008381D701ED91FC917082818380EF82836C
:1053F0008DEA98E2B7010E947E16F80111821082B0
:105400000B5F1F4FF7E2053D1F0709F0BACF0E945F
:10541000192D80918B27882311F00E94212A0F904B
:105420000F900F900F90CF91DF911F910F91FF90F0
:10543000EF90DF90CF90BF90AF909F908F907F9034
:105440000895EF92FF920F931F9381E040E050EE9A
:1054500061E070E020E030E004EA19E2EE24FF248D
:105460000E941514882321F080E090E00E94A42976
:105470001F910F91FF90EF9008950F931F93DF936B
:10548000CF93CDB7DEB728970FB6F894DEBF0FBE27
:10549000CDBFAC01DC019C9111962C9180915828D4
:1054A000882321F4CA010E94471605C1E92FF22F73
:1054B00080913828808F8091442881838250823067
:1054C000A8F48091452890914628938382839F0178
:1054D0002C5F3F4F67E478E288E0DB010D90BD016F
:1054E000D9010D929D018150C1F70AC01382128229
:1054F00014821582168217821086118612861386F0
:10550000208D80918527281761F594818091A827A7
:10551000981739F595818091A927981711F59681EB
:105520008091AA279817E9F497818091AB27981763
:10553000C1F490858091AC27981799F4918580915A
:10554000AD27981771F492858091AE27981749F48A
:1055500093858091AF27981721F4CA010E944716BE
:1055600060C02093852784818093A82785818093BC
:10557000A92786818093AA2787818093AB2780857E
:105580008093AC2781858093AD2782858093AE2759
:1055900083858093AF278091392884878250823019
:1055A000A8F480913A2890913B28968785879F019F
:1055B000215F3F4F6CE378E288E0DB010D90BD0195
:1055C000D9010D929D018150C1F70AC0168615863A
:1055D0001786108A118A128A138A148A158A168AE3
:1055E00080915728878B80914F288770818F809179
:1055F0004F288695869586958370828F8091552851
:10560000838F80915828848F8091592890915A28AF
:10561000968F858F81E180838DEA98E2BA010E949E
:105620007E168091342884FF46C0809163288330A1
:1056300009F443C080914428823071F48091472856
:10564000909148289A838983009145281091462893
:1056500080E060E042E021C0833019F58091472866
:105660008983809148288A83809149288B838091FF
:105670004A288C8380914B288D8380914C288E837F
:1056800080914D288F8380914E28888700914528EE
:105690001091462880E060E043E09E012F5F3F4F7D
:1056A00007C080E060E040E020E030E000E010E093
:1056B0000E94B72702C00E948A2D28960FB6F89440
:1056C000DEBF0FBECDBFCF91DF911F910F91089527
:1056D000AF92BF92CF92DF92EF92FF920F931F9300
:1056E000DF93CF93CDB7DEB768970FB6F894DEBFE0
:1056F0000FBECDBFB82EA92E082F192FDE0114968C
:10570000F801808191819C01F90185E101900D9260
:105710008150E1F78A8982FD11C08091D5278823C5
:1057200021F48091DF27882349F09989D801ED91F0
:10573000FC9180E18083918381EE0BC1F801E080D0
:10574000F1808DE0D7018C93898913968C938E8993
:105750008B5F898385502BE9C22ED12CC81AD108C2
:10576000CE0CDF1CDB82CA828B89882371F0CE01CC
:105770000296BE016C5F7F4FAE014F5F5F4F0E948C
:10578000B5A1282F882309F0C2C08D81823079F419
:10579000EA81FB813297FB83EA8389818E5F89836B
:1057A00080916727909168279183808313C083300D
:1057B00089F42A813B81285030403B832A838981A8
:1057C000885F8983D901E9E5F7E288E001900D92CD
:1057D0008150E1F720916427309165278F8198856A
:1057E0002817390749F48D81882331F08E81882369
:1057F00019F040E450E00FC08D81882351F0EA8118
:10580000FB813297FB83EA8389818E5F89833183B1
:10581000208340E050E03E81332349F18A819B811F
:105820002981323059F4FC013297FB83EA832E5FE1
:10583000298389859A85918380830DC008979B83EE
:105840008A83285F2983FC01DE01199688E00D9088
:1058500001928150E1F7EA81FB813297FB83EA8371
:1058600089818E5F89838F81988591838083EA8186
:10587000FB813197FB83EA838091E22780838F5FEE
:105880008093E227BA0161608B89882319F0BA01FD
:10589000696070618A8980FD60628E89873608F050
:1058A00070618E81382F330F330F20E04D81942F9C
:1058B0009295990F990F907C80E0282B392B8A8143
:1058C0009B81FC013297FB83EA83262B372B3183A4
:1058D0002083298127FF02C025EE19C0FC013397E0
:1058E000FB83EA8320838A819B81F70197838683E8
:1058F0008B89882309F465C0C701B601AE014C5FEE
:105900005F4F0E9489A3282F882309F45AC08989F0
:10591000D801ED91FC9190E19083818322838DEAFF
:1059200098E2B8010E947E1650C080916328825090
:105930008230F8F486E897E2B8010E947E168C382F
:1059400051F49989D801ED91FC9180E18083918394
:1059500081EF8283E4CF8B2D9A2D0E94F62C81E07B
:105960000E942E12882311F40E94212AF70114822A
:105970002CC08091AB28813011F40E94652DD70195
:1059800012961C930E931197C70162E070E041E0FC
:105990000E94031B882321F481E08093642815C0B2
:1059A0009989D801ED91FC9180E18083918381EE0A
:1059B00082838DEA98E2B8010E947E160E948A2DA9
:1059C00004C08A8982FFD5CFB0CF68960FB6F8940D
:1059D000DEBF0FBECDBFCF91DF911F910F91FF9022
:1059E000EF90DF90CF90BF90AF900895AC01E6EBC1
:1059F000F7E220E030E080818823A1F4F901EE0F86
:105A0000FF1FEE0FFF1FE20FF31FEE54F84D8091C2
:105A1000E4279091E527938382835183408381E03B
:105A2000848308952F5F3F4F35962730310519F74E
:105A3000089520E001C0292F822F90E0FC01EE0F95
:105A4000FF1FEE0FFF1FE80FF91FEE54F84D848182
:105A5000922F9F5F882379F7392F41E033C0832F3E
:105A600090E0DC01AA0FBB1FAA0FBB1FA80FB91F34
:105A7000AE54B84D14968C911497882311F1822F4F
:105A800090E0FC01EE0FFF1FEE0FFF1FE80FF91F64
:105A9000EE54F84D44838D919C91119791838083AE
:105AA00012968D919C9113979383828314961C92E6
:105AB000149711961C921E9213961C921E92129786
:105AC0002F5F3F5F373058F208958091AB288130C7
:105AD00051F40E94F11E853831F081E090E00E947F
:105AE000CA111092AB2808958091AB28882389F4BD
:105AF00080E090E00E94CA1180E00E94031F88238A
:105B000021F481E08093AB28089581E090E00E9429
:105B1000CA11089580918C27882331F480911F2821
:105B2000882311F40E94742D0895DF93CF93CDB78D
:105B3000DEB728970FB6F894DEBF0FBECDBF482F53
:105B40009B01DB01ED91FC910680F781E02DDE01E8
:105B50001196369688E001900D928150E1F7D901B7
:105B6000ED91FC918CE18083809164279091652771
:105B70009283818393E093838091592784838091DA
:105B80005A27858380915B27868380915C27878352
:105B900080915D27808780915E27818780915F2734
:105BA00082878091602783879487898185878A810E
:105BB00086878B8187878C81808B8D81818B8E817D
:105BC000828B8F81838B8885848B458B8DEA98E2CD
:105BD000B9010E947E1628960FB6F894DEBF0FBE5C
:105BE000CDBFCF91DF9108950F931F93082F10928F
:105BF0006428109263281092AB281092DF2710922D
:105C0000E1271092D527109285278FEF8093A82740
:105C10008093A9278093AA278093AB278093AC27F2
:105C20008093AD278093AE278093AF27E2EBF7E216
:105C300014821182108213821282359687E2E53D2A
:105C4000F807B1F71092622810921F2888E00E948E
:105C5000271F1FB7F89480E00E94091381E00E947B
:105C6000091382E00E9409131FBF002309F452C0E8
:105C70001092AC2882EC97E09093D8278093D72796
:105C800080E098E7909329288093282811E01093CA
:105C9000B127109284271092E3270E94E2B68093E6
:105CA000E02784EF91E09093E5278093E427109319
:105CB000D62786E08093A72710922C2810922D28B3
:105CC00010922E2810922F281092302810923128EE
:105CD00010923228109233288FEF9FEF90931E2856
:105CE00080931D280E94E2B68093E22710928C27B1
:105CF000109287281092992810929E2810929F281F
:105D00001092A0281092A1281092A22810928D27FC
:105D100010929E271F910F9108950F931F93CF9379
:105D2000DF93EC01088119818091AB28813011F457
:105D30000E94652DF801018180E090E00E94CA1167
:105D400080E0011181E00E947D1D182F81E090E02C
:105D50000E94CA11802F0E94F42D0E948A2D89ED85
:105D600097E20E94271782E298E20E9427178DEAA5
:105D700098E20E94271786E897E20E942717E88199
:105D8000F981118380E280838DEA98E2BE010E944E
:105D90007E16DF91CF911F910F910895DF93CF93DE
:105DA00000D000D0CDB7DEB78091AB28813011F4A0
:105DB0000E94652D8FEF9FEF9A8389839C838B834D
:105DC00083E5BE016F5F7F4F0E94402F80E5BE01DB
:105DD0006D5F7F4F0E94402F81E00E94F42D0E9452
:105DE0008A2D0F900F900F900F90CF91DF91089513
:105DF0000E94B71D8823D1F40E94BE158823B1F0FC
:105E000081E00E94F42D0E948A2D89ED97E26FEFC8
:105E10000E94761682E298E26FEF0E94761686E87C
:105E200097E267E00E94761680E0089585E808957D
:105E3000E82F853419F48091E3270895883030F4F1
:105E4000E82FF0E0E25BF94F8491089580548032AE
:105E500028F4F0E0EA5EF94F849108958E2F81577F
:105E6000833128F4F0E0EB5FF94F84910895E03F2F
:105E700010F480E00895F0E0E756FA4F8491089519
:105E80001F93CF93DF93182FEB018091AB288130C4
:105E900051F40E94652D812FBE010E94221C182FF3
:105EA0000E948A2D04C0812F0E94221C182F812F4E
:105EB000DF91CF911F9108950F931F93CF93DF939D
:105EC0008C01FC01C081D181BE016D5F7F4F898152
:105ED000833509F4F5C0843508F04CC0823409F4E8
:105EE000B5C08334F8F4843009F4A2C0853068F476
:105EF000813009F4F8C0813008F4F2C0823009F42E
:105F0000FBC0833009F07CC0FAC0863009F498C029
:105F1000863008F490C0873009F495C0813409F0C8
:105F20006FC097C08B3409F4B5C08C3480F48634CC
:105F300009F49CC0873420F4853409F061C08CC01A
:105F4000893409F496C08A3409F05AC09AC08F3453
:105F500009F4ABC0803538F48C3409F4A0C08E3419
:105F600009F04EC09FC0803509F4A2C0823509F007
:105F700047C0A3C0833709F4D1C08437F8F489350A
:105F800009F44BC08A3560F48635E1F1873518F4A1
:105F90008535B1F571C08735C1F1883589F538C0CF
:105FA0008D3509F442C08E3518F48A3549F538C06C
:105FB000813709F4A7C0823719F5ADC08C3709F4D1
:105FC000D2C08D3760F4853709F4B4C0853708F442
:105FD000AEC0863709F4B7C0873791F4B7C08238AE
:105FE00009F4D6C0833830F4803809F4C5C081384C
:105FF00039F4C5C0833809F4CFC0803F09F467C0C5
:1060000094EFD3C08091AC28C5C080917427C2C0E2
:106010008091D7279091D82757C080917827BAC010
:1060200080912828909129284FC08091B127B2C033
:1060300080916327AFC0809161279091622744C00F
:1060400080917B27A7C080917127A4C08091D6271B
:10605000A1C0809184279EC04091E32729EE37E2BA
:10606000CB01B90150E00E94D6BA9EC08091E327CF
:1060700091C08091E0278EC08091E4279091E52720
:1060800023C0DB01ECE2F8E288E001900D92815040
:10609000E1F78AC080911D2890911E2815C080913B
:1060A000E22778C08091702775C08091772772C0F1
:1060B000809164279091652707C080918C276AC0E2
:1060C00080916727909168279C838B836DC0DB014B
:1060D000E9E5F7E288E001900D928150E1F764C0B4
:1060E0008091722757C080917F2790918027A0913F
:1060F0008127B091822732C0809158274BC0809170
:10610000662748C0DB01E5E6F8E282E201900D92E5
:106110008150E1F749C0809187283CC0DB01E8E865
:10612000F8E281E101900D928150E1F73DC080914C
:10613000992830C080919A2890919B28A0919C2802
:10614000B0919D280BC080919E2824C080919F28EB
:106150009091A028A091A128B091A2288B839C8324
:10616000AD83BE8321C0DB01E3EAF8E288E0019061
:106170000D928150E1F718C080918D270BC0DB0193
:10618000EEE8F7E280E101900D928150E1F70CC05A
:1061900080919E278B8308C0DB01EFE9F7E288E05E
:1061A00001900D928150E1F790E089818A838EE120
:1061B000888399838DEA98E2B8010E947E16DF9168
:1061C000CF911F910F910895FF920F931F93CF933B
:1061D000DF93182FEB01F42E853509F4AFC0863517
:1061E00008F040C0873409F4E4C08834F8F48234FD
:1061F00009F487C0833468F4853038F4823008F0BD
:10620000D8C0882309F4D5C06CC0813409F069C0B6
:1062100080C0843409F479C0843408F4CAC0853459
:1062200009F47BC0863409F05CC080C0813598F4E5
:106230008E3408F0BEC08A3409F487C08B3420F451
:10624000893409F04EC076C08B3409F497C08C3481
:1062500009F047C09AC0823509F49BC0823508F422
:1062600040C0A7C0843709F422C18537E8F48A35D5
:1062700009F440C08B3550F4873509F49AC087354E
:1062800090F18835A1F1893561F593C0813709F422
:10629000F8C0823718F48D3521F5ECC0823709F447
:1062A000F9C08337F1F4FAC0803809F42BC1813882
:1062B00060F4863709F40CC1863708F4FCC08737D0
:1062C00009F40AC18C3769F414C1823809F42AC16F
:1062D000823808F41EC1833809F42BC1803F09F4C9
:1062E00068C004EF2FC188818093AC282AC18881BF
:1062F0009981BBC08881998190932928809328280F
:1063000020C188818093D6271CC188818093A727CC
:1063100018C188818093842714C129EE37E2409107
:10632000E327C90150E00E94D6BA0BC1888180934F
:10633000E32707C188818093E02703C18881998181
:106340009093E5278093E427FCC0888180932C28D4
:10635000898180932D288A8180932E288B81809338
:106360002F288C81809330288D81809331288E81D5
:10637000809332288F8180933328E3C0888199816C
:1063800090931E2880931D28DCC088818093E2278B
:10639000D8C06881611161E060938C27662331F079
:1063A0000E94652D86E00E94271FCBC00E948A2D87
:1063B000C8C0812FBE010E94221C082F813871F4B1
:1063C0000E94F11E812FBE010E94221C082F8823EB
:1063D00009F0B8C081E080936C1B03C0882309F0EA
:1063E000B1C080917027282F30E080917427482F0A
:1063F00050E060917727CA01861B91092817390759
:106400000CF4C901A82F281B310981E090E002C0DB
:10641000880F991F4A95E2F70197289FA001299FAD
:10642000500D389F500D112420E030E070E0E1E085
:10643000F0E00DC0C901860F971FEF0102C0CC0F1D
:10644000DD1F8A95E2F74C0F5D1F2F5F3F4F2A1724
:1064500088F384E190E09C01429FC001439F900D2E
:10646000529F900D1124865F9E4F9093D827809362
:10647000D72767C090E08881811191E09093B12780
:1064800060C0A5E6B8E2FB0182E201900D92815066
:10649000E1F757C088818093872853C0A8E8B8E205
:1064A000FB0181E101900D928150E1F74AC08881A2
:1064B0008093992846C088819981AA81BB81809365
:1064C0009A2890939B28A0939C28B0939D2839C02C
:1064D000888180939E2835C088819981AA81BB815B
:1064E00080939F289093A028A093A128B093A228DE
:1064F00028C0A3EAB8E2FB0188E001900D92815028
:10650000E1F71FC090E08881811191E090938D2781
:1065100018C0AEE8B7E2FB0180E101900D92815016
:10652000E1F70FC090E08881811191E090939E2760
:1065300008C0AFE9B7E2FB0188E001900D928150FD
:10654000E1F700E0FF2049F080916C1B882329F0DF
:1065500080E00E94031F10926C1B802FDF91CF916F
:106560001F910F91FF900895EF92FF920F931F9349
:106570007C01FC0100811181B8016E5F7F4FF80141
:10658000818141E00E94E430F801918192839FE192
:10659000908381838DEA98E2B7010E947E161F9155
:1065A0000F91FF90EF900895CF93DF93EC01E88176
:1065B000F98183E280836183662311F00E948A2D32
:1065C0008DEA98E2BE010E947E16DF91CF91089578
:1065D000809136288823E1F080E00E9409138091A1
:1065E0003628813031F480915828882311F060E0FA
:1065F00001C06BEE8091D527823031F48091E7277E
:106600009091E8270E94D432109264281092D527E6
:1066100008958091D527823039F48091E7279091B1
:10662000E8276BEE0E94D4321092D527109264288E
:106630000895CF92DF92EF92FF920F931F93DF9313
:10664000CF93CDB7DEB728970FB6F894DEBF0FBE55
:10665000CDBFD82EC92E8091D527882309F03EC002
:10666000809163288330D1F18091DF278823B1F5B1
:106670008091AB28813011F40E94652DED2CFC2C0B
:10668000D701ED91FC9181819F012C5F3F4F8230BA
:1066900031F4848195819A83898342E00DC0AE01F3
:1066A0004F5F5F4F88E0D9010D909D01DA010D9297
:1066B000AD018150C1F743E00281138181E060E0C8
:1066C0009E012F5F3F4F0E94B727882311F4C70117
:1066D00007C0D092E727C092E82705C08D2D9C2DDA
:1066E00061EE0E94D43228960FB6F894DEBF0FBE3A
:1066F000CDBFCF91DF911F910F91FF90EF90DF9071
:10670000CF9008955F926F927F928F929F92AF92F7
:10671000BF92CF92DF92EF92FF920F931F93DF937E
:10672000CF93CDB7DEB761970FB6F894DEBF0FBE3B
:10673000CDBFBC014091DF27423011F0443069F4F5
:106740008091D627882349F0E091E727F091E82748
:1067500020813181D901199604C0A0E0B0E020E089
:1067600030E05091442859830091452810914628E3
:106770001B830A83523069F41E821F821886198691
:106780001A861B8680914728909148289D838C8388
:1067900018C0809147288C83809148288D838091F0
:1067A00049288E8380914A288F8380914B2888873F
:1067B00080914C28898780914D288A8780914E2826
:1067C0008B87909072279C86B0906327BD868091BE
:1067D000592890915A289F878E87188A80915B2824
:1067E00087FF02C081E0888B80915728898B4230D7
:1067F00019F0443009F06FC08091D627882309F43E
:106800006AC0F901F084EC81FD815C806D807E803E
:106810008F80A884C984DA84EB8440E049C0119653
:106820008D919C9112970817190709F03FC08C9120
:106830005817E1F51B968C911B979816B9F51C9685
:106840008C911C97B81691F5523041F413968D91A6
:106850009C911497E817F90749F53DC013968C9160
:106860001397851519F514968C9114978615F1F4E4
:1068700015968C9115978715C9F416968C911697D5
:106880008815A1F417968C9117978A1579F41896A4
:106890008C9118978C1551F419968C9119978D1528
:1068A00029F41A968C911A978E15A9F04F5F51967C
:1068B0004F1508F4B4CF59C0FD01DE01119681E1F6
:1068C0000D9001928150E1F7D90118968C9118979B
:1068D0008F5F18968C9390915C2880915F28882315
:1068E00021F48091D6278823E1F5DB01ED91FC911D
:1068F00087E180838091382881839F012E5F3F4FFD
:10690000AE014F5F5F4F81E1DA010D90AD01D9011A
:106910000D929D018150C1F780915C28838B892F56
:10692000877059F4892F90E08077907024E09595D6
:1069300087952A95E1F7882331F080915D28909121
:106940005E28958B848B80915F28868B8091602850
:1069500090916128908F878B8DEA98E20E947E1635
:1069600009C0CB010E94471605C0E4E0EF1508F40A
:10697000B2CFA2CF61960FB6F894DEBF0FBECDBFE7
:10698000CF91DF911F910F91FF90EF90DF90CF900B
:10699000BF90AF909F908F907F906F905F90089581
:1069A0000F931F93DF93CF9300D000D0CDB7DEB706
:1069B0008C0184E597E29A838983F8018181928131
:1069C0009C838B8386E897E2BE016F5F7F4F0E94B6
:1069D0001B17F80141815281E2EBF7E220E030E041
:1069E000808191814817590779F4F901EE0FFF1F53
:1069F000EE0FFF1FE20FF31FEE54F84D14821182C9
:106A000010820E94192D06C02F5F3F4F3596273008
:106A1000310531F7109262280F900F900F900F9070
:106A2000CF91DF911F910F910895EF92FF920F93F5
:106A30001F93CF93DF93182FEB011092642880915E
:106A4000DF278250823020F4812F0E940C38B5C09D
:106A50008881883009F4A5C0893050F4823009F467
:106A600097C0843009F44DC0813009F0A4C01DC026
:106A70008B3009F446C08C3020F48A3009F09BC07A
:106A800096C08C3009F493C08D3009F094C0809189
:106A90006228882319F0CB010E94D03489819A8121
:106AA000612F4B810E94962986C0193E11F0113E3C
:106AB00041F489819A81612F4FEF5FEF0E94751F2A
:106AC0007AC08093D527409128285091292860E0EA
:106AD00070E024E0440F551F661F771F2A95D1F7F9
:106AE00080E020E030E006EC1FE1EE24FF240E946D
:106AF0001514882309F461C080E090E00E94C61F4D
:106B00005CC089819A810E9447168091D527813087
:106B100009F453C088818430A1F4173881F0E091E2
:106B2000E727F091E827A081B18183E28C93119649
:106B30001C938DEA98E2BF010E947E163CC082E061
:106B400005C0193EC1F1113EB1F183E08093D52714
:106B50004091D7275091D82760E070E094E0440F2F
:106B6000551F661F771F9A95D1F780E020E030E02F
:106B700009E013E3EE24FF240E94151491E09093A2
:106B800064288823D1F080E090E00E94093315C08A
:106B9000CB010E94D03469817A81812F0E94952D8A
:106BA0000AC069817A81812F0E94603804C089817E
:106BB0009A810E9447160E948A2DDF91CF911F91E2
:106BC0000F91FF90EF900895CF93DF93E0912A28E3
:106BD000F0912B28C081D181DE01A656BF4FFA83E8
:106BE000E983882339F087E088838C9323E038E0B9
:106BF0004AE013C086E088838C9318979D0149E58D
:106C000057E288E0FA010190AF01F90101929F017A
:106C10008150C1F723E438EC42E1FD018FEF9FEF93
:106C20009293829332979183808315978091E22784
:106C30008C938F5F8093E2273E932E93FD014293C6
:106C4000FF83EE83CE0162E070E040E00E94031B10
:106C5000882311F080E003C081E080936428DF91F5
:106C6000CF910895CF92DF92FF920F931F93DF93FE
:106C7000CF930F92CDB7DEB7F82E6B01FB010081E9
:106C8000118184E063E77BE10E94402F4091DF2780
:106C90005091D6272091721B66C0423011F04430CB
:106CA00039F4552329F0F8018085853008F05EC05D
:106CB000322F3F5FF80184819581A681B781022E32
:106CC00004C0B695A795979587950A94D2F78170D9
:106CD0009070892B09F446C02093721BF1E0FF16D7
:106CE00021F482E08093DF2705C083E0F81611F4D9
:106CF000F092DF2780E062E77BE10E94402FF82ED0
:106D00008823B9F080912A2890912B280E94471659
:106D100010922B2810922A280E948A2D8AEEF801C0
:106D2000818310868DEA98E2B6010E947E16109249
:106D3000DF271091DF27123009F05DC0FF2061F4DA
:106D400081E00E94E435882309F055C01983CE0103
:106D500001960E94D8374FC08091721B8F5F80933D
:106D6000721B49C0232F2B3108F497CF2093721B3D
:106D7000F1E0FF1609F03FC080912A2890912B285E
:106D80000E94471610922B2810922A288091D6270D
:106D9000882341F0F8018085853010F08AEF07C024
:106DA000882319F0F801118203C08AEEF80181836B
:106DB00080E560E278E20E94402F6091E7277091C1
:106DC000E8278DEA98E20E947E168091E62780935C
:106DD000721B80E062E77BE10E94402F8091B02728
:106DE0008093731B84E063E77BE10E94402F109245
:106DF000DF270E948A2D0F90CF91DF911F910F9175
:106E0000FF90DF90CF900895CF92DF92EF92FF92A4
:106E10000F931F93DF93CF9300D0CDB7DEB7D82E5B
:106E2000C92E082F192FD801ED91FC91809172275E
:106E30008093E627809163278093B0278681809393
:106E4000741B818180936D1B82819381A481B581A4
:106E500080936E1B90936F1BA093701BB093711B5C
:106E600027812093731BD092E727C092E8278BE1FC
:106E7000808380916D1B828380916E1B90916F1B2C
:106E8000A091701BB091711B84839583A683B783F7
:106E90002383108611868091D527882341F4809121
:106EA000DF27882321F480916D1B882341F488EE2D
:106EB00081838DEA98E2B8010E947E166EC08091AF
:106EC000AB28813011F40E94652DF801E080F1803B
:106ED0008BE08093721B80916D1B8150823008F093
:106EE00052C08FEF9FEF9A8389838091642790919E
:106EF0006527909321288093202880E5BE016F5F4D
:106F00007F4F0E94402F80916D1B813021F4D092E1
:106F10002A28C0922B288DE90E944F169093E827CB
:106F20008093E727009729F488EED70111968C9378
:106F30002DC080916D1B823019F4C8010E94471644
:106F40002091E7273091E827D901ED91FC918BE161
:106F5000808380916D1B82838091731B83838091DA
:106F60006E1B90916F1BA091701BB091711B84835D
:106F70009583A683B7831086118680916D1BB90116
:106F80000E9432360AC088EEF70181838DEA98E2CA
:106F9000B8010E947E160E948A2D0F900F90CF910B
:106FA000DF911F910F91FF90EF90DF90CF900895A8
:106FB000CF93DF93C091E727D091E827988129816B
:106FC0008091DF278250833020F5E92FF22F21E0D6
:106FD00030E040E050E00090721B04C0220F331FED
:106FE000441F551F0A94D2F720953095409550952F
:106FF00084819581A681B78182239323A423B5231D
:1070000084839583A683B78380916D1BBE010E9404
:107010003236DF91CF910895DF92EF92FF920F9376
:107020001F93DF93CF930F92CDB7DEB7982F809148
:10703000E2278F5F8093E227D090DF2782E0D81687
:10704000B1F5992341F540EC53E060E070E0009029
:10705000741B04C0440F551F661F771F0A94D2F794
:1070600040545C4F6F4F7F4F94E0440F551F661F95
:10707000771F9A95D1F720E030E008ED17E3EE2472
:10708000FF240E941514882391F0D982CE01019625
:107090000E94D8370CC08091721B8F5F8093721B47
:1070A0006091E7277091E82781E00E9432360F90C7
:1070B000CF91DF911F910F91FF90EF90DF90089596
:1070C000CF93DF93EB01882391F468E77BE10E9483
:1070D000402F882361F484E069E77BE10E94402F20
:1070E00080E566E77BE10E94402F90E001C098EECA
:1070F000E881F98182E2808391838DEA98E2BE0182
:107100000E947E160E948A2DDF91CF910895EF9202
:10711000FF920F931F93CF93DF937C01DC01CD91FE
:10712000DC91A5E7BBE1FE018AE001900D92815060
:10713000E1F780916727909168278F5F9F4F39F41F
:10714000D701ED91FC9182E280838CEE1FC0BE01DD
:10715000695F7F4F8BE00E94402F80917E1B8823C8
:10716000E1F04091761B5091771B88E0B7012091A8
:10717000781B0091791B0E942339882309F05CC099
:10718000D701ED91FC9182E2808388EE81838DEAC4
:1071900098E2B7010E947E164FC0BE016B5F7F4F21
:1071A00087E40E94402F8D818F3009F48E832696CC
:1071B00084E5BE010E94402F8091AB28813011F4FC
:1071C0000E94652D80E566E77BE10E94402F80E00C
:1071D00068E77BE10E94402F182F84E069E77BE19C
:1071E0000E94402F8BE06CE77BE10E94402F11232F
:1071F000A9F486E00E94271F863081F480917C1BD1
:10720000882311F083E001C082E080936328D701D6
:10721000ED91FC9182E28083118207C0D701ED914C
:10722000FC9182E2808388EE81838DEA98E2B70147
:107230000E947E160E948A2DDF91CF911F910F919F
:10724000FF90EF900895DF92EF92FF920F931F93BC
:10725000DF93CF93CDB7DEB72C970FB6F894DEBF90
:107260000FBECDBF182FFB01F42EE52ED22EBE018E
:107270006F5F7F4F808191819C018CE0D9010D90DF
:107280009D01DB010D92BD018150C1F7408151810B
:10729000DA011C931296FC93EE931197BA016E5685
:1072A0007F4FFB0188E08193DB011196FC92DF01A7
:1072B0001196E1829D012F5F3F4F809167271196C4
:1072C0008C93F901319680916827D90111968C939E
:1072D000DF011196D182FD0131969F012F5F3F4F53
:1072E000193029F48A8511968C938B8503C08FEF12
:1072F00011968C938183F901319600839B0128506C
:107300003040D901E9E5F7E288E001900D92815023
:10731000E1F7F90180916427909165279293829318
:10732000193099F4F9013A979F01BE016E5F7F4FC2
:1073300088E0DB010D90BD01D9010D929D018150C6
:10734000C1F762E223E23CED07C08FEF9FEF92931B
:1073500082936CE123E038ED8FEF9FEF929382935D
:107360008091E22782938F5F8093E227329322936A
:107370006293DA011796FC93EE931697CA0162E0C6
:1073800070E041E00E94031B882311F080E003C0FD
:1073900081E0809364282C960FB6F894DEBF0FBE70
:1073A000CDBFCF91DF911F910F91FF90EF90DF90B4
:1073B00008950F931F93CF93DF93EC018DE90E9403
:1073C0004F168C010097F9F0DC01ED91FC918EE0F5
:1073D00080838881818389819A8193838283349693
:1073E000DE01139688E00D9001928150E1F789ED5E
:1073F00097E2B8010E947E16882311F481E004C050
:10740000C8010E94471680E0DF91CF911F910F9134
:1074100008958F929F92AF92CF92DF92EF92FF9258
:107420000F931F93CF93DF934C01F62ED42E122F80
:107430008DE90E944F16EC010097C9F0E881F981AF
:107440008DE0808392828182F38215830683E782B6
:10745000C086A186D48289ED97E2BE010E947E1685
:10746000882311F481E004C0CE010E94471680E019
:10747000DF91CF911F910F91FF90EF90DF90CF9010
:10748000AF909F908F900895BF92CF92DF92EF922E
:10749000FF920F931F93CF93DF93182F6A017B0105
:1074A000B22E8DE90E944F16EC010097B9F0E881E9
:1074B000F9818BE080831183C282D382E482F582DA
:1074C000B682078389ED97E2BE010E947E1688236B
:1074D00011F481E004C0CE010E94471680E0DF91E4
:1074E000CF911F910F91FF90EF90DF90CF90BF90C1
:1074F00008951F93CF93DF93182F8DE90E944F16A5
:10750000EC01009789F0E881F98188E0808311839C
:1075100089ED97E2BE010E947E16882311F481E076
:1075200004C0CE010E94471680E0DF91CF911F91E9
:1075300008951F93CF93DF93182F8DE90E944F1664
:10754000EC01009789F0E881F98189E0808311835B
:1075500089ED97E2BE010E947E16882311F481E036
:1075600004C0CE010E94471680E0DF91CF911F91A9
:1075700008957F928F929F92AF92BF92CF92DF92A7
:10758000EF92FF920F931F93CF93DF93F22ED32EA0
:10759000C42EB52EA62E972E882E792E8DE90E9408
:1075A0004F16EC010097D9F0E881F98182E08083E1
:1075B000F182D282C382B482A5829682878270864B
:1075C00012870187E38689ED97E2BE010E947E164D
:1075D000882311F481E004C0CE010E94471680E0A8
:1075E000DF91CF911F910F91FF90EF90DF90CF909F
:1075F000BF90AF909F908F907F900895DF92EF9211
:10760000FF920F931F93CF93DF93F82ED62EEA01AC
:10761000E22E8DE90E944F168C01009731F1DC01BA
:10762000ED91FC9181E08083F1828881838389815F
:107630009A81958384839F012A5F3F4FDE011396D1
:1076400088E00D90E90109929E018150D1F7E6860C
:10765000D28289ED97E2B8010E947E16882311F448
:1076600081E004C0C8010E94471680E0DF91CF91FD
:107670001F910F91FF90EF90DF9008955F926F92AE
:107680007F928F929F92AF92BF92CF92DF92EF92B2
:10769000FF920F931F93DF93CF93CDB7DEB7D82E12
:1076A0003B01F42E922E532EB02E86E7841708F459
:1076B00055C08DE90E944F168C01009709F44EC009
:1076C000DC01ED91FC9183E08083D182D3012C9188
:1076D000228311968D919C91129794838383CF017D
:1076E0000596A3014D5F5F4F223079F41582168213
:1076F00017821086118612861386148613968D9132
:107700009C911497968385830AC09C0188E0DA01D6
:107710000D90AD01D9010D929D018150C1F7B58643
:10772000E686C786A08A818AF28A2BE930E02F1983
:1077300031092E0F3F1FC901692D752D4F2D50E0C6
:107740000E94D6BA89ED97E2B8010E947E1688237E
:1077500011F481E004C0C8010E94471680E0CF9177
:10776000DF911F910F91FF90EF90DF90CF90BF902E
:10777000AF909F908F907F906F905F900895FF9251
:107780000F931F93CF93DF93182F062FF72E8DE9BA
:107790000E944F16EC010097E1F0812F0E94182FF4
:1077A000482FE881F98186E0808311833296CF01EA
:1077B000602F7F2D50E00E94D6BA89ED97E2BE017E
:1077C0000E947E16882311F481E004C0CE010E943D
:1077D000471680E0DF91CF911F910F91FF900895A0
:1077E0001F930E946E29182F8DEA98E260E070E0E6
:1077F0000E941B17009719F00E94572911E00E9460
:107800009F190E947011812F1F9108958DEA98E2AF
:107810006FEF0E9476160E94F82E089581E0809303
:107820007F1B08953F924F925F926F927F928F924B
:107830009F92AF92BF92CF92DF92EF92FF920F93FF
:107840001F93DF93CF93CDB7DEB762970FB6F8944F
:10785000DEBF0FBECDBF4C015B013A01322ED02EF0
:10786000FE2C80917F1B882321F00E94983E10926D
:107870007F1B4F2D50E09A01237030702115310588
:1078800011F4EE240AC02F5F3F4F81E090E002C068
:10789000880F991F2A95E2F7E82E487F452BA1F41F
:1078A0008114910489F0A114B10471F0432C552482
:1078B00082010D0D111D8E2D90E09A8B898B800F0A
:1078C000911F8038910520F00E948E3E81E0A3C078
:1078D00080916C06882339F06114710409F50E94C7
:1078E0008E3E82E098C061147104D1F040E130E036
:1078F0004150E42FF0E0D301AE0FBF1FE058F44E2B
:107900008C912081822790E0232F30E0822B932BD3
:1079100030E0892B09F031E0442351F730936C06B5
:1079200080916C06882379F0C30160E040E00E94FA
:10793000B93EA0E8BBE1F30180E101900D928150D6
:10794000E1F710926C0681E0F5018083EE2061F092
:107950008E2D90E002979595879523E0880F991FCB
:107960002A95E1F781608083332021F0F501808141
:107970008064808384E0782E7F20F5016080168605
:10798000CC20D1F4EE2051F0D786080D191DC4018A
:10799000B801A501232D0D2D0E940C3E7720C1F1C9
:1079A00081E0F5018083C401840D951DB5014E2D44
:1079B0002D2D0E94263D2CC0772059F081E0F50145
:1079C0008083C401840D951DB5014E2D2D2D0E947F
:1079D000263DEE20E9F0F5016082D786C4017E01E4
:1079E0000894E11CF11CB701A501232D0D2D0E9467
:1079F0000C3E832D90E08D0D911D880D991DB701D2
:107A000049895A890E94C9BA009711F083E003C0DE
:107A10000E948E3E80E062960FB6F894DEBF0FBEE5
:107A2000CDBFCF91DF911F910F91FF90EF90DF902D
:107A3000CF90BF90AF909F908F907F906F905F900E
:107A40004F903F9008950E94723E08954F925F922A
:107A50006F927F928F929F92AF92BF92CF92DF925E
:107A6000EF92FF920F931F93DF93CF93CDB7DEB7C3
:107A700060970FB6F894DEBF0FBECDBF5C016B01FF
:107A8000642E122F80E090E060E040E00E94B93E5A
:107A90007724EE24FF24412E55244E010894811CA6
:107AA000911C25C07394D6011F967C92C6010E943A
:107AB000733EC4010E94853EC8010131110514F0D6
:107AC00080E190E0D501F401282F30E0A401420FBD
:107AD000531F04C08C91919189278D93E417F5076A
:107AE000C9F7A20EB31EE0EFFFEFEE0EFF1E8701F7
:107AF000040D151D10161106ACF26620E9F0D60132
:107B00001F961C92C6010E94733E8E010F5F1F4F8D
:107B1000C8010E94853E20E030E00CC0F801E20F71
:107B2000F31FD5018C9190818927F50181935F0125
:107B30002F5F3F4F621691F760960FB6F894DEBF45
:107B40000FBECDBFCF91DF911F910F91FF90EF90AE
:107B5000DF90CF90BF90AF909F908F907F906F906D
:107B60005F904F900895CF92DF92EF92FF920F9324
:107B70001F93DF93CF93CDB7DEB760970FB6F8941E
:107B8000DEBF0FBECDBF6C01F62E8C01E62E07C006
:107B9000C8010E94733E005F1F4F80EFE80E8FE028
:107BA0008E15B0F30F2D0F70F2949FE0F9222F2D58
:107BB00030E084E0220F331F8A95E1F72C0D3D1D44
:107BC0000023D9F010E07E010894E11CF11CC701EC
:107BD000B901402F50E00E94D6BAE0E1F0E0E01B8E
:107BE000F10B9701200F311FC90160E070E0AF0178
:107BF0000E94F1BAC7010E94733E60960FB6F894D6
:107C0000DEBF0FBECDBFCF91DF911F910F91FF90CF
:107C1000EF90DF90CF9008959F92AF92BF92CF9256
:107C2000DF92EF92FF920F931F93DF93CF93CDB725
:107C3000DEB760970FB6F894DEBF0FBECDBF6C0104
:107C40005B017A01122F902EFA01078780E090E005
:107C500060E040E00E94B93EC7010E94733E80E0B0
:107C600090E061E040E00E94B93E112301F1012F54
:107C70001F3008F00EE019821A83E02EFF249E01C7
:107C80002D5F3F4FC901B601402F50E00E94D6BA88
:107C9000602F6E5FCE0101960E94B33D011738F44C
:107CA000612F601BC6018E0D9F1D0E94B33DC60152
:107CB000810F911D692D0E94B33DC5010E94853E33
:107CC00060960FB6F894DEBF0FBECDBFCF91DF91A7
:107CD0001F910F91FF90EF90DF90CF90BF90AF90EA
:107CE0009F9008950895FC0190E0819180933E015A
:107CF0009F5F9031D1F78091911B806880933C0108
:107D000080913D0180FFFCCF0895FC0190E08091BF
:107D10003E0181939F5F9031D1F708958091B21B0E
:107D20009091B31B0F9719F480E00E94031F0895F0
:107D30008091792790917A279093B31B8093B21BFF
:107D40000F9711F40E94F11E80916D06882319F09F
:107D5000E2EAFBE102C0E2E9FBE190E0819180937D
:107D60003F019F5F9031D1F78091911B80933C013F
:107D700008950F931F93DF93CF93CDB7DEB760972E
:107D80000FB6F894DEBF0FBECDBFDC01162F042F57
:107D90000097F1F01092901B82E080936D0622E92B
:107DA0003BE1AD0180E1FA010190AF01F9010192DF
:107DB0009F018150C1F720E030E0FD01E20FF31F89
:107DC000808180933F012F5F3F4F20313105A9F71C
:107DD000002321F0013009F047C00EC080916D06EC
:107DE000813079F5E2E9FBE1819180933F018BE1FC
:107DF000E23AF807C9F725C080916D068130A1F1FC
:107E00008091901B8823A1F41092911B10923C0149
:107E1000CE0101960E94733EE2EAFBE180913F01B0
:107E200081938BE1E23BF807C9F781E08093901BD7
:107E3000E2EAFBE1819180933F018BE1E23BF807AD
:107E4000C9F700936D06123078F4802F880F880FE1
:107E5000880F88701295110F1072812B8093911BDF
:107E600080933C0181E001C080E060960FB6F894F9
:107E7000DEBF0FBECDBFCF91DF911F910F9108954F
:107E8000089508950895089508951092B4281092C1
:107E9000B3281092B5281092B6281092B7281092E5
:107EA000B8281092B9281092BA281092BB281092C4
:107EB000BC28EDEBF8E28FEF9FEF91838083128275
:107EC00013821482158216821782108611863A96C2
:107ED00029E2E731F20789F708950895089580EFC0
:107EE0000E94793A8EE696E00E9438BC81E0809349
:107EF000B81B80E50E94793A08958F929F92AF92C5
:107F0000BF92CF92DF92EF92FF920F931F93DF9376
:107F1000CF93CDB7DEB7C65CD0400FB6F894DEBFC6
:107F20000FBECDBF282F6B015A01833309F487C1DF
:107F3000843320F4823309F095C2E7C0863321F000
:107F40008C3309F08FC282C2DA0112969C9112978B
:107F500011968C91C82EDD24C90ED11CE5E0F0E00D
:107F6000CE0EDF1EC40ED51E8091ED149091EE143E
:107F7000009709F0BCC000D000D0EDB7FEB7319635
:107F80008FE796E0ADB7BEB712969C938E9311978C
:107F9000DA018C91828313820E94FCBB750100E0A0
:107FA00010E00F900F900F900F9023EB822E26E0A1
:107FB000922E22C00115110521F08AE390E00E9463
:107FC00031BC00D000D0EDB7FEB73196ADB7BEB72B
:107FD00012969C928E921197D70115968C9182835E
:107FE00013820E94FCBB0F5F1F4F0894E11CF11C21
:107FF0000F900F900F900F90F501818190E008177E
:108000001907C0F200D086EB96E0ADB7BEB7129666
:108010009C938E9311970E94FCBB00E010E00F90A0
:108020000F9093EBE92E96E0F92E24C0011511056F
:1080300021F08AE390E00E9431BC00D000D0ADB7BF
:10804000BEB71196EDB7FEB7F282E182F5018181EC
:10805000E00FF11FE80FF11D858112968C931297A6
:1080600013961C920E94FCBB0F5F1F4F0F900F9046
:108070000F900F90D50112968C9190E00817190778
:10808000A8F28E01055C1F4FB601685F7F4FC801E3
:108090000E94748B00D000D08BEB96E0EDB7FEB75A
:1080A00092838183148303830E94FCBB0F900F9003
:1080B0000F900F90B601685E7F4FC8010E94748BCD
:1080C00000D000D08CEC96E0ADB7BEB712969C9372
:1080D0008E93119714961C930E9313970E94FCBBDA
:1080E0000F900F900F900F908FEC96E004C00297C6
:1080F00020F481ED96E00E9438BCF5016381748123
:10810000C60140810E94488CE5C1DA018C9185301E
:1081100009F48BC0863040F48330B9F0843028F500
:10812000813009F0D7C10CC0873009F440C08730D6
:1081300070F18B3009F442C08D3009F0CBC15FC0C3
:10814000FA01818180939807C5C18A010F5F1F4F93
:1081500080E5B8010E94BF3B80E50E94793A8EE03D
:1081600090E062E070E0A8010FC0DA0111968D91F5
:108170009C9112979093B51B8093B41B8CE490E074
:1081800062E070E044EB5BE10E940411A3C1ABE547
:10819000B6E2FA01319688E001900D928150E1F744
:1081A000B5016F5F7F4F80EF0E94BF3B93C14F5F70
:1081B0005F4F88E090E066E070E0E6CF87E0E82E71
:1081C000F12CEC0EFD1E89E0F70111928A95E9F77A
:1081D0008CE2888782E08F878E01075E1F4FCA017D
:1081E0000196B8010E94CB8A882309F473C1C801A3
:1081F000B70141E021E030E00E94C8836BC18FEEFF
:1082000096E0BE016F5F7F4F0E94E7938981809364
:108210005929C501029660E820E030E040E050E0D6
:1082200003E010E00E943C6555C10E949D60FC0186
:10823000E95EFE4FD50111968C91878B4BC1FA01F7
:108240002081253009F4EFC0263070F4223011F17E
:10825000233020F4213009F03DC118C02330E9F06B
:10826000243009F037C11EC0283009F45BC0293022
:1082700030F4263029F1273009F02CC139C02930DB
:1082800009F48AC02A3009F025C1A9C08091980755
:108290002A83D2C02A832B83D0C0809199079091E2
:1082A0009A0704C08091B41B9091B51B2C839E83C8
:1082B0008D8383E363E070E0AE014C5F5F4FC3C02A
:1082C000FE01709689E0DF011D928A95E9F7288BFF
:1082D000DE015196EBE5F6E288E001900D928150C7
:1082E000E1F783E369E070E0AE01405F5F4FABC050
:1082F0008E01005F1F4F89E0F80111928A95E9F71E
:10830000288B80E090E068E070E046E050E09E015D
:108310002F5E3F4F0E94361183E369E070E0A801B1
:108320000E94128DFE01B99682E1DF011D928A95AD
:10833000E9F788E089A70E949D60AC01B2E0CB1606
:10834000D10408F4C7C0F501818190E027E131E054
:10835000829FF001839FF00D929FF00D1124E40F96
:10836000F51FD50112968C912DE1829FC001112439
:108370004996DE019B96E80FF91F80E101900D926E
:108380008150E1F7F50181818AA783E362E170E022
:10839000AE01475D5F4F57C0FE01ED59FF4F82E3CD
:1083A000DF011D928A95E9F721938F0181E00E94F8
:1083B0003197009741F0F801DC0181E30D900192C3
:1083C0008150E1F705C081E3D8011D928A95E9F754
:1083D00083E362E370E0AE014D595F4F34C0FE01AC
:1083E000EB56FF4F82E3DF011D928A95E9F789E0A2
:1083F00081938F0180E00E943197009741F0F8014E
:10840000DC0181E30D9001928150E1F705C081E329
:10841000D8011D928A95E9F783E362E370E0AE012B
:108420004B565F4F10C01B821A822A830E949D60A8
:10843000FC01E95EFE4F87898B8383E362E070E095
:10844000AE014E5F5F4F0E94128D44C081E0809369
:108450006326A4E6B6E2FA0186E001900D9281500F
:10846000E1F738C0EDB7FEB738970FB6F894FEBF06
:108470000FBEEDBF319684EF96E0ADB7BEB7129652
:108480009C938E931197B382A28224831582D78204
:10849000C6820E94FCBB750100E010E0EDB7FEB79C
:1084A00038960FB6F894FEBF0FBEEDBF0CC06091BA
:1084B0006F3970917039D7018D917D0190E00E94E4
:1084C000D0BB0F5F1F4F0C151D0588F384E297E0AA
:1084D0000E9438BCC5010E942FB6CA53DF4F0FB6A9
:1084E000F894DEBF0FBECDBFCF91DF911F910F91EA
:1084F000FF90EF90DF90CF90BF90AF909F908F90C4
:108500000895662341F085E297E00E9438BC81E03F
:108510000E94993A08959093B51B8093B41B81E013
:10852000809321298093B81B80E50E94793A0895B1
:10853000DF93CF930F92CDB7DEB7882321F081E090
:108540000E94993A16C021E02093B71B80917603D0
:1085500090917703892B31F40E94453F83E564EBCA
:108560007BE105C0298382E5BE016F5F7F4F0E94DA
:10857000BF3B0F90CF91DF9108950F93DF93CF937F
:1085800000D00F92CDB7DEB721E02983882321F0F8
:1085900081E00E94993A48C0663409F440C06734CB
:1085A00020F4613409F040C018C06235D9F0633559
:1085B000D9F58091760390917703892BA9F52A83C9
:1085C00081E4BE016E5F7F4F0E94BF3B84E18B83DD
:1085D00086E4BE016D5F7F4F25C082E5BE016F5FFF
:1085E0007F4F20C08091760390917703892B99F477
:1085F00041E050E060E070E00090980704C0440F54
:10860000551F661F771F0A94D2F781E021E000E032
:108610000E94443A09C080EF0E94793A05C085E47F
:108620006BE977E00E94BF3B0F900F900F90CF91C6
:10863000DF910F910895EF92FF920F93DF93CF9305
:10864000CDB7DEB729970FB6F894DEBF0FBECDBF0A
:108650007A01882321F081E00E94993A67C0603F47
:1086600009F047C0ABE5B6E2FA0188E001900D924F
:108670008150E1F78091760390917703892B91F0F7
:1086800041E050E060E070E00090980704C0440FC3
:10869000551F661F771F0A94D2F781E025E000E09E
:1086A0000E94443A8091B71B882309F43FC010927E
:1086B000B71B88E08987F7018081888781818F8354
:1086C00082818E8383818D8384818C8385818B835A
:1086D00086818A8387818983CE0101960E94C98918
:1086E0008091760390917703892B01F50E941CA558
:1086F0001DC06035D9F4FA014081518150939A0729
:10870000409399078091B81B882381F01092B81B81
:108710008091B51B89838091B41B8A8382E089870D
:10872000CA01BE016F5F7F4F0E94268929960FB64E
:10873000F894DEBF0FBECDBFCF91DF910F91FF90B8
:10874000EF900895AF92CF92DF92EF920F93CF9375
:10875000DF93282F8091760390917703892BA1F4E2
:108760008091990790919A076091980740E02FE0D7
:108770000FE0EE24E394CC24AA240E94093A89E372
:1087800097E00E9438BC6BC02223E9F5E60100E0C7
:1087900036E4C32E37E0D32E5FC04B858091980717
:1087A0004817E1F58C858823C9F529813A818091A4
:1087B000990790919A072817390781F588818230A7
:1087C00039F48B819C8190931829809317291FC0BD
:1087D0008330C9F48B81809319298C8180931A2965
:1087E0008D8180931B298E8180931C298F8180939A
:1087F0001D29888580931E29898580931F298A8554
:108800008093202904C081E00E94993A28C0842FD7
:1088100060E0AE0120E80E94FE3A21C000D000D006
:1088200000D0EDB7FEB73196ADB7BEB71296DC9269
:10883000CE9211974283138289819A819583848392
:108840000E94FCBB61960F5F8DB79EB706960FB670
:10885000F8949EBF0FBE8DBF0E1508F49ECFDF911A
:10886000CF910F91EF90DF90CF90AF9008956F92DE
:108870007F928F929F92AF92BF92CF92DF92EF92B0
:10888000FF920F931F93CF93DF93D22EC32EB42E5C
:10889000A52E962E872E782E692E8DB79EB70A9715
:1088A0000FB6F8949EBF0FBE8DBFEDB6FEB608940E
:1088B000E11CF11C8AE797E0EDB7FEB79283818354
:1088C000872D962D00E20E94A3AEC901BA01F701DF
:1088D0002283938344837583D682C782B086A18620
:1088E0000E94FCBBEDEBF8E2C1E0D0E08DB79EB793
:1088F0000A960FB6F8949EBF0FBE8DBF00811181FE
:108900009FEF0F3F190759F182818D1509F057C06C
:1089100083818C1509F053C084818B1509F04FC0F9
:1089200085818A1509F04BC08681891509F047C0F9
:108930008781881509F043C08085871509F03FC0FD
:1089400081858615E1F52D2D3C2D4B2D5A2D692D58
:10895000782D872D962DEE240E94B93A36C0FE015F
:10896000EE0FFF1FCE0163E0880F991F6A95E1F7B4
:10897000E80FF91FED54F74DC08311822D2D3C2DCA
:108980004B2D5A2D692D782D872D962D0C2F10E00B
:10899000EE240E94B93AFE01EE0FFF1FEE0FFF1FFB
:1089A000EC0FFD1FEE0FFF1FEB54F74DD082C1827D
:1089B000B282A382948285827682678206C02196E3
:1089C0003A96CA30D10509F099CFDF91CF911F9126
:1089D0000F91FF90EF90DF90CF90BF90AF909F905E
:1089E0008F907F906F900895EF920F93DF93CF93C6
:1089F000CDB7DEB70E94EE45CF91DF910F91EF909A
:108A00000895FC01DB0118968C911897883099F530
:108A10008C9192E089279085981709F057C091852D
:108A200011968C911197981709F050C09285129663
:108A30008C911297981709F049C0938513968C91E1
:108A40001397981709F042C0948514968C91149747
:108A50009817E1F5958515968C9115979817B1F5AE
:108A6000968516968C911697981781F520E0978534
:108A700017968C9154C0863061F58C9192E08927CD
:108A80009085981719F5918511968C9111979817E3
:108A9000E9F4928512968C9112979817B9F4838510
:108AA0008F3FA1F484858E3F89F4958513968C9130
:108AB0001397981759F4968514968C9114979817D4
:108AC00029F420E0978515968C9129C080E090E0EC
:108AD0000895823011F080E00895208530E0809183
:108AE000563190E08D7F28173907F9F491858091F0
:108AF00057319817D1F482858823B9F483858F3F45
:108B0000A1F484858E3F89F48585882371F4968548
:108B10008C91981751F420E0978511968C919813B9
:108B200021E081E02827822F089580E090E00895D9
:108B300081E08093DC20089591E09093CE20109204
:108B4000CF2080E28093D02082E08093D1208DE0FE
:108B50008093D22088EB8093D3209093DC200895DB
:108B60000F931F93CF93DF93EC011092DC201091B1
:108B7000CE2001E010C0113061F480ED90E2BE0122
:108B800048E050E00E94C9BA009719F42EEC30E298
:108B900008C00093DC208091DC20882361F320E072
:108BA00030E0C901DF91CF911F910F9108950F938C
:108BB0001F93CF93DF93EC018B010E94B045892B6B
:108BC00011F480E006C0CE01B8010E940145811178
:108BD00081E0DF91CF911F910F910895CF92DF92A5
:108BE000EF92FF920F931F93DF93CF93CDB7DEB732
:108BF0002A970FB6F894DEBF0FBECDBF7C016B0184
:108C000081E0809359291092BD1B1092BB1B80916B
:108C10005529909156298093B91B9093BA1B409384
:108C2000572910925829B90150E00E94D6BAD701AD
:108C30002C91223081F414968C9114978983139689
:108C40008C918A8389819A819093442980934329C6
:108C500020934B29B2C0233009F09AC0F701238139
:108C6000348145815681678170858185928508E3CD
:108C70000E94A3AE2B83D70113962C9113971496C1
:108C80003C91149715964C91159716965C911697F2
:108C900017966C91179718967C91189719968C9146
:108CA00019971A969C9100E30E94A3AE2C83F701BA
:108CB00023813481458156816781708581859285C4
:108CC00008E20E94A3AE2D83D70113962C9113972F
:108CD00014963C91149715964C91159716965C91A5
:108CE000169717966C91179718967C911897199666
:108CF0008C9119971A969C9100E20E94A3AE2E8344
:108D0000F701238134814581568167817085818592
:108D1000928508E10E94A3AE2F83D70113962C9170
:108D2000139714963C91149715964C911597169697
:108D30005C91169717966C91179718967C911897D7
:108D400019968C9119971A969C9100E10E94A3AEF6
:108D50002887F70123813481458156816781708599
:108D60008185928508E00E94A3AE2987D7011396DA
:108D70008C918A87E7E5F9E27497DE01139688E023
:108D80000D9001928150E1F788E080934B2915C046
:108D900000D000D000D0EDB7FEB731968FEA97E053
:108DA000ADB7BEB712969C938E93119783EC97E064
:108DB0009383828380E396E0C4C0D6012C91223055
:108DC00081F414968C911497898313968C918A83DD
:108DD00089819A8190934D2980934C29209354291D
:108DE000BDC0233009F099C0F6012381348145814B
:108DF0005681678170858185928508E30E94A3AEC4
:108E00002B83D60113962C91139714963C911497AB
:108E100015964C91159716965C91169717966C912E
:108E2000179718967C91189719968C9119971A96FE
:108E30009C9100E30E94A3AE2C83F6012381348130
:108E400045815681678170858185928508E20E94FF
:108E5000A3AE2D83D60113962C91139714963C91B3
:108E6000149715964C91159716965C911697179630
:108E70006C91179718967C91189719968C91199761
:108E80001A969C9100E20E94A3AE2E83F6012381E4
:108E9000348145815681678170858185928508E19D
:108EA0000E94A3AE2F83D60113962C91139714968C
:108EB0003C91149715964C91159716965C911697C0
:108EC00017966C91179718967C91189719968C9114
:108ED00019971A969C9100E10E94A3AE2887F6018B
:108EE0002381348145815681678170858185928592
:108EF00008E00E94A3AE2987D60113968C918A8739
:108F0000ACE4B9E2FE01339688E001900D92815005
:108F1000E1F788E08093542921C000D000D000D030
:108F2000EDB7FEB731968FEA97E0ADB7BEB71296B0
:108F30009C938E93119783EC97E0938382838AE4CA
:108F400096E0958384830E94FCBBEDB7FEB736960E
:108F50000FB6F894FEBF0FBEEDBF1DC586EC90E2C4
:108F60000E94FA85892B41F01092BF1B1092BE1B04
:108F70001092C1201092C020E091B91BF091BA1B51
:108F8000908180E02181422F50E0482B592BCA016B
:108F90008070987F892F9927803C910549F0803E09
:108FA0009105C9F0EE24FF2410E020E030E025C058
:108FB0007FEFE72E77E0F72EE422F522928180E022
:108FC000238130E0282B392B8091BB1B8C5F809351
:108FD000BB1B10E012C01481928180E0238130E03D
:108FE000282B392B6FEFE62E67E0F62EE422F522D0
:108FF0008091BB1B8B5F8093BB1B8091C0209091A5
:10900000C120892B39F1E114F10409F4C4C4809121
:10901000BE1B9091BF1BE816F90609F0BCC48091F5
:10902000C4209091C5208217930709F0B4C4009121
:1090300042298AE399E263E479E2402F50E00E94FA
:10904000C9BA009709F0A7C480914B29081709F005
:10905000A2C422C0E114F104F9F0F092BF1BE09227
:10906000BE1B3093C5202093C42086EC90E240E2E2
:1090700051EA67E070E00E9423862AE339E24091DA
:109080004B29E3E4F9E2C901BF0150E00E94D6BADE
:1090900080914B29809342299091BB1B953009F414
:1090A00008C44091B91B5091BA1B292F30E0FA0136
:1090B000E20FF31F6081862F807E803609F0DEC3C9
:1090C0002E5F3F4F240F351F3093DB202093DA2093
:1090D000818187FF06C02F5F3F4F3093DB202093B5
:1090E000DA208091BB1BE091B91BF091BA1BE80F0D
:1090F000F11D808190E09C012071307083FD47C09C
:10910000E091DA20F091DB20232B71F5A1ECBBE19B
:10911000319683E001900D928150E1F7E091DA20E1
:10912000F091DB2040813496F093DB20E093DA204D
:10913000242F30E0C9018F73907095958795959590
:10914000879580668093C01B46954695407396E050
:10915000220F331F9A95E1F7422B8091C11B8F702C
:10916000482B4093C11B3FC080E68093C01B908179
:10917000892F8695869580739F70892B8093C11B5C
:10918000818192819093C31B8093C21B1DC0232BAE
:1091900009F5E091DA20F091DB20808186958695B3
:1091A0008F7080668093C01B8081982F96959695CE
:1091B00090738295880F880F807C892B8093C11BC8
:1091C0001092C31B1092C21B3396F093DB20E093E6
:1091D000DA2009C080E68093C01B1092C11B109258
:1091E000C31B1092C21B8091BB1BE091B91BF09175
:1091F000BA1BE80FF11D808182FD0BC0E091DA20DF
:10920000F091DB2081918093C61BF093DB20E093EB
:10921000DA208091BB1BE091B91BF091BA1BE80FDB
:10922000F11D808190E0837090708130910561F034
:10923000823091051CF4892B79F019C08230910598
:1092400029F00397A1F406C081E001C080E4809377
:10925000C71B0DC08FEFFBCFE091DA20F091DB2030
:1092600081918093C71BF093DB20E093DA20E0919B
:10927000B91BF091BA1B8091BB1BE80FF11D218136
:10928000822F90E026FF86C027FD02C020E003C0A9
:10929000228122952F7080739070892BF1F01092AB
:1092A000DC2091E00DC08091CE20813039F4809196
:1092B000CF20821719F48EEC90E208C09093DC2046
:1092C0008091DC20882379F380E090E09093D9208E
:1092D0008093D820892B09F4ECC28091BB1BE091CC
:1092E000B91BF091BA1BE80FF11D818190E08073EA
:1092F000907080319105A9F0813191051CF4892B82
:1093000041F0BFC08032910531F1C09709F0B9C07A
:1093100032C080E1E8ECFBE1DF011D928A95E9F7BC
:10932000B0C0E091D820F091D920A8ECBBE13296F2
:1093300088E001900D928150E1F7A0EDBBE18091B2
:10934000DA209091DB209C01F90188E001900D92D8
:109350008150E1F761C0E091D820F091D920A8ECCC
:10936000BBE1329688E001900D928150E1F786E0F2
:10937000E0EDFBE160C0E091D820F091D920A8ECAD
:10938000BBE1329688E001900D928150E1F788ECC4
:109390009BE173C0807390708031910521F1813120
:1093A00091051CF4892B41F06CC080329105D1F1FC
:1093B000C09709F066C052C0A8ECBBE18091DA20EA
:1093C0009091DB209C01F90180E101900D92815088
:1093D000E1F78091DA209091DB2040969093DB209A
:1093E0008093DA204EC08EEF8093C81B80E8809374
:1093F000C91BEAECFBE186E0DF011D928A95E9F7E3
:1094000036962091DA203091DB20C901DC0188E01A
:109410000D9001928150E1F78091DA209091DB204C
:109420000896DCCF8EEF8093C81B80E88093C91B21
:109430008CE0EAECFBE1DF011D928A95E9F7E0910F
:10944000DA20F091DB20819191919093D71B80934A
:10945000D61BF093DB20E093DA2013C08EEF8093CD
:10946000C81B80E88093C91BEAECFBE186E0DF01C2
:109470001D928A95E9F7CF01029763E479E20E9491
:10948000F164E091B91BF091BA1B8091BB1BE80F0E
:10949000F11D4181842F90E09C012470307043FFC6
:1094A00078C0232B09F055C18370907081309105ED
:1094B000D9F0823091051CF4892B41F04AC18230E9
:1094C0009105A1F1039709F044C14EC0A8EDBBE19D
:1094D0008091DA209091DB209C01F90180E10190DC
:1094E0000D928150E1F7E1C08FEF8093D81BE0919E
:1094F000DA20F091DB2081918093D91B2AED3BE1AA
:1095000089E0D9011D928A95E9F7D901199685E07C
:1095100001900D928150E1F78091DA209091DB204B
:1095200006969093DB208093DA2013C18FEF80930F
:10953000D81BE091DA20F091DB2081918093D91B38
:109540002AED3BE18BE0D9011D928A95E9F7D9011B
:10955000199683E001900D928150E1F78091DA2015
:109560009091DB200496DDCF8FEF8093D81B82E0B3
:109570008093D91B8DE0EAEDFBE1DF011D928A9516
:10958000E9F7E091DA20F091DB2081918093E71BED
:10959000C8C0232B09F46AC047FD02C090E002C096
:1095A00092819F701092DC2021E00DC08091CE202E
:1095B000813039F48091CF20891719F42EEC30E2F4
:1095C00008C02093DC208091DC20882379F320E000
:1095D00030E03093D9202093D8202115310509F4AB
:1095E00068C18091BB1BE091B91BF091BA1BE80FD9
:1095F000F11D818190E08370907082309105E9F0D7
:109600008330910539F1019709F0A3C0A8EDBBE1C2
:10961000F901329688E001900D928150E1F7A0EEB9
:10962000BBE18091DA209091DB209C01F90188E078
:1096300001900D928150E1F757C0A8EDBBE1F9010F
:10964000329688E001900D928150E1F786E0E0EEDD
:10965000FBE159C0A8EDBBE1F901329688E0019029
:109660000D928150E1F788ED9BE16FC0837090709F
:109670008130910501F1823091051CF4892B41F074
:1096800068C082309105B1F1039709F062C04EC005
:10969000A8EDBBE18091DA209091DB209C01F901DB
:1096A00080E101900D928150E1F78091DA20909154
:1096B000DB20409636CF8EEF8093D81B80E88093D6
:1096C000D91BEAEDFBE186E0DF011D928A95E9F7FF
:1096D00036962091DA203091DB20C901DC0188E048
:1096E0000D9001928150E1F78091DA209091DB207A
:1096F000089617CF8EEF8093D81B80E88093D91BF4
:109700008CE0EAEDFBE1DF011D928A95E9F7E0913B
:10971000DA20F091DB20819191919093E71B809367
:10972000E61BF093DB20E093DA2013C08EEF8093EA
:10973000D81B80E88093D91BEAEDFBE186E0DF01CE
:109740001D928A95E9F7CF0102976CE479E20E94B5
:10975000F1648091BD1B885D8093BD1B8091BB1B14
:10976000E091B91BF091BA1BE80FF11D808182FFD7
:1097700056C0A091DA20B091DB208C91887F803F89
:1097800009F04DC081E18093C61B8C91803F29F187
:10979000833F09F08EC0E0ECFBE1B89611968C9106
:1097A000119782958F7090E080559F409093E81BB1
:1097B000818311968C91119790E08F7090708055F5
:1097C0009F409283838312968D919C9113979093DF
:1097D000EF1B8093EE1B149619C011968D919C91EE
:1097E00012979093E91B8093E81B13968D919C919F
:1097F00014979093EB1B8093EA1B15968D919C9187
:1098000016979093EF1B8093EE1B1796B093DB2077
:10981000A093DA208091BD1B885F8093BD1B90913F
:10982000DA208091B91B981B9093BB1BE114F104C3
:1098300051F41092C41B8091BD1B8852891B9091DA
:109840005729890F0CC0E8EDFFEFEE0EFF1EF092D6
:10985000C41B88E290E0E80EF91E8E2D885280939A
:10986000C51B8091C61B813121F58091C41B90914D
:10987000C51B9093ED1B8093EC1B1BC0613409F05A
:109880008AC0892F8F5F8093BB1BA0ECBBE1FA01DC
:10989000E80FF11D88E201900D928150E1F780916F
:1098A000BB1B885D8093BB1B8091BD1B885D809333
:1098B000BD1B409157299091BB1B491B4093BC1B7A
:1098C000212F30E083E0220F331F8A95E1F780914A
:1098D000BD1B280F311D2054344EE091B91BF0916F
:1098E000BA1BE90FF11DC901BF0150E00E94D6BAB1
:1098F000EF28C9F08091C0209091C120892B31F4CC
:109900008091BD1B8093C0201092C1202091BC1B70
:109910008091C0209091C120820F911D9093C12011
:109920008093C0200BC02091BD1B8091BC1B90E098
:10993000820F911D9093BF1B8093BE1B2091C0206E
:109940003091C1202115310539F08091BE1B9091D5
:10995000BF1B28173907F9F409ED19E220EC3BE1A8
:109960004091BE1B5091BF1BC801B9010E94D6BADD
:109970006091BE1B7091BF1B1092BF1B1092BE1B4B
:109980001092C1201092C02010925B2910925A2987
:10999000C8010E9471682A960FB6F894DEBF0FBE08
:1099A000CDBFCF91DF911F910F91FF90EF90DF908E
:1099B000CF9008956F927F928F929F92AF92BF92B5
:1099C000CF92DF92EF92FF920F931F93DF93CF938B
:1099D000CDB7DEB72B970FB6F894DEBF0FBECDBF65
:1099E0003C01FE0131968BE0DF011D928A95E9F77B
:1099F00082E089832091990730919A07611471045C
:109A000039F48FEF9FEF9D838C833B832A8313C0B0
:109A10003B832A83F3014085423079F4308120E092
:109A2000818190E0822B932B9D838C8349838F5F70
:109A30009F4F09F0B8C050E0B7C0483009F09EC051
:109A4000D3012C9130E040E050E060E070E080E035
:109A500090E008E30E9422AF122FF32EE42ED52EC1
:109A6000C62EB72EA82E992EF301218130E040E0BA
:109A700050E060E070E080E090E000E30E9422AF00
:109A8000122BF32AE42AD52AC62AB72AA82A992A09
:109A9000D30117968C911797182B12962C9130E0C2
:109AA00040E050E060E070E080E090E008E20E947A
:109AB00022AF122BF32AE42AD52AC62AB72AA82ACB
:109AC000992AF301238130E040E050E060E070E04B
:109AD00080E090E000E20E9422AF122BF32AE42AF9
:109AE000D52AC62AB72AA82A992AD30114962C91D6
:109AF00030E040E050E060E070E080E090E008E1BD
:109B00000E9422AF122BF32AE42AD52AC62AB72AAA
:109B1000A82A992AF301258130E040E050E060E076
:109B200070E080E090E000E10E9422AF122BF32A67
:109B3000E42AD52AC62AB72AA82A992AD301169632
:109B40002C9130E040E050E060E070E080E090E098
:109B500008E00E9422AF122BF32AE42AD52AC62A53
:109B6000B72AA82A992A1C83FD82EE82DF82C88642
:109B7000B986AA869B8683E0898315C000D000D071
:109B800000D0EDB7FEB7319687EE97E0ADB7BEB720
:109B900012969C938E93119783EC97E09383828324
:109BA00080E395E029C051E08091592990E0FC01C3
:109BB000B3E0EE0FFF1FBA95E1F7E80FF91FEE597A
:109BC000F64D8085823029F1883011F483E022C07F
:109BD00000D000D000D0EDB7FEB7319687EE97E009
:109BE000ADB7BEB712969C938E93119783EC97E016
:109BF000938382838BE395E0958384830E94FCBBEF
:109C0000EDB7FEB736960FB6F894FEBF0FBEEDBFA8
:109C100015C082E02091552930915629BE016F5F11
:109C20007F4F4091572900E2E52ECC24AA248824B6
:109C30000E943E3B10925829109257292B960FB63E
:109C4000F894DEBF0FBECDBFCF91DF911F910F9172
:109C5000FF90EF90DF90CF90BF90AF909F908F904C
:109C60007F906F9008951F93CF93DF93EC01109234
:109C7000BD1B1092BB1B1092582910925729E091DE
:109C80005529F0915629F093BA1BE093B91B3296EF
:109C9000F093DB20E093DA20329780E68083809196
:109CA000BB1BE091B91BF091BA1BE80FF11D1182AB
:109CB0008091BB1BE091B91BF091BA1BE80FF11D1D
:109CC000128281EF99E20E94B045892B31F481EE36
:109CD00099E20E94B045892BB1F08091BB1B90E0C6
:109CE0000196E091B91BF091BA1BE80FF91F808132
:109CF000806880838091DA209091DB200196909398
:109D0000DB208093DA208091D929482F50E0909170
:109D1000DA299A0184E0220F331F8A95E1F7892F0F
:109D200082958F70822B282F269526958295880FF5
:109D3000880F807C282B692F70E0CB018F7090708A
:109D4000892B99F58091DB299091DC29892B69F584
:109D50008091BB1BE091B91BF091BA1BE80FF11D7C
:109D60008081886080838091D92990E08F70907085
:109D7000892B81F48091DA29807F61F48091BB1B6B
:109D8000E091B91BF091BA1BE80FF11D8081806151
:109D9000808355C0E091DA20F091DB202083809110
:109DA000DA209091DB20019646C04F705070452B11
:109DB00041F5862F807F29F58091BB1BE091B91B6F
:109DC000F091BA1BE80FF11D808180618083E091E2
:109DD000DA20F091DB20207C8091DA298F70282B0B
:109DE0002083E091DA20F091DB208091DB299091B3
:109DF000DC29928381838091DA209091DB20039685
:109E00001AC0E091DA20F091DB208091D92990915D
:109E1000DA29A091DB29B091DC2980839183A28388
:109E2000B383E091DA20F091DB2020838091DA2067
:109E30009091DB2004969093DB208093DA20809130
:109E4000DF29813161F48091BB1BE091B91BF09156
:109E5000BA1BE80FF11D8081846080830EC0E09101
:109E6000DA20F091DB2080838091DA209091DB2052
:109E700001969093DB208093DA208091E029803452
:109E800079F08F3FC9F0813011F58091BB1BE091D3
:109E9000B91BF091BA1BE80FF11D808181600AC0E7
:109EA0008091BB1BE091B91BF091BA1BE80FF11D2B
:109EB00080818260808319C08091BB1BE091B91BB7
:109EC000F091BA1BE80FF11D80818360F3CFE09120
:109ED000DA20F091DB2080838091DA209091DB20E2
:109EE00001969093DB208093DA208091E129909174
:109EF000E229892BB9F58091E3299091E429892BF6
:109F000089F58091E5299091E629892B59F5809171
:109F1000E7299091E829892B29F58091E9299091E9
:109F2000EA29892BF9F48091EB299091EC29892B6E
:109F3000C9F48091ED299091EE29892B99F48091B3
:109F4000EF299091F029892B69F48091BB1B90E057
:109F50000196E091B91BF091BA1BE80FF91F8081BF
:109F6000806446C081EE99E20E94B0459093D9206A
:109F70008093D820892B09F46EC08091BB1B90E0A0
:109F80000196E091B91BF091BA1BE80FF91F80818F
:109F9000806C80838091BB1B90E00296A091B91BDE
:109FA000B091BA1BA80FB91FE091D820F091D92029
:109FB00081818295807F9C91892B8C936091592916
:109FC00089E0689FB00111246E59764D81EE99E2C7
:109FD0000E940145882371F08091BB1B90E001969F
:109FE000E091B91BF091BA1BE80FF91F80818063E3
:109FF0008083B3C08091E9299091EA29892B81F46B
:10A000008091EB299091EC29892B51F48091ED29D5
:10A010009091EE29892B21F48091EF2987FF4AC086
:10A020008091BB1B90E00196E091B91BF091BA1BA7
:10A03000E80FF91F8081806180832091DA203091C0
:10A04000DB20C901DC01E9EEF9E288E001900D9224
:10A050008150E1F766C08091E1298E3F09F067C029
:10A060008091E229803809F062C06091592989E025
:10A07000689FB00111246E59764D81EE99E20E94DD
:10A080000145882309F0A8CF8091E9299091EA2918
:10A09000892B69F58091EB299091EC29892B39F571
:10A0A0008091ED299091EE29892B09F58091EF2976
:10A0B00087FD1DC08091BB1B90E00196E091B91B0C
:10A0C000F091BA1BE80FF91F808180628083E091D4
:10A0D000DA20F091DB208091EF299091F029918393
:10A0E00080838091DA209091DB20029632C08091AB
:10A0F000BB1B90E00196E091B91BF091BA1BE80FF1
:10A10000F91F8081806180832091DA203091DB20EB
:10A11000C901DC01E9EEF9E288E001900D9281507D
:10A12000E1F78091DA209091DB20089612C08091AF
:10A13000DA209091DB209C01D901E1EEF9E280E187
:10A1400001900D928150E1F78091DA209091DB200F
:10A1500040969093DB208093DA208091F1298F3F05
:10A1600009F0DDC08091BB1B90E00196E091B91B26
:10A17000F091BA1BE80FF91F80818860808380917D
:10A18000F229823009F042C08091F3299091F4299C
:10A19000892BE1F58091F5299091F629892BB1F56C
:10A1A0008091F7299091F829892B81F58091F929DF
:10A1B0009091FA29892B51F58091FB299091FC29E6
:10A1C000892B21F58091FD299091FE29892BF1F4AD
:10A1D0008091FF298823D1F48091BB1B90E00196E8
:10A1E000E091B91BF091BA1BE80FF91F80818360E1
:10A1F0008083E091DA20F091DB208091002A808337
:10A200008091DA209091DB20019671C18091F32931
:10A210009091F429892B09F074C08091F5299091CF
:10A22000F629892B09F06DC08091F7299091F829C2
:10A23000892B09F066C08091F9299091FA29892B20
:10A2400081F58091FB299091FC29892B51F5809112
:10A25000FD29882331F58091BB1B90E00196E091A8
:10A26000B91BF091BA1BE80FF91F808182608083CF
:10A27000E091DA20F091DB208091F2298083E09157
:10A28000DA20F091DB203196AEEFB9E283E00D9059
:10A2900001928150E1F78091DA209091DB200496C1
:10A2A00026C18091F9299091FA29892B51F5809145
:10A2B000FB29882331F58091BB1B90E00196E0914A
:10A2C000B91BF091BA1BE80FF91F80818160808370
:10A2D000E091DA20F091DB208091F2298083E091F7
:10A2E000DA20F091DB203196ACEFB9E285E00D90F9
:10A2F00001928150E1F78091DA209091DB2006965F
:10A30000F6C08091DA209091DB209C01D901E1EF29
:10A31000F9E280E101900D928150E1F7E3C081EF15
:10A3200099E20E94B0459093D9208093D820892B40
:10A3300009F459C08091BB1B90E00196E091B91BD4
:10A34000F091BA1BE80FF91F8081846080838091AF
:10A35000BB1B90E00296E091B91BF091BA1BE80F8D
:10A36000F91FA091D820B091D920808111969C919D
:10A37000892B808381EF99E2BE010E9401458823E9
:10A3800009F042C08091F9299091FA29892B81F432
:10A390008091FB299091FC29892B51F48091FD2912
:10A3A0009091FE29892B21F48091FF2987FF50C0CD
:10A3B0008091BB1B90E00196E091B91BF091BA1B14
:10A3C000E80FF91F8081816080832091DA2030912D
:10A3D000DB20C901DC01E9EFF9E288E001900D9290
:10A3E0008150E1F76CC08091F1298E3F09F06DC07A
:10A3F0008091F229803809F068C081EF99E2BE01AE
:10A400000E940145882371F08091BB1B90E001966A
:10A41000E091B91BF091BA1BE80FF91F80818360AE
:10A42000808369C08091F9299091FA29892B69F577
:10A430008091FB299091FC29892B39F58091FD2988
:10A440009091FE29892B09F58091FF2987FD1DC078
:10A450008091BB1B90E00196E091B91BF091BA1B73
:10A46000E80FF91F808182608083E091DA20F0910B
:10A47000DB208091FF299091002A91838083809135
:10A48000DA209091DB20029632C08091BB1B90E0D5
:10A490000196E091B91BF091BA1BE80FF91F80817A
:10A4A000816080832091DA203091DB20C901DC01BA
:10A4B000E9EFF9E288E001900D928150E1F7809197
:10A4C000DA209091DB20089612C08091DA209091DA
:10A4D000DB209C01D901E1EFF9E280E101900D92CE
:10A4E0008150E1F78091DA209091DB2040969093A3
:10A4F000DB208093DA2088E28093BD1B8091DF29E6
:10A50000813109F064C09091012A8091022A805B18
:10A51000904F0F9770F59091032A8091042A20EFB5
:10A52000803B920730F18F5B904F18F5E091DA2075
:10A53000F091DB2083EF8083E091DA20F091DB2043
:10A540009091042A905B8091022A8295807F980FD7
:10A550009183E091DA20F091DB208091072A90919D
:10A56000082A938382838091DA209091DB200496DD
:10A5700025C0E091DA20F091DB2080EF8083E0912C
:10A58000DA20F091DB208091012A9091022AA0919B
:10A59000032AB091042A81839283A383B483E09138
:10A5A000DA20F091DB208091072A9091082A968387
:10A5B00085838091DA209091DB2007969093DB20B1
:10A5C0008093DA208091BD1B885F8093BD1BA09192
:10A5D000DA208091B91BA81BA093BB1B8091BD1BE7
:10A5E000482F50E0E0915A29F0915B29E41BF50BCC
:10A5F0002A2F30E085E690E0821B930B6091B91B17
:10A600007091BA1B8E179F0708F0EAC0CB01049621
:10A610004A2F50E00E94DFBAE091B91BF091BA1BBB
:10A6200080915A2990915B29906C9083E091B91B9D
:10A63000F091BA1B80915A298183E091B91BF09166
:10A64000BA1B8091C3208283E091B91BF091BA1BA1
:10A650008091C22083838091BB1B8C5F8093BB1B46
:10A6600015E6412F481B487F4093BC1B6091B91BE6
:10A670007091BA1B680F711D2091BD1B30E02752ED
:10A68000364DCB01B90150E00E94D6BA2091BB1BD8
:10A690008091BC1B90E0820F911D9093582980936C
:10A6A0005729CE010E94DA4C2091BD1B8091BC1B22
:10A6B00090E0820F911D9093C1208093C02085E08F
:10A6C0008093BB1BE091B91BF091BA1B80915A2972
:10A6D00090915B29906E9083E091B91BF091BA1B29
:10A6E00080915A2981838091BB1B181B187F10937E
:10A6F000BC1B5CC0E091B91BF091BA1B13E036950E
:10A7000027951A95E1F7248360915A2970915B2966
:10A710004091C0205091C1209B01241B350B80919A
:10A72000BC1B90E02817390720F4862F841B8093E8
:10A73000BC1B8091BB1B6091B91B7091BA1B680F49
:10A74000711D4091BC1B2091C0203091C120275227
:10A75000364DCB01B90150E00E94D6BA2091BB1B07
:10A760008091BC1B90E0820F911D9093582980939B
:10A770005729CE010E94DA4C1092DC2007C00E94BB
:10A78000F03B8091DC208F5F8093DC208091DC2087
:10A790008233A8F32091BC1B8091C0209091C120EE
:10A7A000820F911D9093C1208093C0202091C020E2
:10A7B0003091C12080915A2990915B29281739073F
:10A7C00008F498CF8091C2209091C3200196909375
:10A7D000C3208093C2201092C1201092C0201CC0C0
:10A7E000260F371F4752564DC901BA01AF010E94CB
:10A7F000D6BA2091BB1B80915A2990915B29820F78
:10A80000911D2091BD1B821B910990935829809323
:10A810005729CE010E94DA4C81E0DF91CF911F9140
:10A820000895FC015381560F50936129272F332738
:10A830004281420F40936029A181A0935F29E0816A
:10A84000E0935E29842F90E08217930748F48A2FC3
:10A850008F5F80935F29882319F4EF5FE0935E296F
:10A86000852F90E070708617970790F4842F8F5F84
:10A8700080936029882361F480915F298F5F8093A2
:10A880005F29882329F480915E298F5F80935E2958
:10A8900008959C0141505040460F571FFB010EC0C8
:10A8A000708160E08181DB01A80FB11D2A0F3B1F81
:10A8B0002A173B0710F42F5F3F4F3296E417F50736
:10A8C00078F3E417F50749F4908180E0280F391FE9
:10A8D0002817390710F42F5F3F4FC90108959C01D5
:10A8E000AB0180E090E0B9010E944954282F892FE4
:10A8F000922F089580E090E069ED79E248E250E01F
:10A900000E944954009719F42FEF3FEF02C0382FEF
:10A91000292FC90108950F931F931091DD2900E09D
:10A920009091DE20091B11099091DE29090F111D5C
:10A930009801280F311DC90161EE79E240E250E033
:10A940000E9449546091DE2070E06F5F754DA80150
:10A950000E944954009719F42FEF3FEF02C0382F9F
:10A96000292FC9011F910F9108958AE30E948B54EA
:10A97000089586E00E948B54089581E10E948B54D3
:10A9800008950F931F93CF93DF93182F092F4091B2
:10A99000E1205091E220BCE24F5F5F4F8DE74030F5
:10A9A000580710F040E050E1342F252FA0E00EC0F2
:10A9B000AB9FF0011124E358F64D85A1882329F0BF
:10A9C000808991898217930739F3AF5FA23081F7AD
:10A9D0004093E1205093E2201092E020E0E0F0E08C
:10A9E00020E03CE21AC0239FD0011124A358B64DA9
:10A9F00095968C919597882321F42093E020FD0172
:10AA000010C0873049F4309731F096969C91969714
:10AA100086A1891708F4FD012F5F223020F32093CF
:10AA2000E020309771F182E085A38091E320808F50
:10AA30008091E420818F8091E520828F8091E620B3
:10AA4000838F84EC94E0978F868F91A380A381E01D
:10AA500090E0958F848F17A281E086A383E084A382
:10AA600012A280E183A3508B418B738B628BEF0129
:10AA7000212F302FC901DC0180E10D900992815016
:10AA8000E1F7CF01DF91CF911F910F910895AC01B4
:10AA90001092E02020E013C0E22FF0E0322F3F5F61
:10AAA000EE0FFF1FEB52F64D8081918184179507C1
:10AAB00029F42093E020118210820895232F223060
:10AAC00058F32093E0200895AC011092E02020E09C
:10AAD00012C0E22FF0E0322F3F5FEE0FFF1FEB526C
:10AAE000F64D80819181892B29F42093E0205183B8
:10AAF00040830895232F223060F32093E0200895AF
:10AB0000BC0180917B2990917C2944960E9411542C
:10AB1000E0917B29F0917C2980915E29848B809142
:10AB20005F29858B80916029868B80916129878B35
:10AB30000895282F892F922F0895EF92FF920F9357
:10AB40001F939C0144275527F22EE32E00E010E0CE
:10AB5000362F272F40E050E0A90133272227E22A91
:10AB6000F32A042B152BB701C8011F910F91FF90F9
:10AB7000EF900895FC0140915C2950915D2929EDE9
:10AB80003EE2241B350B621773070CF49B0112166F
:10AB9000130664F42093DB2E3093DC2EE417F507C4
:10ABA00029F0CA01BF01A9010E94D6BA089582E026
:10ABB0008093DF20A091DE202A2F30E0F901EF5FA3
:10ABC000F54D8181682F70E0F3E0660F771FFA95ED
:10ABD000E1F7695F7F4F42E0285D3F4F3CC0F901DC
:10ABE000E80FF91FE752F64D8081882319F0813074
:10ABF00019F42EC04F5F2FC090E0807C9070803899
:10AC0000910549F0803C910549F08034910501F5AA
:10AC10004093DF2009C04093DF2008C04093DF202D
:10AC20008091F1298F3F11F481E00895242F30E0C5
:10AC300040E050E02A0F311D411D511D285D3F4F5E
:10AC40004F4F5F4F84E062E00E94B66C82E008954F
:10AC500081818E5F480F842F90E0681779070CF090
:10AC6000BECF4093DF2080E008950F931F93CF93D2
:10AC7000DF93C0917B29D0917C29843009F4C5C22F
:10AC800005E11AE210937A290093792910935D293E
:10AC900000935C29833069F48DA18F70833011F0AB
:10ACA0000C94DA5E8C8D9D8D892B11F00C94DA5EFC
:10ACB00093C0823009F094C010925B2910925A29F7
:10ACC0001092DC2E1092DB2E8091E6208F5F809315
:10ACD000E620882399F48091E5208F5F8093E5201A
:10ACE000882361F48091E4208F5F8093E42088239F
:10ACF00029F48091E3208F5F8093E3202DA12730FA
:10AD000011F0253051F48EA18F5F8EA3883711F09A
:10AD10000C94DA5E1DA20C94DA5E222311F40C94DA
:10AD2000DA5E8C8D9D8D892B09F452C08EA18150E5
:10AD30008EA38F5F11F00C94DA5E3FA1383029F0BA
:10AD40002150223048F4353039F41DA280E8809338
:10AD500074290E949B6ED0C6353010F080E307C086
:10AD600083E090E002C0880F991F3A95E2F78EA326
:10AD70008FA18F5F8FA38DA190E08F709070833033
:10AD8000910501F1843091054CF48130910509F46D
:10AD900061C4029711F00C94DA5E0DC08630910503
:10ADA00009F4BEC68830910509F4BAC6049711F0BB
:10ADB0000C94DA5EB5C6E091DE20F0E0EF5FF54D71
:10ADC00015864FC484E0809374290E949B6ED6C67A
:10ADD0002F70233009F0EEC788E08093742980C675
:10ADE000853019F5E0917729F0917829808991894A
:10ADF000892B09F4DFC710927C2910927B29C801A6
:10AE00000C9790937A298093792990935D29809368
:10AE10005C291092DC2E1092DB2E10925B2910928E
:10AE20005A2988E080937429EEC18091D929807FC6
:10AE3000803609F0BFC79091DD2980E02091DE299E
:10AE4000AC01420F511D9A0180915A2990915B29C2
:10AE50008417950708F4AEC7285D3F4F30935B29F0
:10AE600020935A298091E1298F3F09F4A3C7C80193
:10AE7000849760E840E050E00E949862892B09F0D6
:10AE800067C0C80184970E940D60882309F060C0E4
:10AE90008091F1298F3F09F058C08091F2298230CA
:10AEA00009F053C08091F3299091F429892B09F07E
:10AEB0004CC08091F5299091F629892B01F580915C
:10AEC000F7299091F829892BD1F48091F929909153
:10AED000FA29892BA1F48091FB299091FC29892BD7
:10AEE00071F48091FD299091FE29892B41F4809184
:10AEF000FF29882321F48091002A813049F1809133
:10AF0000F5299091F629892B01F58091F7299091E7
:10AF1000F829892BD1F48091F9299091FA29892B6C
:10AF2000A1F48091FB299091FC29892B71F48091E7
:10AF3000FD299091FE29892B41F48091FF298823D6
:10AF400021F48091002A823019F00E94E95E3AC70C
:10AF50008FED99E290937629809375291092DE20E7
:10AF60001092DD20E0917529F091762980818B3255
:10AF700009F44BC08C3248F4863009F4B1C18131F8
:10AF800009F4B5C0882389F06BC08A3309F474C012
:10AF90008B3320F48C3209F063C00CC78B3309F477
:10AFA00009C78C3309F05CC006C08091DD2080FDAC
:10AFB00057C0816009C08091DD2081FF04C086FDFB
:10AFC0004FC0806401C082608093DD200E94D7550D
:10AFD000813009F4EFC6813018F0823019F6F2C6DC
:10AFE0002091DE20E22FF0E0CF018F5F954D90930E
:10AFF000762980937529285FFC018181880F880F4D
:10B00000880F280F2093DE20ADCF8091DD2082FDB8
:10B0100027C084608093DD209091DE20E92FF0E04E
:10B02000DF01AF5FB54D13968C911397882349F0DC
:10B03000BA969F01442737FD4095542F84E060E085
:10B0400018C0B0937629A0937529985FEF5FF54DEE
:10B050008181880F880F880F980F9093DE2082CF10
:10B06000E95DF9429F01442737FD4095542F84E064
:10B0700061E00E94B66CA6C60E94B5548F5F9F4FD8
:10B0800009F098C6E091DE20F0E0EF5FF54DE08139
:10B09000E538B9F0E63828F4E038B1F0E138D9F411
:10B0A00018C0E73829F0E73848F0E838A1F403C0C1
:10B0B0000E94007814C00E941C7611C00E94DD6FAF
:10B0C0000EC00E94087D0BC00E9412050E94956D63
:10B0D00006C00E94109C10925B2910925A29809100
:10B0E0005A2990915B29892B09F464C66BC680911B
:10B0F0005A2990915B29C09790935B2980935A2994
:10B1000089E09AE290937A2980937929E091DE2070
:10B11000F0E0EF5FF54D86819781892B31F00E9439
:10B12000BD548F5F9F4F09F045C68DED9EE2909311
:10B1300078298093772948C02889398921153105D4
:10B14000F1F18091DE20E82FF0E0EF5FF54D828194
:10B1500093818217930799F52A893B892115310537
:10B1600029F0808191818217930749F5888199811F
:10B17000892BE1F48A819B81892BC1F48C819D818B
:10B18000892BA1F48E819F81892B81F488859985F3
:10B19000892B61F48A859B85892B41F48C859D855B
:10B1A000892B21F48E859F85892BC1F081EE99E250
:10B1B000BE0140E150E00E94C9BA009779F069965B
:10B1C000D0937829C0937729C0917729D091782995
:10B1D000BFE2CF30DB0708F4AFCFECC510927C297B
:10B1E00010927B2982E08093742989E09AE29093FF
:10B1F0007A298093792990935D2980935C29109214
:10B20000DC2E1092DB2E0E945B6C2091DB2E3091A5
:10B21000DC2E2115310509F4CDC5C901C0969093E6
:10B220005B2980935A29285F3F4F3093DD2988524C
:10B230008093DE29A0917729B091782954968C913A
:10B2400054978093E02981E18093DF29E091DE200B
:10B25000F0E0EF5FF54D3483258317821682509618
:10B260008D919C9151979183808352968D919C9161
:10B27000539793838283A1EFB9E22091772930918C
:10B280007829C901FC0180E101900D928150E1F71C
:10B2900081EE99E261EF79E20E94F96385E19AE239
:10B2A00090937A29809379298091DE20C82FD0E06D
:10B2B000CF5FD54D0E94BD54809590959F838E831E
:10B2C0008091DE20E82FF0E0EF5FF54D86819781D9
:10B2D000892B09F065C58FEF9FEF9783868360C543
:10B2E0000E94B9548F5F9F4F09F064C58091DE20A2
:10B2F000082F10E00F5F154DCDE7D9E28DA188230F
:10B30000D9F0D80112962D913C911397888999898B
:10B310002817390789F42D913C918A899B89281730
:10B32000390751F481EE99E2BE0140E150E00E94FC
:10B33000C9BA009709F4B2C1AC96B9E2C93ADB07C1
:10B34000E9F2E0F2F80185858F73823001F58281A0
:10B3500093819093E9208093E8201092E02013C01D
:10B36000E42FF0E0EE0FFF1FEB52F64D2091E820A6
:10B370003091E920808191812817390709F489C02B
:10B380004F5F4093E0204091E020423048F38091AD
:10B39000DE20E82FF0E0DF01AF5FB54D1D968C9108
:10B3A0001D9782FD07C584E11D968C931D978CE344
:10B3B00090E090935B2980935A29FD0180E5848772
:10B3C00097811B968C911B9717968C931797938751
:10B3D00096811A968C911A9716968C931697928747
:10B3E000958119968C91199715968C93159791873D
:10B3F00094819093E02018968C91189714968C93D2
:10B40000149790871B968C911B978F5F1B968C933C
:10B410001B978823C1F41A968C911A978F5F1A96FE
:10B420008C931A97882379F419968C9119978F5FCA
:10B4300019968C931997882331F418968C91189744
:10B440008F5F18968C93E091DE20F0E0DF01AF5F14
:10B45000B54D2D913C9111973093E9202093E82030
:10B46000FD01828193819183808313963C932E9377
:10B470001297E1EFF9E2DF01509780E10D90019220
:10B480008150E1F781EE99E261EF79E20E94F96380
:10B4900054C41092E020C0E0D0E04CE250E03CE226
:10B4A00025C0822F90E0849FF001859FF00D949F2E
:10B4B000F00D1124E358F64D85A1882339F48CE270
:10B4C000289FE0011124C358D64D14C0873059F489
:10B4D000209721F096A18EA1891728F4239FE001DF
:10B4E0001124C358D64D2F5F2093E0202091E020F7
:10B4F0002230B8F2209709F45DC4D0937C29C09320
:10B500007B2983E08EA38CA31AA284E08BA31FA2C5
:10B51000E091DE20F0E0EF5FF54D82819381998B21
:10B52000888B808191819B8B8A8BDE01E1EEF9E231
:10B5300080E101900D928150E1F781E08DA380912F
:10B54000E320888F8091E420898F8091E5208A8F85
:10B550008091E6208B8F81E090E09D8F8C8FE09131
:10B56000DE20F0E0EF5FF54D87818F8BE091DE20EC
:10B57000F0E0EF5FF54D86818E8BE091DE20F0E00C
:10B58000EF5FF54D85818D8BE091DE20F0E0EF5F80
:10B59000F54D84818C8B81E090E00E948055E09194
:10B5A000DE20F0E0EF5FF54D848590E0807F9070C5
:10B5B000813591050CF44EC01092E02035C0F901A0
:10B5C000E752F64D84AD8093E720882309F442C00A
:10B5D000813021F44F5F4093E02026C08230C1F4D7
:10B5E00085AD8430A9F436AD20E087AD90E0822BA4
:10B5F000932B9093E9208093E820F4E0853C9F070B
:10B6000010F084EC94E09F8F8E8F99A388A322C0C2
:10B610008091E020E82FF0E0EA5EF54DE081EE2336
:10B62000C9F0E80FE093E0204091E020242F30E0C3
:10B63000E091DE20F0E0EF5FF54D848582958F701C
:10B6400090E00597880F991F880F991F28173907D1
:10B650000CF4B5CFE091DE20F0E0EF5FF54D80E136
:10B660008587E091DE20F0E0DF01AF5FB54D1D96EC
:10B670008C911D9782601D968C931D97FD0182E031
:10B68000848B84E0858B868B84EC878B80E490E0D0
:10B6900090935B2980935A2980E60EC3D0937C292E
:10B6A000C0937B29109274298091DE20A82FB0E0EE
:10B6B000FD01EF5FF54D858582FF03C01DA280E28D
:10B6C00093C2848582958F70880F880F8093E020C5
:10B6D00020915A2930915B2928523040281B31098A
:10B6E00030935B2920935A298DA18F70823039F4D1
:10B6F000AF5FB54D1D968C918F73823139F1232B3D
:10B7000059F4E091DE20F0E0EF5FF54D858590E0A3
:10B7100083709070892BD1F08091DE20E82FF0E0CB
:10B72000EF5FF54D94818C89981709F0B2C295812D
:10B730008D89981709F0ADC296818E89981709F006
:10B74000A8C297818F89981709F0A3C2E091DE20E3
:10B75000F0E0EF5FF54D858584FF52C06C8D7D8DE7
:10B760006115710509F44CC0CE0148960E94115430
:10B770008091DE20E82FF0E0EF5FF54D208580918D
:10B780005E292817E9F5918580915F299817C1F501
:10B79000928580916029981799F593858091612908
:10B7A000981771F5288F80915F29898F8091602982
:10B7B0008A8F809161298B8F8FA18823D1F42AA150
:10B7C0009CA18EA1981B822F869586958695981BA5
:10B7D000392F320F3AA38BA1282F26952695821B4D
:10B7E00097FD9195890F8BA3369536953695830FE6
:10B7F0008CA381E0809374298CA18EA31D8E1C8E56
:10B800008DA1282F30E0C9018F7090708430910590
:10B8100009F4EFC1853091055CF48230910591F116
:10B82000833091050CF0CAC0019709F0C3C210C063
:10B830008630910509F425C2863091050CF4FDC1CE
:10B840008730910509F425C2089709F0B3C2C6C133
:10B850008091742980FFAEC283E08DA380E4809341
:10B8600074291D8E1C8E20915A2930915B29211537
:10B87000310509F431C182E480937429C9010E9421
:10B8800080552AC18091742980FF8DC08091DE206F
:10B89000E82FF0E0EF5FF54D85858F73823109F079
:10B8A00082C0848590E0807F9070813591050CF492
:10B8B0004EC01092E02035C0F901E752F64D84AD3C
:10B8C0008093E720882309F442C0813021F44F5F40
:10B8D0004093E02026C08230C1F485AD8430A9F4C5
:10B8E00036AD20E087AD90E0822B932B9093E9203A
:10B8F0008093E82024E0853C920710F084EC94E0EB
:10B900009F8F8E8F99A388A322C08091E020E82F7B
:10B91000F0E0EA5EF54DE081EE23C9F0E80FE09338
:10B92000E0204091E020242F30E0E091DE20F0E0A4
:10B93000EF5FF54D848582958F7090E00597880FB5
:10B94000991F880F991F281739070CF4B5CF83E08A
:10B950008DA3E091DE20F0E0EF5FF54D84818C8BCC
:10B96000E091DE20F0E0EF5FF54D85818D8BE09179
:10B97000DE20F0E0EF5FF54D86818E8BE091DE20DA
:10B98000F0E0EF5FF54D87818F8B81E090E00E94C2
:10B99000805582E4809374291D8E1C8E10925B2941
:10B9A00010925A2999C080E2809374290E949B6E5C
:10B9B000E0917B29F0917C2915A2E9CC8091DE20D1
:10B9C000E82FF0E0EF5FF54D858580FF25C024FD71
:10B9D00023C08C8D9D8D892B09F0ECC180915A2953
:10B9E00090915B2901960E94805520917429822FA5
:10B9F00080618093742980915A2990915B29892BC9
:10BA000019F02261209374290E949B6E81E090E0DE
:10BA10009D8F8C8F88E082C085FF25C0328920E011
:10BA2000838990E0282B392B8091792990917A296C
:10BA3000820F931F90937A2980937929E091DE20D9
:10BA4000F0E0EF5FF54D328920E0838990E0282B0C
:10BA5000392B80915A2990915B29821B930B9093EB
:10BA60005B2980935A2920915A2930915B2921150D
:10BA7000310559F08DA184FD08C080917429826040
:10BA800080937429C9010E948055E091DE20F0E086
:10BA9000EF5FF54D968580E02785820F911D90938D
:10BAA000E9208093E82028A139A12817390710F050
:10BAB000892B21F43093E9202093E8208091E8201D
:10BAC0009091E9209F8F8E8F8091742990E08370F0
:10BAD0009070892B09F46EC11092DC2E1092DB2E2F
:10BAE0000E949B6E80917429282F85FF0CC01092B4
:10BAF000DC2E1092DB2E1DA2E091DE20F0E0EF5F45
:10BB0000F54D84E1CCC084FF12C01092DC2E10925F
:10BB1000DB2E81E090E09D8F8C8F84E08DA31FA2AF
:10BB2000E091DE20F0E0EF5FF54D81E1B8C080915B
:10BB3000DB2E9091DC2E892B01F120FF02C01D8E9F
:10BB40001C8E8C8D9D8D0097A1F42E8D3F8D809144
:10BB5000DB2E9091DC2E2817390720F43093DC2E51
:10BB60002093DB2E8091DB2E9091DC2E9D8F8C8F8D
:10BB700004C09093DC2E8093DB2E1FA280915C2961
:10BB800090915D2990937A29809379298091DB2E79
:10BB90009091DC2E892B81F08C8D9D8D009761F02A
:10BBA000CC9690935B2980935A29E091DE20F0E0B7
:10BBB000EF5FF54D88E110C08091742981FFFAC0D4
:10BBC0008CE390E090935B2980935A29E091DE20EA
:10BBD000F0E0EF5FF54D80E1858768C080917429C2
:10BBE00080FFE8C01DA280E1809374290E949B6EB3
:10BBF000E1C080915A2990915B29009711F00E9431
:10BC00008055E091DE20F0E0EF5FF54D8585909165
:10BC1000742980FF0BC090FF06C087E08DA31EA291
:10BC20001D8E1C8E1DC086E08DA31AC090FF22C001
:10BC300085E08DA31D8E1C8EBDC080915A299091E8
:10BC40005B29009711F00E948055E091DE20F0E022
:10BC5000EF5FF54D858580FF0DC087E08DA31EA2A7
:10BC600081E090E00E94805580E1809374290E94D9
:10BC70009B6E0FC080915A2990915B29892B49F4C2
:10BC800099C08091742980FF95C087E08DA31EA282
:10BC900091C0E091DE20F0E0EF5FF54D80E1858717
:10BCA0008CE390E090935B2980935A29E091DE2009
:10BCB000F0E0EF5FF54D80E58487E091DE20F0E075
:10BCC000EF5FF54D8C8980878D8981878E8982878A
:10BCD0008F898387888D8483898D85838A8D8683E8
:10BCE0008B8D878386E08093DF298889998991836A
:10BCF00080838A899B8993838283A1EFB9E2FE01C5
:10BD000080E101900D928150E1F781EE99E261EFBF
:10BD100079E20E94F9638DA1E091DE2084FF06C0E4
:10BD2000F0E0EF5FF54D1786168607C0F0E0EF5F95
:10BD3000F54D84E0868784EC87878091592990E0CF
:10BD400027E131E0829FF001839FF00D929FF00D7B
:10BD50001124E85DF04D84818093E02980915A2977
:10BD600090915B2988979093DD2980915A29885278
:10BD70008093DE29E091DE20F0E08F010F5F154D0A
:10BD8000D80153961C92539752961C92F801118A2F
:10BD9000108A0E94B95480959095F801918B808B00
:10BDA00080E68093D9291092DA291092DC2910922A
:10BDB000DB2908C010925B2910925A291092DE20CC
:10BDC0001092DD2010927429DF91CF911F910F9175
:10BDD00008951F9310915929212F30E087E191E0B8
:10BDE000289FF001299FF00D389FF00D1124E85D88
:10BDF000F04D8389882341F1109259290BC081EFBE
:10BE000099E20E9495828823C1F4809159298F5F1D
:10BE10008093592980915929823088F328C00E9443
:10BE2000B57E892B51F4809159298F5F80935929D0
:10BE300080915929823098F31DC08091E02981506A
:10BE40008093E029882329F410925B2910925A29C3
:10BE500017C089ED99E2489660E840E050E00E9402
:10BE60009862892B69F081E00E94355609C01092D2
:10BE70005929DECF10925B2910925A291093592923
:10BE80001F9108950F931F93CF93DF938C014091DF
:10BE9000E1205091E2204F5F5F4F8DE7403058071F
:10BEA00010F040E050E1342F252F8091ED2E90913D
:10BEB000EE2E8217930779F38091062F9091072F2A
:10BEC0008217930741F34093E1205093E2201092B0
:10BED000E02020E0A9E1B0E01CC0322F3F5F822FBC
:10BEE00090E08A9FF0018B9FF00D9A9FF00D112436
:10BEF000E352F14D80899189892B51F42093E02000
:10BF000089E1289FD0011124A352B14D49F434C0D6
:10BF1000232F223010F32093E020A0E0B0E02CC0CB
:10BF200050965C93509751964C93519753967C93AF
:10BF30006E9352970115110531F480E1ED011992CC
:10BF40008A95E9F707C0ED01F80180E101900992B7
:10BF50008150E1F78091592990E027E131E0829FFB
:10BF6000F001839FF00D929FF00D1124E85DF04DDC
:10BF7000848154968C935497CD01DF91CF911F917A
:10BF80000F910895CF92DF92EF92FF920F930E944C
:10BF900022670E94998480E009C0E82FF0E0EE0F4C
:10BFA000FF1FEB52F64D118210828F5F8230A8F393
:10BFB00020E04CE250E00DC0822F90E0849FF00121
:10BFC000859FF00D949FF00D1124E358F64D15A2B6
:10BFD0002F5F223088F380E094E09093E2208093FA
:10BFE000E12020E049E150E00EC0822F90E0849FE4
:10BFF000F001859FF00D949FF00D1124E352F14D57
:10C00000118A108A2F5F223080F32093E0200F9155
:10C01000FF90EF90DF90CF900895CF93DF93DC01F6
:10C020008C918F3F09F066C011968C9111978230E8
:10C0300009F060C012968D919C911397892B09F09D
:10C0400059C014968D919C911597892B09F052C077
:10C0500016968D919C911797892B09F04BC01896D5
:10C060008D919C911997892B09F044C01B968C9156
:10C070001B97813009F03EC01C968C911C978F3F16
:10C08000C9F51092F4202091592930E040E0CDE12B
:10C09000D0E087E191E0289FB001299F700D389F83
:10C0A000700D112423C0842F90E08C9FF0018D9F90
:10C0B000F00D9C9FF00D1124E60FF71FE85DF04D89
:10C0C00081A592A58F5F9F4F81F01D969C911D9732
:10C0D00086A1981751F417969C91179780A19817ED
:10C0E00021F44093F42081E006C04F5F4830D8F23D
:10C0F0004093F42080E0DF91CF91089540E020E06C
:10C1000030E0FC01E20FF31F5081FB01E20FF31F4F
:10C11000E0815E1731F4485F2F5F3F4F403889F769
:10C120000AC0E527842F885FE7FD05C04F5F4817E9
:10C1300011F0EE0FF9CF842F089588E29FE2089561
:10C14000E0915929F0E0DF01AB50BF4D1C92EE0F9A
:10C15000FF1FDF01A550BF4D6D917C91E950FF4D50
:10C16000808191810E94B27A08950E94E2B6AA2746
:10C1700097FDA095BA2FBC01CD0120E838E046EF2D
:10C1800057E10E9445B59B01AC012058324C424317
:10C19000544FB901CA0108954F925F926F927F92F6
:10C1A0008F929F92BF92CF92DF92EF92FF920F9366
:10C1B0001F938091592990E038E2C32E3FE2D32E9D
:10C1C00027E1422E21E0522E849DF001859DF00D45
:10C1D000949DF00D1124EC0DFD1D65817681878104
:10C1E00090850E94E6B320E030E040E05FE30E94EB
:10C1F0009CB40E94BAB33B014C010E94E2B6B82E37
:10C200000E94E2B6FB2CEE24E80EF91E00E010E0DE
:10C210008091592990E09C01249DC001259D900D9D
:10C22000349D900D1124C80ED91EF60165817681CA
:10C23000878190850E94E6B30E94BAB39B01AC014E
:10C24000C801B7010E9445B59B01AC01260D371D01
:10C25000481D591DB901CA011F910F91FF90EF9020
:10C26000DF90CF90BF909F908F907F906F905F9066
:10C270004F9008951F93CF93DF939C0110915929FC
:10C28000A12FB0E0FD01EB50FF4D8081882309F024
:10C290004AC02115310591F0CFEFD0E2F90180E1DC
:10C2A000019009928150E1F7FD01EE0FFF1FE95067
:10C2B000FF4D8FEF90E29183808307C0FD01EE0F69
:10C2C000FF1FE950FF4D118210826115710591F039
:10C2D000CFE0D1E2FB0180E1019009928150E1F7CA
:10C2E000FD01EE0FFF1FE550FF4D8FE091E29183BE
:10C2F000808307C0FD01EE0FFF1FE550FF4D118247
:10C300001082AB50BF4D81E08C930E94E2B66FEF7C
:10C310007FE70E9432B5AC01662757FD6095762F06
:10C32000812F0E949786DF91CF911F910895EF9200
:10C33000FF920F931F930E94B5607B018C01E091E7
:10C340005929F0E0EE50FF4D8081833078F481E090
:10C35000E81684E2F80684EF080780E0180730F05A
:10C36000E12C24E2F22E24EF022F112D80E090E048
:10C3700060E070E00E94B27A80915929E82FF0E0E5
:10C38000EE50FF4D90819F5F9083B801A7010E94FE
:10C39000D4861F910F91FF90EF90089580915929B5
:10C3A000A82FB0E087E191E0A89FF001A99FF00DD0
:10C3B000B89FF00D1124E85DF04D84898823E1F0E9
:10C3C000AE50BF4D8C918823B9F40E94B560AC018A
:10C3D000CB01DA01AC01BD01413084E2580784EFA2
:10C3E000680780E0780720F040E054E264EF70E0F6
:10C3F000809159290E94D48608951F93109159293C
:10C40000E12FF0E0E051FF4D8081882399F40E94F4
:10C41000E2B6AA2797FDA095BA2FBC01CD0120E86E
:10C4200034E84EE150E00E9467B5AB01BC01812FBA
:10C430000E9411871F9108950E94B57E892BD1F427
:10C44000E0915929F0E0E051FF4D8081843090F473
:10C450000E94C87380915929E82FF0E0E051FF4D08
:10C4600090819F5F908340E45BE46CE470E00E9405
:10C4700011870895809159290E945486E091592985
:10C48000F0E0E051FF4D10820E945B6B0895AF9287
:10C49000BF92CF92DF92EF92FF921F93CF93DF93E1
:10C4A0006C011092F4208091592990E03DE1A32E77
:10C4B000B12C27E131E0829F7001839FF00C929FA5
:10C4C000F00C112427C0812F90E08A9D90018B9D54
:10C4D000300D9A9D300D11242E0D3F1DF901E85DA0
:10C4E000F04DEF01A99681A592A58F5F9F4F79F03E
:10C4F000C9018F5B904DB60140E150E00E94C9BA7E
:10C50000009729F48FEF9FEF9983888307C01F5FFF
:10C510001093F4201091F4201830A8F2DF91CF91FD
:10C520001F91FF90EF90DF90CF90BF90AF90089554
:10C53000AF92BF92CF92DF92EF92FF920F931F9331
:10C54000CF93DF936C01062F7A011092F420209193
:10C55000592930E00695069506954DE1A42EB12C9B
:10C5600087E191E0289FE001299FD00D389FD00DF1
:10C57000112438C0212F30E02A9DF0012B9DF00DB1
:10C580003A9DF00D1124EC0FFD1FE85DF04D81A5E3
:10C5900092A58F5F9F4F19F184A995A98E159F05CC
:10C5A00019F0E114F104D9F42A9DC0012B9D900DDE
:10C5B0003A9D900D11248C0F9D1F8F5B904DB601FD
:10C5C000402F50E00E94C9BA009749F48DE1189FAE
:10C5D000900111242C0F3D1F2F5B304D09C01F5FB0
:10C5E0001093F4201091F420183020F220E030E075
:10C5F000C901DF91CF911F910F91FF90EF90DF90D4
:10C60000CF90BF90AF9008951F93CF93DF93BC015D
:10C6100010915929E12FF0E0EE0FFF1FE651FF4D79
:10C620008081918140E150E00E94C9BA0097B9F43D
:10C63000812F0E946086A0915929B0E0FD01EE0F84
:10C64000FF1FE651FF4D208131818FEF9FEFE90100
:10C65000998B888B11821082A251BF4D1C92DF9161
:10C66000CF911F9108951F93DC0150968D919C915D
:10C670005197892B09F510915929E12FF0E0EE0F20
:10C68000FF1FE651FF4D80819181892BA9F4B18371
:10C69000A0830E94E2B6AA2797FDA095BA2FBC01FD
:10C6A000CD0120E834E84EE150E00E9467B5AB01CF
:10C6B000BC01812F0E94A7871F9108951F93CF93DC
:10C6C000DF9320915929A22FB0E0FD01EE0FFF1F4B
:10C6D000E651FF4D408151814115510509F485C056
:10C6E000C7E1D1E0AC9FF001AD9FF00DBC9FF00D14
:10C6F0001124E85DF04DA251BF4D9C91808D98179B
:10C7000048F580E090E060E070E00E94E9741091EC
:10C710005929212F30E0F901E251FF4D80818F5FCF
:10C7200080832C9FF0012D9FF00D3C9FF00D112474
:10C73000E85DF04D658576858785908928EE33E044
:10C7400040E050E00E94FFB4AB01BC01812F0E9489
:10C75000A7874BC0822F0E9460862091592930E024
:10C76000F901EE0FFF1FE651FF4DA081B18181E07D
:10C7700090E051969C938E93509711821082F9010C
:10C78000E251FF4D10821092F42040E0ADE1B0E0A4
:10C790002C9FB0012D9F700D3C9F700D112421C066
:10C7A000242F2F5F842F90E08A9FF0018B9FF00D44
:10C7B0009A9FF00D1124E60FF71FE85DF04D81A55B
:10C7C00092A5892B69F44093F4208DE1489FC00124
:10C7D0001124860F971F8F5B904D0E94336305C015
:10C7E000422F4830E8F24093F420DF91CF911F911F
:10C7F00008955F926F927F928F929F92AF92BF92B5
:10C80000CF92DF92EF92FF920F931F93CF93DF931C
:10C81000682E592E7B01FB0180818E3F21F481819E
:10C82000803821F465C08F3F09F462C081E08093B5
:10C83000F420CC2400E0EDE18E2E912C77E1A72EA0
:10C8400071E0B72E69E0762E4CC08091592990E0B6
:10C850002D2D30E0289DE001299DD00D389DD00D73
:10C8600011248A9DB0018B9D700D9A9D700D11242D
:10C870006C0F7D1FFB01E85DF04D81A592A501972E
:10C8800059F56F5B704DC7010E947E60182F8C15A3
:10C8900018F160915929862F90E09C012A9DC001D2
:10C8A0002B9D900D3A9D900D11248C0F9D1F679D1F
:10C8B000B00111246E59764D8F5B904D0E94014559
:10C8C000882341F080915929813021F458E0C52E08
:10C8D000C10E01C0C12E0D2D8091F4208F5F809379
:10C8E000F420D090F42037E03D1508F0AECF44C0DE
:10C8F0001092F4200DE110E0C7E1D1E049E0F42E00
:10C9000036C060915929262F30E090E0809FA00129
:10C91000819F500D909F500D11242C9FC0012D9F81
:10C92000900D3C9F900D1124480F591FFA01E85DAE
:10C93000F04D818D8E3FB1F4828D803899F46F9DDA
:10C94000B00111246E59764DCA018F5B904D0E9443
:10C950000145882339F080915929813019F40091DB
:10C96000F4200AC08091F4208F5F8093F42080919E
:10C97000F420883030F200E0402F50E02091592917
:10C9800030E08DE190E0489FF001499FF00D589F05
:10C99000F00D112487E191E0AC01249FC001259F97
:10C9A000900D349F900D1124E80FF91F262D352D81
:10C9B000C901DC01EF5BF04D80E101900D928150E7
:10C9C000E1F7DF91CF911F910F91FF90EF90DF90F2
:10C9D000CF90BF90AF909F908F907F906F905F901F
:10C9E0000895CF93DF93FC01DB0118968C91189783
:10C9F000883039F4EF0128960D9009928150E1F7C3
:10CA00001BC08630E9F49F01285F3F4FAB0183E0F4
:10CA1000EA010990AE01E90109929E018150C1F736
:10CA20008FEF83878EEF8487EF012D96139683E037
:10CA30000D9009928150E1F7808592E0892714C01A
:10CA40008230B1F411968C91119787878C918687EB
:10CA500015868EEF84878FEF8387128680915731FA
:10CA60008187809156318D7F8087DF91CF910895A6
:10CA70008FEF9FEF0E94C0687F928F929F92AF923C
:10CA8000BF92CF92DF92EF92FF920F931F93CF93BB
:10CA9000DF93882E792E69017A010130110519F48E
:10CAA000603409F0C6C01092F42090905929A92C46
:10CAB000BB2440E0ADE1B0E087E191E0A89EB00189
:10CAC000A99E700DB89E700D1124AEC0C42FD0E089
:10CAD000542F5F5FCA9F9001CB9F300DDA9F300DBE
:10CAE0001124260F371FF901E85DF04D81A592A5AD
:10CAF0008F5F9F4F09F097C04093F420F901EF5BDF
:10CB0000F04D882D972D9C01D90180E10D90019267
:10CB10008150E1F70130110501F58DE190E09C01B4
:10CB2000C29FC001C39F900DD29F900D112427E199
:10CB300031E0A901A49E9001A59E300DB49E300D58
:10CB40001124820F931F69E0969EB00111246E5943
:10CB5000764D8F5B904D0E94F1648091592990E051
:10CB60002091F42030E0FDE1AF2EB12C2A9DA001F0
:10CB70002B9D500D3A9D500D1124C7E1D1E0BC0111
:10CB80006C9FC0016D9F900D7C9F900D1124480FEC
:10CB9000591FFA01E85DF04D12A611A615AB04ABC2
:10CBA000C114D104E104F10411F1CA018D5A904D70
:10CBB000B701A6010E9423862091F42030E08091E5
:10CBC000592990E02A9DF0012B9DF00D3A9DF00D22
:10CBD00011249C012C9FC0012D9F900D3C9F900D16
:10CBE0001124E80FF91FE85DF04D13AA02C081E09F
:10CBF00083AB8091F4202DE1829FC001112420910C
:10CC0000592930E047E151E0B901649F9001659FE7
:10CC1000300D749F300D1124820F931F8F5B904D48
:10CC20000E94336306C0452F483008F44FCF40932D
:10CC3000F420DF91CF911F910F91FF90EF90DF9043
:10CC4000CF90BF90AF909F908F907F900895EF927C
:10CC5000FF920F931F93CF93DF9381E08093F42093
:10CC60000DE110E0C7E1D1E0EE24EA94FE2C47C0CC
:10CC70008091592990E030E0209FA001219F500D24
:10CC8000309F500D11249C012C9FC0012D9F900DB1
:10CC90003C9F900D1124480F591FFA01E85DF04D9B
:10CCA00081A592A58F5F9F4F29F183A9813011F152
:10CCB000CA018D5A904D0E94FA85892BD9F0209196
:10CCC000F42030E08091592990E0209FF001219FCD
:10CCD000F00D309FF00D11249C012C9FC0012D9F61
:10CCE000900D3C9F900D1124E80FF91FE85DF04D69
:10CCF000F2A6E1A68091F4208F5F8093F42020912A
:10CD0000F420283008F4B4CFDF91CF911F910F9118
:10CD1000FF90EF9008959F92AF92BF92CF92DF92D3
:10CD2000EF92FF920F931F93DF93CF93CDB7DEB7B0
:10CD3000E2970FB6F894DEBF0FBECDBF1092F4207D
:10CD40000DE1A02EB12C17E1E12E11E0F12E8E01A4
:10CD50000F5F1F4FB7E1CB2EB8E0DB2EADE19A2E6F
:10CD60005AC02E2F30E08091592990E02A9DF00181
:10CD70002B9DF00D3A9DF00D1124AC014E9DC0018C
:10CD80004F9D900D5E9D900D1124E80FF91FE85DF9
:10CD9000F04D81A592A55FEF8F3F9507B9F1ADB733
:10CDA000BEB718970FB6F894BEBF0FBEADBFEDB7B4
:10CDB000FEB7319612961C930E931197D382C282BE
:10CDC00035832483978386830E946DBC2DB73EB73D
:10CDD000285F3F4F0FB6F8943EBF0FBE2DBF609146
:10CDE000F420699DB00111248091592990E0AC0193
:10CDF0004E9DC0014F9D900D5E9D900D1124680FBA
:10CE0000791F6F5B704DC8010E94748B8091F42074
:10CE10008F5F8093F420E091F420E83008F4A1CFF4
:10CE2000E2960FB6F894DEBF0FBECDBFCF91DF9173
:10CE30001F910F91FF90EF90DF90CF90BF90AF9038
:10CE40009F9008955F926F927F928F929F92AF9280
:10CE5000BF92CF92DF92EF92FF920F931F93CF93E7
:10CE6000DF933B014C01142F522EE601809159298A
:10CE700090E027E1A22E21E0B22E8A9D60018B9DD9
:10CE8000D00C9A9DD00C112428E23FE2C20ED31E92
:10CE900080E095E0A0E0B0E0F60180839183A2837A
:10CEA000B38380E4848380E395E7A0E0B0E08583EA
:10CEB0009683A783B0870E94CC60F6016187728752
:10CEC000838794878091592990E09C012A9DC00115
:10CED0002B9D900D3A9D900D1124FC01E85DF04DC5
:10CEE00028EE33E040E050E0258736874787508BB7
:10CEF00021E0208F728A618A138A148B558A068BEF
:10CF0000278B875C9F4CB70146E050E00E9421BB15
:10CF1000F09059296F2D70E020E00DE110E06A9D3E
:10CF2000A0016B9D500D7A9D500D1124AFEFBFEF06
:10CF300010C0822F90E0809FF001819FF00D909FA4
:10CF4000F00D1124E40FF51FE85DF04DB2A7A1A785
:10CF50002F5F283070F39B0183E0220F331F8A95E7
:10CF6000E1F7A901460F571FFA01EE59F64D8885E2
:10CF70008087E0E00BC0F0E0DA01AE0FBF1FAE59D2
:10CF8000B64DEC0FFD1F80818C93E92F9E2F9F5F84
:10CF90008885E81780F3E093F420C7E1D1E06C9F27
:10CFA000A0016D9F500D7C9F500D1124DA01A85DEA
:10CFB000B04DAF5FBE4F9FEF9D9382E08D931D926A
:10CFC0001D921D921D921D921D921D921D921D92E9
:10CFD00011E01D939D93F901E60FF71FEE59F64DF1
:10CFE0008085E80FF11D339781918D9381918D9309
:10CFF00080818C93A051B140552009F45AC08EEF26
:10D0000090E85A969C938E9359975C961C921E9228
:10D010005B975E961C921E925D9790961C921E9254
:10D020005F9792961C921E92919794961C921E92D4
:10D03000939796961C921E92959798961C921E9284
:10D04000979769E0F69EB00111246E59764DCA019A
:10D050008F5B904D0E94F1648091592990E0FC0112
:10D06000EC9FC001ED9F900DFC9F900D1124FC01E1
:10D07000E85DF04D12A611A623E030E035AB24ABFD
:10D0800013AB8F5B904D0E9433630E94FD6161146E
:10D0900071048104910469F08091592990E08C9F7A
:10D0A000F0018D9FF00D9C9FF00D1124E85DF04D77
:10D0B000138B8091592940E452E46FE070E00E94A4
:10D0C0004E87DF91CF911F910F91FF90EF90DF90EE
:10D0D000CF90BF90AF909F908F907F906F905F9018
:10D0E000089541E00E94488C0895CF93DF93EC01AE
:10D0F0008881833319F48981833389F020E030E01B
:10D10000FE01E20FF31FD901AE59B64D90818C910B
:10D11000981799F42F5F3F4F2630310589F78C859A
:10D120009D8586589D4D49F4109259296E50704046
:10D13000CE010E9640E00E94488CDF91CF91089579
:10D14000CF93DF9320915929E22FF0E0DF0124E013
:10D15000AA0FBB1F2A95E1F7AD53B94CEC0180E152
:10D1600009900D928150E1F784E0EE0FFF1F8A9540
:10D17000E1F7ED53F94C8FEF8787DF91CF91089559
:10D18000FFCF0F931F93CF93DF9380915A299091F4
:10D190005B29009709F458C18150954008F045C1BA
:10D1A0008091F1299091F229892B59F58091F329E9
:10D1B0009091F429892B29F58091F5299091F629F0
:10D1C000892BF9F48091F7299091F829892BC9F4DA
:10D1D0008091F9299091FA29892B99F48091FB2962
:10D1E0009091FC29892B69F48091FD299091FE2969
:10D1F000892B39F48091FF299091002A892B09F419
:10D2000014C18091F1298F3F09F414C180915929EB
:10D21000813071F48091760390917703892B41F4EA
:10D2200081EF99E20E949582882311F41092592986
:10D2300081EF99E20E949582882331F081EF99E293
:10D240000E946383EC0114C080915929813041F41C
:10D250008091760390917703892B11F410925929CC
:10D260000E94B57EFC01009709F4DFC0C081D18126
:10D27000209739F08A8D9B8D8530910509F065C026
:10D280000BC081EF99E260E070E040E020E030E028
:10D290000E94C883EC0102C01B8E1A8E88A98823C5
:10D2A00029F010925A311092593118AA80915931AF
:10D2B00090915A31892BA9F42DE531E33FA72EA790
:10D2C00040915A2950915B294093593150935A31DA
:10D2D000E9EDF9E2C901BF010E94D6BA80915A294D
:10D2E00088AB81EE99E260E840E050E00E949862ED
:10D2F000892B19F081EE99E202C080E090E060E0B5
:10D3000070E0AE010E94E9748091592990E027E114
:10D3100031E0829FF001839FF00D929FF00D112468
:10D32000E85DF04D658576858785908928EE33E048
:10D3300040E050E00E94FFB4AB01BC01CE018496F6
:10D340000E94238681E08CA775C0009729F588A9E3
:10D35000882329F010925A311092593118AA8091DD
:10D36000593190915A31892B09F06EC02DE531E386
:10D370003FA72EA740915A2950915B2940935931DC
:10D3800050935A31E9EDF9E2C901BF010E94D6BAC2
:10D3900080915A2988AB58C0029761F483E090E0ED
:10D3A0009B8F8A8FCE014C9640E45BE46CE470E086
:10D3B0000E9423868091592990E027E131E0829FE5
:10D3C000F001839FF00D929FF00D1124E85DF04D68
:10D3D000658576858785908928EE33E040E050E0CA
:10D3E0000E94FFB4AB01BC01CE0184960E9423864B
:10D3F0008E01005F1F4FC8010E94748548A9442315
:10D40000A1F040935A2910925B2929ED39E26EA5CB
:10D410007FA5C90150E00E94D6BA10925A311092ED
:10D42000593118AAC8010E94748510925B29109284
:10D430005A290AC080E090E00E94748510925B290E
:10D4400010925A291092DE20DF91CF911F910F91F7
:10D4500008950F931F93DF93CF93CDB7DEB76097F7
:10D460000FB6F894DEBF0FBECDBF8C0164367105D8
:10D4700020F0FC01108280E035C0FB01ED51F94C39
:10D480008081882319F4F80110822CC040918530E6
:10D4900050918630DE01119620E030E04130510598
:10D4A00019F4EDE1F0E002C0E0E0F0E0C901880F1E
:10D4B000991FE80FF91FE85AFF4C808191818D93E5
:10D4C0009D932F5F3F4F2730310541F7CB010E94DD
:10D4D0009955988B8F87C801BE016F5F7F4F0E945F
:10D4E000748B81E060960FB6F894DEBF0FBECDBF9F
:10D4F000CF91DF911F910F910895CF92DF92EF921C
:10D50000FF920F931F93DF93CF9300D0CDB7DEB779
:10D510001092592901EF19E28FEF92E09093F229CE
:10D520008093F1291092F4291092F3291092F62990
:10D530001092F5291092F8291092F7291092FA29E1
:10D540001092F9291092FC291092FB291092FE29C1
:10D550001092FD2980E092E09093002A8093FF29A9
:10D5600098EEE92E9FEFF92EE00EF11E89E0D7012B
:10D5700097968C93C8014097B8010E94F963109266
:10D58000DE2080E68093D929F7011182138212826E
:10D5900081E186832FEF278380E1C82ED12CC00E36
:10D5A000D11E82E099E0D60113969C938E93129738
:10D5B0009093022A8093012A80E094E315969C932D
:10D5C0008E93149717961C921E921697085E1F4F03
:10D5D00082E08093092A81E0F8018183138212821C
:10D5E000278B158A148A168A8091592990E027E1A1
:10D5F00031E0829FA001839F500D929F500D112416
:10D60000FA01E85DF04D84A995A9892BB1F0D70105
:10D61000D496FA01EF5BF04D80E101900D928150BC
:10D62000E1F781E0809359290E942E7F10925929B9
:10D63000FC01B29681A181FD05C010925B29109278
:10D640005A292EC021E23AE2AF0180E1DA010D90C1
:10D65000AD01D9010D929D018150C1F78089F8017A
:10D6600082A711A610A681E083A78CE590E0909395
:10D670005B2980935A2984E390E09A8389838A8185
:10D68000D70114968C931497898115968C930E94D8
:10D69000BD5480959095F601978386830E94C1685A
:10D6A0000F900F90CF91DF911F910F91FF90EF900E
:10D6B000DF90CF9008950F931F930E94B57E892B22
:10D6C00059F580915929E82FF0E034E0EE0FFF1F63
:10D6D0003A95E1F7ED53F94C87858823E9F01786F1
:10D6E000CF0160E420E030E040E050E001E00E9443
:10D6F000CC808091592990E024E0880F991F2A95C9
:10D70000E1F78D53994C60E420E030E040E050E0D8
:10D7100001E010E00E943C658091592990E007E10A
:10D7200011E0809FF001819FF00D909FF00D11247A
:10D73000E85DF04D83898823A1F00E94B57E892B96
:10D7400071F08091592990E0809FF001819FF00D48
:10D75000909FF00D1124E85DF04D128A118A0E940D
:10D76000CE610E948B661F910F9108958091592977
:10D77000813071F480918530909186308F5F9F4F1A
:10D7800009F185E790E30E9498450E9413050895EA
:10D79000809152308823B1F4809185309091863009
:10D7A0008F5F9F4F79F480916E2F90916F2F8F5FD5
:10D7B0009F4F41F080913D2F882321F08EE59FE21D
:10D7C0000E94984508958091A229882359F08DE7F9
:10D7D00099E290937C2980937B2982E00E943556C0
:10D7E0000E94C1688091CE29882359F089EA99E284
:10D7F00090937C2980937B2982E00E9435560E9479
:10D80000C16808950F931F93DF93CF93CDB7DEB711
:10D8100069970FB6F894DEBF0FBECDBF8C01E62F1F
:10D82000623708F03DC08091853090918630019735
:10D83000B9F580915B3190915C31892B89F58091AC
:10D840001F21882369F560935B3110925C312FE5CD
:10D8500036E3C901BA014E2F50E00E94D6BA81E0EA
:10D860008093592980EF93EB9A8B898B9C8B8B8BC0
:10D8700080E48D8BDE011196E5E7F0E380E1019015
:10D880000D928150E1F71F87088BCE01019690938E
:10D8900078298093772985E00E9435560E94C168D7
:10D8A00069960FB6F894DEBF0FBECDBFCF91DF9162
:10D8B0001F910F91089580917429883081F5E0912E
:10D8C0005B31F0915C31309709F44FC02FE536E3BE
:10D8D00080915C2990915D29B901AF010E94D6BA6F
:10D8E00080915B3190915C31E0915C29F0915D29F0
:10D8F000E80FF91F2DE020830196E0915C29F0915B
:10D900005D29E80FF91F2AE0208301969093DC2E11
:10D910008093DB2E10925C3110925B31089582303F
:10D9200021F581E080931F21E0915C29F0915D2930
:10D9300080915A2990915B29E80FF91F108200D03D
:10D9400000D087E298E0EDB7FEB7928381838091A3
:10D950005C2990915D29948383830E94FCBB109283
:10D960001F210F900F900F900F900895CF92DF928C
:10D97000EF92FF920F931F93CF93DF93D82EC62E73
:10D9800079018A011092DE20A2E2B1E2E1EFF9E230
:10D9900080E101900D928150E1F780915A29909198
:10D9A0005B29C09690935B2980935A2981509540BA
:10D9B00030F080E095E090935B2980935A2969EDDF
:10D9C00079E240915A2950915B2940535040CB0154
:10D9D000C0960E94DFBA80E68093D9291092DA2996
:10D9E0001092DC291092DB298AE38093DF29809151
:10D9F000592990E027E131E0829FF001839FF00DEB
:10DA0000929FF00D1124E85DF04D84818093E02910
:10DA10008091E1299091E229892B51F58091E329A8
:10DA20009091E429892B21F58091E5299091E629AF
:10DA3000892BF1F48091E7299091E829892BC1F491
:10DA40008091E9299091EA29892B91F48091EB2921
:10DA50009091EC29892B61F48091ED299091EE2928
:10DA6000892B31F48091EF299091F029892BD1F005
:10DA7000E1EFF9E2DF01509780E10D9001928150D2
:10DA8000E1F7809122218F3F91F484E0D81651F480
:10DA900022E0C21639F481EE99E262E271E20E945C
:10DAA000F9630EC010925B2910925A2935C0A1EE7D
:10DAB000B9E2E2E2F1E280E101900D928150E1F7FA
:10DAC000E091DE20CE2FD0E0FE01EF5FF54DD08259
:10DAD000C182C801B7010E949D55CB5FD54D6883B7
:10DAE00079838A839B8380915A2990915B298897B7
:10DAF0009093DD29889688528093DE298091DE20DC
:10DB0000C82FD0E0CF5FD54D1B821A820E94B5543A
:10DB1000809590959B838A83DF91CF911F910F9180
:10DB2000FF90EF90DF90CF90089549ED59E28091FA
:10DB3000592990E027E131E0829FF001839FF00DA9
:10DB4000929FF00D1124E85DF04D84818093E029CF
:10DB50008091F1298F3F81F4DA015896FA013896C5
:10DB600080E101900D928150E1F781EE99E261EF41
:10DB700079E20E94F9631BC0A2E2B1E2FA01389691
:10DB800080E101900D928150E1F7E1EEF9E2DF01D1
:10DB9000509680E10D9001928150E1F7A1EFB9E23A
:10DBA000E2E2F1E280E101900D928150E1F76091B3
:10DBB000DE20662301F18AE38093DF2970E0409143
:10DBC0005A2950915B29461B570B50935B29409370
:10DBD0005A29485250405093DD29485D5F4F842FA9
:10DBE00088528093DE296B5F754D4C52504085E022
:10DBF0009AE20E94DFBA1092DE2081E88093012A27
:10DC00001092022A1092042A1092032A0E94B554FC
:10DC1000809590959093042A8093032A08950F93FA
:10DC20001F93CF93DF9320E62093D9291092DA290E
:10DC30001092DC291092DB292AE32093DF2920911E
:10DC4000592930E047E151E0249FF001259FF00D74
:10DC5000349FF00D1124E85DF04D24812093E029DC
:10DC6000A1EFB9E2FC0180E101900D928150E1F752
:10DC700081EE99E261EF79E20E94F9638AE3809391
:10DC8000DF2980E390E090935B2980935A2980916B
:10DC90002021909121210196909321218093202190
:10DCA0002091DE20C22FD0E0CB5FD54D19821882A3
:10DCB0000E9499559B838A838091DE20482F50E0F3
:10DCC00020915A2930915B29FA01EB5FF54D81E6ED
:10DCD000848331968F5F8138D9F7C90180969093FC
:10DCE0005B2980935A29285030403093DD2988528F
:10DCF0008093DE298A010F5F154D80E8F80180834B
:10DD00001182138212820E94B55480959095F80179
:10DD1000938382838091202190912121DF91CF9163
:10DD20001F910F910895FC0171A760A70895FC0150
:10DD3000768B658B0895A0917B29B0917C291097F3
:10DD400019F0FD01B89605C0E0917729F091782986
:10DD500075968091742986FF22C050962D913C9132
:10DD6000519780913421909135218217930731F496
:10DD70008091362190913721009769F48091382164
:10DD8000909139218217930751F480913A21909113
:10DD90003B21009721F0918380831382128220819E
:10DDA00031812115310521F082819381F901099595
:10DDB0000895009749F090937C2980937B2983E014
:10DDC0000E9435560E94C1680895009749F09093CB
:10DDD00078298093772985E00E9435560E94C16892
:10DDE0000895CF93DF93EC018091362190913721F4
:10DDF0008C179D0771F480913421909135210E94F8
:10DE000047551092352110923421109237211092EB
:10DE1000362180913A2190913B218C179D0771F416
:10DE200080913821909139210E94475510923921D3
:10DE30001092382110923B2110923A21E2EAF9E245
:10DE4000838194818C179D0719F4148213821082A8
:10DE5000BC96CF018597855D994290F3EDEDFEE28A
:10DE6000858996898C179D0711F4118A108A7996F5
:10DE70008FE2EF30F807A0F3DF91CF910895AC0166
:10DE800010923321E4E3F1E220E014C0808191811B
:10DE90008417950769F4828193818617970741F467
:10DEA0002093332111821082CA010E9447550895A0
:10DEB00034962F5F223050F3209333210895CF936F
:10DEC000DF93EA010E94425FFC01009711F0D68BBC
:10DED000C58BCF01DF91CF910895EF92FF920F9301
:10DEE0001F93DF93CF93CDB7DEB760970FB6F8944B
:10DEF000DEBF0FBECDBF8C017B018FEF92E09A8316
:10DF000089831C821B821E821D8218861F821A86AC
:10DF100019861C861B861E861D8680E091E0988BE4
:10DF20008F87CE010196B8010E94425FFC010097E5
:10DF300021F0F68AE58A118B008BCF0160960FB62F
:10DF4000F894DEBF0FBECDBFCF91DF911F910F912F
:10DF5000FF90EF900895AC0110923221E4E3F1E2DA
:10DF600020E012C0322F3F5F80819181892B51F4D4
:10DF7000209332215183408373836283CA010E94BC
:10DF8000645508953496232F223060F32093322174
:10DF900008950F931F93CF93DF938A010E94C1547A
:10DFA000EC01009721F019A708A70E94D96ECE01B5
:10DFB000DF91CF911F910F9108959F92AF92BF92E1
:10DFC000CF92DF92EF92FF920F931F93CF93DF9345
:10DFD0008091592990E027E131E0829FE001839F01
:10DFE000D00D929FD00D1124C85DD04D8F8988230C
:10DFF00009F4C2C38091E0298F3F09F0B3C3809137
:10E00000E1298E3F09F0AEC38091E229803809F002
:10E01000A9C38091DE20A82FB0E0FD01EF5FF54D90
:10E020008181882309F09EC3AB5FB54D8C9181112E
:10E030008C83E091DE20F0E0EB5FF54D24813581AB
:10E0400046815781211531054105510509F448C024
:10E050008091592990E0C7E1D1E08C9FF0018D9F1C
:10E06000F00D9C9FF00D1124E85DF04DE580F680E9
:10E0700007811085CA01B9010E949D55E616F70671
:10E080000807190769F10091592910E0E091DE2095
:10E09000F0E0EB5FF54D64817581868197810E9488
:10E0A0009D550C9FF0010D9FF00D1C9FF00D11244C
:10E0B000E85DF04D658376838783908700915929C9
:10E0C00010E00E94CC600C9FF0010D9FF00D1C9F92
:10E0D000F00D1124E85DF04D618772878387948786
:10E0E000E091DE20F0E0EB5FF54D60857185828583
:10E0F00093856115710581059105A1F0009159295C
:10E1000010E00E949D5527E131E0029FF001039F3E
:10E11000F00D129FF00D1124E85DF04D65877687B4
:10E120008787908B1092402110923F2110924221BC
:10E130001092412140E009C0E42FF0E0EE0FFF1FF4
:10E14000ED5BFE4D118210824F5F4430A8F3409387
:10E1500053218CE080933E2160915A2970915B2974
:10E160003AC0F901E752F64D8181882309F4F8C2DB
:10E170008081833071F0853039F08130E1F4F093A3
:10E180004021E0933F2117C0F0934221E0934121C9
:10E1900012C040E0443079F0542F5F5FE42FF0E08C
:10E1A000EE0FFF1FED5BFE4D80819181892B09F4FD
:10E1B000DEC2452FEFCF80913E21E091DE20F0E0DE
:10E1C000E752F64DE80FF11D95A5990F990F990F9C
:10E1D000980F90933E219091DE2080913E21282F30
:10E1E00030E0290F311D245D3F4F2617370708F413
:10E1F000B8CF40935321E0914121F09142213097D3
:10E20000C1F00091592910E0648175818681978160
:10E210000E949D5527E131E0029FF001039FF00D20
:10E22000129FF00D1124E85DF04D608371838283AD
:10E230009383109253219924939480C164817581B2
:10E24000868197810E949D557B018C01E09153212D
:10E25000F0E0EE0FFF1FED5BFE4D0190F081E02D31
:10E2600060857185828593850E949D55E616F70627
:10E270000807190708F45DC1E0915321F0E0EE0FA3
:10E28000FF1FED5BFE4D0190F081E02D80898E3FF8
:10E2900021F48189803809F44CC1838187FF7CC0D7
:10E2A000CF0140960E942C82EC0190934E218093E6
:10E2B0004D21E09153210097C1F5F0E0EE0FFF1FD3
:10E2C000ED5BFE4D0190F081E02D648175818681CA
:10E2D0009781611571058105910509F45DC0EF0114
:10E2E00060966F3F2FEF72072FEF82072FEF920795
:10E2F00071F012810E949D5520E432E44FE050E01D
:10E300000E94FFB49B01AC01CE01612F06C0CE017B
:10E31000628120E030E040E050E000E00E94CC80EC
:10E3200090934E2180934D2137C0F0E0EE0FFF1FF8
:10E33000ED5BFE4D0190F081E02D64817581868159
:10E340009781611571058105910549F06F3FEFEFE8
:10E350007E07EFEF8E07EFEF9E0749F404C0CE0172
:10E360000E94297F19C089A1816089A315C00E94DC
:10E370009D5520E432E44FE050E00E94FFB4AB0131
:10E38000BC01CE0141960E942386E0914D21F0917F
:10E390004E2181A18E7F81A3E0915321F0E0EE0F09
:10E3A000FF1FED5BFE4D0190F081E02D838186FF24
:10E3B000C0C084819581A681B7810097A105B10570
:10E3C00009F4B7C0CF014096628141E050E00E945D
:10E3D0009862DC019093522180935121E091532166
:10E3E000009709F478C0F0E0EE0FFF1FED5BFE4DE3
:10E3F0000190F081E02D64817581868197816F3F66
:10E40000FFEF7F07FFEF8F07FFEF9F0709F460C063
:10E410000E949D5561527C418040904040F5E091C2
:10E420005321F0E0EE0FFF1FED5BFE4D0190F081F8
:10E43000E02D64817581868197810E949D557B01C5
:10E440008C01809151219091522142960E94D58554
:10E450005B016C01C801B70120E432E44FE050E0F9
:10E460000E94FFB4A616B706C806D90600F50091AB
:10E470005121109152210E5E1F4FE0915321F0E087
:10E48000EE0FFF1FED5BFE4D0190F081E02D6481EA
:10E490007581868197810E949D5520E432E44FE08A
:10E4A00050E00E94FFB4AB01BC01C80109C08091DB
:10E4B000512190915221429640E058E467E27DEA72
:10E4C0000E942386E0915121F0915221128E31C099
:10E4D0005A969C922EC0F0E0EE0FFF1FED5BFE4DB2
:10E4E0000190F081E02D6481758186819781EF0133
:10E4F00060966F3F2FEF72072FEF82072FEF920783
:10E5000071F012810E949D5520E432E44FE050E00A
:10E510000E94FFB49B01AC01CE01612F06C0CE0169
:10E52000628120E030E040E050E001E010E00E9435
:10E530003C65809153218F5F80935321E09153215B
:10E54000E43058F4F0E0EE0FFF1FED5BFE4D01905C
:10E55000F081E02D309709F071CE81EE99E20E94B2
:10E560006383FC0190934C2180934B2160913F2168
:10E57000709140216115710509F461C0009771F433
:10E580006E5F7F4F81EE99E241E022E030E00E9431
:10E59000C88390934C2180934B2151C0828D938DE1
:10E5A000892B21F482E090E0938F828F209159296A
:10E5B000822F90E0FC0133E0EE0FFF1F3A95E1F768
:10E5C000E80FF91FEE59F64DA084213061F4E09177
:10E5D0003F21F09140218181813019F098E0A92EEE
:10E5E00002C082E0A82E00913F21109140210E5FD1
:10E5F0001F4FE0904B21F0904C21E7016096C8013D
:10E60000BE014A2D50E00E94C9BA009721F4F701DB
:10E61000808DA81671F0CE01B8014A2D50E00E94FD
:10E62000D6BAE0914B21F0914C2182E090E0938F9B
:10E63000828FE0914B21F0914C2181E0818FE0911C
:10E64000DE20F0E0EB5FF54D82819381E0914B217C
:10E65000F0914C21892B09F454C0309771F481EE6C
:10E6600099E260E070E041E025E030E00E94C8837C
:10E6700090934C2180934B2102C081E0818F809147
:10E680004B2190914C210E94677E8C0190935021E8
:10E6900080934F21E091DE200097D9F400914B2127
:10E6A00010914C21F0E0EB5FF54D828193810E9447
:10E6B0009955A0E0B0E0BC01CD0120E432E44FE088
:10E6C00050E00E94FFB4AB01BC01C8010E94A481CC
:10E6D00025C0F0E0EB5FF54D828193810E94995552
:10E6E000A0E0B0E0BC01CD0120E432E44FE050E016
:10E6F0000E94FFB4AB01BC01C80102960E942386B0
:10E700000DC0309759F0CF010E94677E9093502141
:10E7100080934F21009711F00E941E7FE0914B21C2
:10E72000F0914C213097C9F040A94423B1F04093B7
:10E730005A2910925B2929ED39E266A577A5C9010E
:10E7400050E00E94D6BA10925A3110925931E0919D
:10E750004B21F0914C2110AA0FC00E94B66B02C051
:10E760004093532110925B2910925A2905C02752D9
:10E77000364D318320831FCDDF91CF911F910F91B3
:10E78000FF90EF90DF90CF90BF90AF909F90089553
:10E79000EF92FF920F931F93DF93CF9300D0CDB7EB
:10E7A000DEB780915929282F30E087E191E0289F3A
:10E7B000F001299FF00D389FF00D1124E85DF04D18
:10E7C0008789882309F4FCC0F90183E0EE0FFF1F5D
:10E7D0008A95E1F7E20FF31FEE59F64D2085822F5F
:10E7E00090E00296022F0E5F87709070081B892BB5
:10E7F00009F0085F89ED99E220E62093D92910926B
:10E80000DA291092DC291092DB292AE32093DF29F0
:10E810002FEF2093E029FC0178962FEF32E0309320
:10E82000F2292093F1291382128215821482178211
:10E83000168211861086138612861586148620E0AD
:10E8400032E0378726870896BF010E94F96320913E
:10E85000DE20A22FB0E0FD01EF5FF54D85E880835B
:10E860001182FD01EB5FF54D10821182128213823D
:10E870001092DD298091E1299091E229892B99F567
:10E880008091E3299091E429892B69F58091E5290C
:10E890009091E629892B39F58091E7299091E82913
:10E8A000892B09F58091E9299091EA29892BD9F4DE
:10E8B0008091EB299091EC29892BA9F48091ED2985
:10E8C0009091EE29892B79F48091EF299091F0298C
:10E8D000892B49F488E08093DE29D096B0935B2998
:10E8E000A0935A295DC0E02EFF24822F90E0C096AD
:10E8F0008E0D9F1D90935B2980935A29085F00938A
:10E90000DE290850A75FB54DB0934021A0933F2169
:10E9100081E08C9306950695069511960C931197B8
:10E92000209159291296822F90E0FC0103E0EE0F0E
:10E93000FF1F0A95E1F7E80FF91FEE59F64D4085E4
:10E9400089E0289F900111242E59364DCD01B9013F
:10E9500050E00E94D6BA8091592990E0FC0113E062
:10E96000EE0FFF1F1A95E1F7E80FF91FEE59F64D6C
:10E97000808590E09701281B390B225030403A8364
:10E98000298320913F21309140212E5F3F4F280F56
:10E99000391FC90160E070E049815A810E94F1BAD3
:10E9A0008091DE20082F10E00F5F154DF8011382D3
:10E9B00012820E94B55480959095F80193838283CA
:10E9C0000F900F90CF91DF911F910F91FF90EF90DB
:10E9D0000895FF920F931F93CF93DF938C01EA0169
:10E9E00080915929282F30E087E191E0289FF0019C
:10E9F000299FF00D389FF00D1124E85DF04D8789B7
:10EA0000882309F413C1F90153E0EE0FFF1F5A9553
:10EA1000E1F7E20FF31FEE59F64D2085822F90E0CB
:10EA2000029642E0F42EF20E87709070F81A892B4D
:10EA300011F088E0F80E1092DE2080E68093D9294C
:10EA40001092DA291092DC291092DB298AE3809354
:10EA5000DF299FEF9093E029E1EFF9E2611571055D
:10EA6000B9F49093F12982E0818313821282158296
:10EA700014821782168211861086128681E083879F
:10EA800094878D8585878E859F859787868707C024
:10EA9000DF01FB0180E101900D928150E1F787E8F1
:10EAA0008093012A1092022A1092052A1092062AB7
:10EAB0001092072A1092082AA9E0BAE2FE0180E12A
:10EAC00001900D928150E1F71092DD29CE0160E8AE
:10EAD00040E050E00E949862892B09F070C0011557
:10EAE000110549F0A1EEB9E2F80180E101900D9223
:10EAF0008150E1F706C081EE99E261EF79E20E9470
:10EB0000F96388E1F80EF092DE2988EEF80E0F2DF9
:10EB100010E0005C1F4F10935B2900935A290054AA
:10EB20001040A091DE20B0E0A75EB54DB09340212B
:10EB3000A0933F2181E08C93F694F694F69411967D
:10EB4000FC921197209159291296822F90E0FC0196
:10EB500033E0EE0FFF1F3A95E1F7E80FF91FEE598A
:10EB6000F64D408589E0289F900111242E59364D9D
:10EB7000CD01B90150E00E94D6BA8091592990E0A8
:10EB8000FC0123E0EE0FFF1F2A95E1F7E80FF91FC4
:10EB9000EE59F64D808590E0081B190B025010408D
:10EBA00020913F21309140212E5F3F4F280F391F88
:10EBB000C90160E070E0A8010E94F1BA29C010927A
:10EBC000E2291092E1291092E4291092E32910928F
:10EBD000E6291092E5291092E8291092E72910926F
:10EBE000EA291092E9291092EC291092EB2910924F
:10EBF000EE291092ED291092F0291092EF2988E168
:10EC00008093DE2980E490E090935B2980935A29D9
:10EC10008091DE20C82FD0E0CF5FD54D1B821A82B5
:10EC20000E94B554809590959B838A83DF91CF9104
:10EC30001F910F91FF900895BF92CF92DF92EF92B4
:10EC4000FF920F931F93DF93CF93CDB7DEB72B9730
:10EC50000FB6F894DEBF0FBECDBF8091592990E06A
:10EC600027E131E0829FF001839FF00D929FF00D2C
:10EC70001124E85DF04D8789882309F4B1C1909192
:10EC8000DE20E92FF0E0DF01AB5FB54DDC90809135
:10EC9000E0298F3F09F0A0C1EF5FF54D8181882306
:10ECA00009F09AC114968C9114978F3F09F494C17E
:10ECB000E0E4BE2EBD20D6FE05C08091F1298F3F35
:10ECC00009F48AC184E180933E2110924021109280
:10ECD0003F2160915A2970915B29292F30E0245DF2
:10ECE0003F4FA9014752564D1AC0FC01E752F64D5D
:10ECF0008181882309F470C18081823021F4F093EE
:10ED00004021E0933F2180913E21FA01E80FF11D5F
:10ED10009181990F990F990F980F90933E218091AF
:10ED20003E21F901E80FF11DCF01E617F707E8F2E0
:10ED3000CD01049660E840E050E00E949862FC013A
:10ED40009093522180935121009769F08089918995
:10ED5000892B09F041C18091DE2090E0875F954DBD
:10ED60000E94046339C18091DE2090E0875F954D59
:10ED70000E94638390934C2180934B21892B09F44B
:10ED80002BC120915929822F90E0FC0173E0EE0FF6
:10ED9000FF1F7A95E1F7E80FF91FEE59F64D008550
:10EDA000213051F4E0913F21F09140218181813067
:10EDB00011F008E001C002E020913F213091402194
:10EDC0002E5F3F4FCE010196B901402F50E00E94C7
:10EDD000D6BA0987E0903F21F0904021E114F10478
:10EDE00011F410E018C080914B2190914C219B8729
:10EDF0008A87BC01605F7F4FC7010296402F50E0B9
:10EE00000E94C9BA982FEA85FB85808D081711F0FA
:10EE100011E001C0192F60E8C62ECD20E0914B21F2
:10EE2000F0914C21828D938D009709F045C0E1143B
:10EE3000F10409F4D1C09F01205F3F4FA7014E5F4D
:10EE40005F4FC901BA01402F50E00E94D6BAE0914D
:10EE50004B21F0914C21008FE0904B21F0904C2100
:10EE6000BB2021F181E090E0F701938F828F8091A8
:10EE7000592990E027E131E0829FF001839FF00D56
:10EE8000929FF00D1124E85DF04D618572858385B8
:10EE9000948528EE33E040E050E00E94FFB4AB01DF
:10EEA000BC01C7014C960E94238674C082E090E0AA
:10EEB000F701938F828F6EC0D5FC0AC0112341F0F9
:10EEC000019709F089C082E090E0938F828F84C01F
:10EED000E114F10489F09F01205F3F4FA7014E5FCD
:10EEE0005F4FC901BA01402F50E00E94D6BAE091AD
:10EEF0004B21F0914C21008FBB2041F1E0904B2140
:10EF0000F0904C2181E090E0F701938F828F809107
:10EF1000592990E027E131E0829FF001839FF00DB5
:10EF2000929FF00D1124E85DF04D61857285838517
:10EF3000948528EE33E040E050E00E94FFB4AB013E
:10EF4000BC01C7014C960E94238610C080913F21CE
:10EF500090914021892B51F0112341F0E0914B21F8
:10EF6000F0914C2182E090E0938F828FE0914B21D1
:10EF7000F0914C21818D882369F0CC2059F4CF0188
:10EF80000E94677E9093502180934F21009711F04B
:10EF90000E941E7FE0914B21F0914C21C18EE091A7
:10EFA0004B21F0914C2140A94423B1F040935A29C0
:10EFB00010925B2929ED39E266A577A5C90150E0D9
:10EFC0000E94D6BA10925A3110925931E0914B21D9
:10EFD000F0914C2110AA04C010925B2910925A297A
:10EFE0002B960FB6F894DEBF0FBECDBFCF91DF9149
:10EFF0001F910F91FF90EF90DF90CF90BF900895F9
:10F00000BF92CF92DF92EF92FF920F931F93DF9305
:10F01000CF93CDB7DEB729970FB6F894DEBF0FBEFA
:10F02000CDBF50915929652F70E087E191E0689F2D
:10F03000F001699FF00D789FF00D1124E85DF04D0F
:10F040008789882309F47EC28091E0298F3F09F0E7
:10F0500075C28091DE20282F30E0F901EB5FF54D7D
:10F0600084818F3F09F46AC2F901EF5FF54D818118
:10F07000882309F063C21092402110923F2184E15D
:10F0800080933E2100915A2910915B2944E1F901B6
:10F09000BC9616C0DC01A752B64D11968C91119703
:10F0A000882309F449C28C91813021F4B093402126
:10F0B000A0933F2111968C91880F880F880F480FDD
:10F0C000CF01840F911D8017910720F340933E21BB
:10F0D000A0913F21B0914021109709F499C08091EF
:10F0E000E1299091E229892B59F58091E3299091AA
:10F0F000E429892B29F58091E5299091E629892B2E
:10F10000F9F48091E7299091E829892BC9F480913D
:10F11000E9299091EA29892B99F48091EB29909122
:10F12000EC29892B69F48091ED299091EE29892BA6
:10F1300039F48091EF299091F029892B09F4FEC1CF
:10F14000FB0113E0EE0FFF1F1A95E1F7E60FF71F23
:10F15000EE59F64DB084513051F411968C911197BF
:10F16000813019F078E0B72E02C062E0B62E9D0122
:10F170002E5F3F4F8E010F5F1F4FC801B9014B2D0E
:10F1800050E00E94D6BAB98681EE99E20E9463836C
:10F190007C0190934C2180934B21009749F481EEA0
:10F1A00099E2B80140E022E030E00E94C88330C01C
:10F1B00000913F21109140210E5F1F4F50E1C52E5D
:10F1C000D12CC80ED91EC801B6014B2D50E00E94AB
:10F1D000C9BA009721F4F701808DB81681F0C601F5
:10F1E000B8014B2D50E00E94D6BAE0914B21F0912E
:10F1F0004C21B08EE0914B21F0914C2105C0F701DC
:10F20000828D938D892B21F482E090E0938F828F01
:10F210008091DE2090E0875F954D60E840E050E00F
:10F220000E9498629093522180935121892B09F476
:10F2300085C18091E1299091E229892B09F074C060
:10F240008091E3299091E429892B09F06DC0809188
:10F25000E5299091E629892B09F066C08091E7297C
:10F260009091E829892B09F05FC08091E92990915C
:10F27000EA29892B09F058C08091EB299091EC295B
:10F28000892B09F051C08091ED299091EE29892BAD
:10F2900009F04AC08091EF299091F029892B09F05B
:10F2A00043C081EF99E20E940D60882309F446C1B2
:10F2B000E0915121F091522180899189892B61F14E
:10F2C0008FEF92E09093F2298093F1291092F42924
:10F2D0001092F3291092F6291092F5291092F8292C
:10F2E0001092F7291092FA291092F9291092FC290C
:10F2F0001092FB291092FE291092FD2980E091E0E6
:10F300009093002A8093FF2981EE99E261EF79E2E0
:10F310000E94F96350E255C08091DE2090E0875F43
:10F32000954D0E9404630AC181EE99E260E840E0D5
:10F3300050E00E949862892B09F000C181EF99E2A8
:10F340000E940D608823B9F0E1EFF9E2DF015097E8
:10F3500080E10D9001928150E1F78091DE20E82F4D
:10F36000F0E0A1EEB9E2E75FF54D80E101900D928A
:10F370008150E1F725C081EF99E260E840E050E07C
:10F380000E9498622091512130915221281739070B
:10F3900009F0D4C0E1EFF9E2DF01509780E10D9070
:10F3A00001928150E1F78091DE20E82FF0E0A1EE9C
:10F3B000B9E2E75FF54D80E101900D928150E1F7F0
:10F3C00050E61092DE2080915929282F30E087E105
:10F3D00091E0289FF001299FF00D389FF00D112436
:10F3E000E85DF04D838981115068F90143E0EE0F2B
:10F3F000FF1F4A95E1F7E20FF31FEE59F64D208506
:10F40000822F90E00296422F4E5F87709070481BCB
:10F41000892B09F0485F80E68093D9291092DA2978
:10F420001092DC291092DB291092DD29485E40936E
:10F43000DE2948518AE38093DF298FEF8093E0290A
:10F4400088E88093012A1092022A5093052AA9E0A5
:10F45000BAE22091512130915221C901FC0180E191
:10F4600001900D928150E1F7042F10E0005C1F4FD6
:10F4700010935B2900935A2900541040A091DE207C
:10F48000B0E0A75EB54DB0934021A0933F2182E04C
:10F490008C9346954695469511964C9311972091DD
:10F4A00059291296822F90E0FC0133E0EE0FFF1FE6
:10F4B0003A95E1F7E80FF91FEE59F64D408589E0DE
:10F4C000289F900111242E59364DCD01B90150E0ED
:10F4D0000E94D6BA8091592990E0FC01A3E0EE0F7A
:10F4E000FF1FAA95E1F7E80FF91FEE59F64D808549
:10F4F00090E0081B190B0250104020913F213091E1
:10F5000040212E5F3F4F280F391FC90160E070E096
:10F51000A8010E94F1BA8091DE20082F10E00F5F51
:10F52000154DF801138212820E94B5548095909572
:10F53000F8019383828306C040933E2110925B2999
:10F5400010925A2929960FB6F894DEBF0FBECDBF90
:10F55000CF91DF911F910F91FF90EF90DF90CF90AF
:10F56000BF9008956F927F928F929F92AF92BF92B9
:10F57000CF92DF92EF92FF920F931F93DF93CF937F
:10F5800000D0CDB7DEB7AC0180915929282F30E0EB
:10F5900087E191E0289FF001299FF00D389FF00D41
:10F5A0001124E85DF04D8789882309F420C2F90110
:10F5B000A3E0EE0FFF1FAA95E1F7E20FF31FEE594C
:10F5C000F64D2085822F90E00296E2E0DE2ED20EEC
:10F5D00087709070D81A892B11F088E0D80E6115C9
:10F5E000710529F58FEF92E09093F2298093F1292C
:10F5F0001092F4291092F3291092F6291092F5290D
:10F600001092F8291092F7291092FA291092F929EC
:10F610001092FC291092FB291092FE291092FD29CC
:10F6200080E091E09093002A8093FF2908C0A1EF29
:10F63000B9E2FB0180E101900D928150E1F74115A3
:10F64000510549F0A1EEB9E2FA0180E101900D9275
:10F650008150E1F706C081EE99E261EF79E20E9404
:10F66000F9631092DE2080E68093D9291092DA297E
:10F670001092DC291092DB298AE38093DF298FEF37
:10F680008093E02986E88093012AE9EDF9E211A64A
:10F690008091592990E007E111E0809FF001819F5E
:10F6A000F00D909FF00D1124E85DF04D8481809362
:10F6B000052A818992890E9499559093082A8093FE
:10F6C000072A8091DE20E82EFF24E5E0FAE2EE0E24
:10F6D000FF1E8091592990E0809FF001819FF00DDD
:10F6E000909FF00D1124E85DF04D65817681878152
:10F6F00090850E949D55F701648375838683978367
:10F700008091DE20E82EFF2485E09AE2E80EF91EC3
:10F710008091592990E0809FF001819FF00D909F8A
:10F72000F00D1124E85DF04D65857685878590891B
:10F730000E949D55F70160877187828793870D2D01
:10F7400010E0085C1F4F10935B2900935A2908535F
:10F750001040A091DE20B0E0AF5EB54DB0934021E7
:10F76000A0933F2181E08C938D2D8695869586957B
:10F7700011968C931197209159291296822F90E01F
:10F78000FC0133E0EE0FFF1F3A95E1F7E80FF91F98
:10F79000EE59F64D408589E0289F900111242E599D
:10F7A000364DCD01B90150E00E94D6BA8091592959
:10F7B00090E0FC0123E0EE0FFF1F2A95E1F7E80F30
:10F7C000F91FEE59F64D808590E0081B190B025089
:10F7D000104020913F21309140212E5F3F4F280F54
:10F7E000391FC90160E070E0A8010E94F1BAFCE095
:10F7F000DF0ED0923E210E942E7F7C011092532179
:10F80000B2E29B2EA3E06A2EF0EC7F2EE4E08E2E77
:10F81000AA24AA94BA2C6501C8C0899DF0011124BC
:10F82000EE0DFF1D81A18670863009F0B9C0808180
:10F830008E3F21F48181803809F4B2C08091DE20AE
:10F84000082F10E0045D1F4F80913E21482F50E0AB
:10F85000D801A752B64DA40FB51F6C9213967C9297
:10F86000139711968C92119720915321822F90E03B
:10F87000FC0175E0EE0FFF1F7A95E1F7880F991FE5
:10F88000E80FF91FEE0DFF1D808912968C931297D9
:10F89000299DF0011124EE0DFF1D81A180FF0DC0F7
:10F8A0001496AD92BD92CD92DC9217971896AD92B8
:10F8B000BD92CD92DC921B9743C0040F151F0752D7
:10F8C000164D658976898789908D20E432E44FE072
:10F8D00050E00E9445B5CA01B9010E949D55F8014A
:10F8E00064837583868397838091DE2090913E2187
:10F8F000092F10E0080F111D0B5F154D809153214A
:10F9000090E0FC0145E0EE0FFF1F4A95E1F7880FFC
:10F91000991FE80FF91FEE0DFF1D658D768D878D00
:10F9200090A120E432E44FE050E00E9445B5CA01C6
:10F93000B9010E949D55F80160877187828793877E
:10F94000E091DE20F0E080913E21EB5FF54DE80F85
:10F95000F11D14861586168617868091532190E036
:10F96000DC0125E0AA0FBB1F2A95E1F7880F991F3C
:10F97000A80FB91F7096AE0DBF1D80E10D900192CA
:10F980008150E1F780913E21805E80933E218091FD
:10F990005A2990915B29809690935B2980935A29EC
:10F9A000809153218F5F8093532180915321843024
:10F9B00008F433CF80915A2990915B2988979A83D4
:10F9C00089838A818093DD2989818093DE298091D2
:10F9D000DE20082F10E00F5F154DF8011382128210
:10F9E0000E94B55480959095F801938382830F907F
:10F9F0000F90CF91DF911F910F91FF90EF90DF90CB
:10FA0000CF90BF90AF909F908F907F906F90089510
:10FA1000BF92CF92DF92EF92FF920F931F93DF93EB
:10FA2000CF93CDB7DEB769970FB6F894DEBF0FBEA0
:10FA3000CDBF50915929052F10E087E191E0089F33
:10FA4000F001099FF00D189FF00D1124E85DF04DB5
:10FA50008789882309F4F8C08389882309F4F0C0D2
:10FA60008091E0298F3F09F0EBC08091DE20682F64
:10FA700070E0FB01EF5FF54D8181882309F0E0C064
:10FA80001092402110923F2184E080933E21E0902B
:10FA90005A29F0905B2920E030E044E0FB01BC965D
:10FAA00011C0DC01A752B64D11969C911197992374
:10FAB00009F4C0C08C91813009F49D01990F990F10
:10FAC000990F490FCF01840F911D8E159F0548F3A3
:10FAD00020933F213093402140933E212115310551
:10FAE00009F493C08091E1299091E229892B59F57D
:10FAF0008091E3299091E429892B29F58091E529CA
:10FB00009091E629892BF9F48091E7299091E829D1
:10FB1000892BC9F48091E9299091EA29892B99F4DC
:10FB20008091EB299091EC29892B69F48091ED2942
:10FB30009091EE29892B39F48091EF299091F02949
:10FB4000892B09F47DC0F80183E0EE0FFF1F8A9531
:10FB5000E1F7E00FF11FEE59F64DB084513049F452
:10FB6000F9018181813019F008E0B02E02C012E065
:10FB7000B12E2E5F3F4F8E010F5F1F4FC801B9019D
:10FB80004B2D50E00E94D6BAB98681EE99E20E94D0
:10FB900063837C0190934C2180934B21009749F41F
:10FBA00081EE99E2B80140E022E030E00E94C88393
:10FBB0002CC000913F21109140210E5F1F4FB0E1FA
:10FBC000CB2ED12CC80ED91EC801B6014B2D50E04A
:10FBD0000E94C9BA009721F4F701808DB81661F030
:10FBE000C601B8014B2D50E00E94D6BAE0914B21DE
:10FBF000F0914C21B08E05C0F701828D938D892B39
:10FC000021F482E090E0938F828F10925B29109212
:10FC10005A29DE011A96E1EEF9E280E101900D9297
:10FC20008150E1F780E090E0BE01665F7F4F0E9467
:10FC30003A610AC03093402120933F2140933E21F6
:10FC400010925B2910925A2969960FB6F894DEBF7C
:10FC50000FBECDBFCF91DF911F910F91FF90EF901D
:10FC6000DF90CF90BF9008952091592930E040E077
:10FC7000ABE0B0E086E190E0289FB001299F700DD5
:10FC8000389F700D11240FC0842F90E08A9FF001DF
:10FC90008B9FF00D9A9FF00D1124E60FF71FEC5982
:10FCA000FB4D12864F5F423078F34093A0250895B4
:10FCB00090E028E831E0A901849F9001859F300DF4
:10FCC000949F300D11242C5A3E4DC9010895CF93B5
:10FCD000DF93DC011092A6251092A5251092A02595
:10FCE00050915929252F30E040E0CBE0D0E086E16B
:10FCF00090E0289FB001299F700D389F700D11244E
:10FD000029C0842F90E08C9FF0018D9FF00D9C9F67
:10FD1000F00D1124E60FF71FEC59FB4D8285882367
:10FD2000C1F0808191818A179B0799F44093A025A7
:10FD30008BE0489FC001112426E1529F90011124BD
:10FD4000820F931F8C599B4D9093A6258093A525D8
:10FD500005C04F5F4230A8F24093A0258091A525B1
:10FD60009091A625DF91CF9108950F931F93CF9384
:10FD7000DF931092A6251092A5251092A0259091B0
:10FD80005929292F30E086E1989FD001112440E0C5
:10FD900050E060E00BE010E086E190E0289FE00199
:10FDA000299FD00D389FD00D11242BE036C0862F0F
:10FDB00090E0809FF001819FF00D909FF00D112445
:10FDC000EC0FFD1FEC59FB4D8285882329F1019032
:10FDD000F081E02D309701F1828D938D009711F025
:10FDE000059759F441155105B9F4629FA0011124FA
:10FDF0004A0F5B1F4C595B4D0FC06093A0258BE0F1
:10FE0000689FC00111248A0F9B1F8C599B4D9093B2
:10FE1000A6258093A52509C06F5F623040F25093FC
:10FE2000A6254093A5256093A0258091A5259091B6
:10FE3000A625DF91CF911F910F910895FC011286A5
:10FE40000190F081E02D828D938D059709F415A620
:10FE50000895FC0181A18D7F81A3089520915929E6
:10FE600088E8289F9001112420573B4DC90108952F
:10FE70007F928F929F92AF92BF92CF92DF92EF923A
:10FE8000FF920F931F93CF93DF9390915929A92F3E
:10FE9000B0E086E1989FE001112420E030E040E0EE
:10FEA0000BE010E086E190E0A89FB001A99F700DE3
:10FEB000B89F700D11245BE018C0842F90E0809FE4
:10FEC000F001819FF00D909FF00D1124E60FF71FB8
:10FED000EC59FB4D8285813039F4459F9001112406
:10FEE0002C0F3D1F2C593B4D4F5F423030F3309368
:10FEF000A6252093A5254093A0251092A425109215
:10FF0000A32587E191E0A89FF001A99FF00DB89F7C
:10FF1000F00D1124E85DF04D8789882309F4DCC0D9
:10FF20001092A02511E3812E912CB8E8AB2EB1E000
:10FF3000BB2EA1E37A2EF2E0CF2ED12CC7E1D1E087
:10FF4000E4E0EE2EF12CC3C08091592990E0242FDB
:10FF500030E0289DD001299DB00D389DB00D1124B1
:10FF60008A9D90018B9D300D9A9D300D1124A20F1A
:10FF7000B31FAC5ABE4D9D968C919D97813009F070
:10FF8000A1C0479DF0011124E20FF31FEC5AFE4D72
:10FF9000F093A425E093A325828D938D8130910564
:10FFA00001F18130910538F08330910549F10497D2
:10FFB00009F088C034C084A5833018F09D961C9247
:10FFC00081C0CF0184960E94FA85892B09F47AC0FA
:10FFD0004091A3255091A42580E090E060E070E07E
:10FFE00048C0CF014C960E94FA85892B09F46AC05B
:10FFF000E091A325F091A425D38EC28E14A662C0F1
:020000021000EC
:10000000CF014C960E94FA85892B09F45BC0E091E0
:10001000A325F091A425F38EE28E14A623C084A517
:100020008330D0F014A6CF010E94677EFC0190932C
:10003000A6258093A525009749F012860190F081AE
:10004000E02D828D938D059709F415A6E091A325E7
:10005000F091A42515A636C0CF0184960E94FA859A
:10006000892B81F14091A3255091A42580E090E057
:10007000BA010E94E9740091A3251091A4258091F2
:10008000592990E08C9FF0018D9FF00D9C9FF00D01
:100090001124E85DF04D658576858785908928EE89
:1000A00033E040E050E00E94FFB4AB01BC01C80166
:1000B00084960E942386E091A325F091A42584A52F
:1000C0008F5F84A78091A0258F5F8093A0254091AA
:1000D000A025483008F438CF1092A2251092A1250F
:1000E00081E08093A025C8E8D0E002E218E841C092
:1000F00050915929252F30E0842F90E0FC0175E0C4
:10010000EE0FFF1F7A95E1F7880F991FE80FF91F8F
:100110002C9FC0012D9F900D3C9F900D1124E80F46
:10012000F91FEF54FB4D808181FF1EC0409FF001FD
:100130001124519FC0011124E80FF91FE057FB4D16
:10014000F093A225E093A12581A180FD0DC0CF01F0
:1001500041960E94FA85892B39F0E091A125F09112
:10016000A22581A18D7F81A38091A0258F5F80939F
:10017000A0254091A025443008F4BACFDF91CF915B
:100180001F910F91FF90EF90DF90CF90BF90AF90B5
:100190009F908F907F900895AF92BF92CF92DF9201
:1001A000EF92FF920F931F93CF93DF93182FB92EE7
:1001B000A62E69017A011092A2251092A12581E054
:1001C0008093A0258091592990E041E028E830E013
:1001D000829FB001839F700D929F700D112419C0F2
:1001E000242F2F5F842F90E0FC0135E0EE0FFF1FDE
:1001F0003A95E1F7880F991FE80FF91FE60FF71FEF
:10020000EF54FB4D808181FD03C04093A02510C0B9
:10021000422F443028F34093A025443049F40E94F3
:10022000E2B663E070E00E9432B58F5F8093A02554
:100230009091A02582E2989FF00111248091592984
:1002400028E8829FC0011124E80FF91FE057FB4DF9
:10025000F093A225E093A125EF01212F3B2DC901A9
:10026000DC0180E10D9009928150E1F7A08AC11470
:10027000D104E104F10469F0CF014196B701A60170
:100280000E942386E091A125F091A22581A18E7F75
:1002900002C081A1816081A32091592930E0609141
:1002A000A025862F90E0FC01A5E0EE0FFF1FAA9588
:1002B000E1F7880F991FE80FF91F88E890E0289F61
:1002C000A001299F500D389F500D1124E40FF51FF8
:1002D000EF54FB4D80818260808300FF13C0862F26
:1002E00090E0FC0165E0EE0FFF1F6A95E1F7880FD3
:1002F000991FE80FF91FE40FF51FEF54FB4D8081A4
:10030000846012C0862F90E0FC0125E0EE0FFF1FF5
:100310002A95E1F7880F991FE80FF91FE40FF51FE1
:10032000EF54FB4D80818B7F80838091A12590913C
:10033000A225DF91CF911F910F91FF90EF90DF9059
:10034000CF90BF90AF900895EF92FF920F931F93BD
:10035000CF93DF93EC017A018B011092A6251092C6
:10036000A5251092A0252091592930E040E0ABE06E
:10037000B0E086E190E0289FB001299F700D389F82
:10038000700D112416C0242F2F5F842F90E08A9FB8
:10039000F0018B9FF00D9A9FF00D1124E60FF71FCF
:1003A000EC59FB4D8285882319F44093A0250FC09A
:1003B000422F423040F34093A025423041F40E9446
:1003C000E2B662E070E00E9432B58093A025E09131
:1003D000A0258BE0E89FF00111248091592926E1A6
:1003E000829FC0011124E80FF91FEC59FB4DF093D7
:1003F000A625E093A525C193D193CF01B801A7010C
:100400000E9423862091A02530E04091592950E098
:100410008BE090E0289FF001299FF00D389FF00DB0
:10042000112486E190E09C01429FC001439F900D02
:10043000529F900D1124E80FF91FEC59FB4D81E0FC
:1004400082878091A5259091A625DF91CF911F915C
:100450000F91FF90EF900895EF92FF920F931F93EB
:10046000CF93DF937C011092A2251092A1251092C8
:10047000A02500915929202F30E088E890E0289F9E
:10048000E001299FD00D389FD00D11243EC0812F4F
:1004900090E0FC0175E0EE0FFF1F7A95E1F7880F01
:1004A000991FE80FF91FEC0FFD1FEF54FB4D8081E2
:1004B00081FF28C0212F30E0C90155E0880F991F26
:1004C0005A95E1F7220F331F820F931F8C0F9D1F48
:1004D00080579B4DB70140E150E00E94C9BA009798
:1004E00089F482E2189FC001112428E8029F90013C
:1004F0001124820F931F80579B4D9093A2258093C8
:10050000A12508C01F5F1093A0251091A0251430CD
:1005100008F4BDCF8091A1259091A225DF91CF91C4
:100520001F910F91FF90EF900895EF92FF921F930C
:10053000CF93DF937C011092A0258091592990E000
:1005400028E830E0829FE001839FD00D929FD00D7C
:10055000112442C0812F90E0FC0175E0EE0FFF1FD7
:100560007A95E1F7880F991FE80FF91FEC0FFD1F2F
:10057000EF54FB4D808181FF2CC0212F30E0C90159
:1005800055E0880F991F5A95E1F7220F331F820F0C
:10059000931F8C0F9D1F212F30E0F901B5E0EE0F66
:1005A000FF1FBA95E1F7220F331FE20FF31FEC0F85
:1005B000FD1FE057FB4D408946954695469580576F
:1005C0009B4DB70150E00E94C9BA009711F481E039
:1005D00009C01F5F1093A0251091A025143008F4C6
:1005E000B9CF80E0DF91CF911F91FF90EF900895F8
:1005F000CF92DF92EF92FF920F931F93CF93DF93EF
:10060000EC011092A4251092A3251092A025009130
:100610005929202F30E0E1E3CE2ED12C88E891E05B
:10062000289F7001299FF00C389FF00C11243AC0CC
:10063000812F90E08C9D90018D9D300D9C9D300D03
:1006400011242E0D3F1DF901EC5AFE4D85A588237E
:1006500031F1408D8885481711F5C9018C599E4D9F
:10066000BE0150E00E94C9BA0097C9F481E3189F07
:10067000C0011124402F50E028E831E0B901469F25
:100680009001479F300D569F300D1124820F931F0C
:100690008C5A9E4D9093A4258093A32507C01F5F7D
:1006A0001093A0251091A025183010F28091A32559
:1006B0009091A425DF91CF911F910F91FF90EF9022
:1006C000DF90CF900895CF92DF92EF92FF920F9339
:1006D0001F93CF93DF937C011092A4251092A32542
:1006E0001092A02500915929202F30E0F1E3CF2E60
:1006F000D12C88E891E0289FE001299FD00D389FF8
:10070000D00D112434C0812F90E08C9DF0018D9D7F
:10071000F00D9C9DF00D1124EC0FFD1FEC5AFE4DC9
:1007200085A5882309F1CF01B70140E150E00E947F
:10073000C9BA0097C9F481E3189FC0011124402F62
:1007400050E028E831E0B901469F9001479F300D05
:10075000569F300D1124820F931F8C5A9E4D9093FB
:10076000A4258093A32507C01F5F1093A025109197
:10077000A025183040F28091A3259091A425DF9107
:10078000CF911F910F91FF90EF90DF90CF90089540
:10079000BF92CF92DF92EF92FF920F931F93CF936E
:1007A000DF93D82EC92E8B01B42E79011092A42587
:1007B0001092A3251092A0252091592930E040E005
:1007C000A1E3B0E088E891E0289FB001299F700D77
:1007D000389F700D112416C0242F2F5F842F90E0B6
:1007E0008A9FF0018B9FF00D9A9FF00D1124E60F68
:1007F000F71FEC5AFE4D85A5882319F44093A025D8
:100800000FC0422F483040F34093A025483041F4B8
:100810000E94E2B668E070E00E9432B58093A025A5
:10082000409159299091A02581E3989FE0011124DE
:10083000242F30E088E891E0BC01269FC001279F6B
:10084000900D369F900D1124C80FD91FCC5ADE4D44
:10085000D093A425C093A325DE012D2D3C2DC901E5
:10086000FC0180E101900D928150E1F70115110525
:10087000C9F01092A025E0E00AC0F0E0DE01AE0F62
:10088000BF1FE00FF11F808150968C93E92FD80194
:1008900018968C919E2F9F5FE81778F3E093A02520
:1008A000888F1BC0842F90E0FC01A3E0EE0FFF1F98
:1008B000AA95E1F7E80FF91FEE59F64D40859E0124
:1008C000205F3F4FC90160E070E050E00E94F1BA44
:1008D000E091A325F091A425108EE091A325F0913D
:1008E000A425B18EF38EE28ECF014C9640E050E00D
:1008F00060E070E00E9423868091A3259091A4255A
:10090000849640E050E060E070E00E942386E09131
:10091000A325F091A42514A681E085A7CF01DF913E
:10092000CF911F910F91FF90EF90DF90CF90BF90EC
:1009300008951F9310915929412F50E020E0A1E321
:10094000B0E088E891E0489FB001499F700D589F42
:10095000700D11240FC0822F90E08A9FF0018B9FB1
:10096000F00D9A9FF00D1124E60FF71FEC5AFE4D83
:1009700015A62F5F283078F320E0ABE0B0E086E1E9
:1009800090E0489FB001499F700D589F700D112451
:100990000FC0822F90E08A9FF0018B9FF00D9A9FED
:1009A000F00D1124E60FF71FEC59FB4D12862F5F57
:1009B000223078F320E088E890E0489FB001499F1A
:1009C000700D589F700D112414C0822F90E0FC010F
:1009D000A5E0EE0FFF1FAA95E1F7880F991FE80F1A
:1009E000F91FE60FF71FEF54FB4D80818D7F808349
:1009F0002F5F243050F32093A02587E191E0489F9A
:100A0000F001499FF00D589FF00D1124E85DF04D65
:100A10008589882309F464C088E890E0489F9001A4
:100A2000499F300D589F300D1124D901A057BB4D5F
:100A30008EEF90E811969C938E9384E490E0489F0B
:100A4000F001499FF00D589FF00D1124EE0FFF1F8C
:100A5000EE56FB4D11821082FA01EE0FFF1FCA0104
:100A600075E0880F991F7A95E1F7E80FF91FEE0FEF
:100A7000FF1FEE0FFF1FEC56FB4D118210821796E1
:100A80001C921E921697FA0194E0EE0FFF1F9A95A2
:100A9000E1F7E40FF51F83E0EE0FFF1F8A95E1F702
:100AA000E856FB4D118210821B961C921E921A97DB
:100AB0001D961C921E921C971F961C921E921E97AA
:100AC00080E450968C932F543B4DF90180818360D4
:100AD0008083812F40EA56E861E070E00E94E4875D
:100AE0001F910895FFCF0895CF92DF92EF92FF926A
:100AF0000F931F93DF93CF93CDB7DEB729970FB630
:100B0000F894DEBF0FBECDBF8C0180915929882398
:100B100039F501151105A1F483E389838A83809156
:100B2000FD298B838091FE298C838091FF298D8301
:100B30008091002A8E8386E089878E010F5F1F4F88
:100B4000E0905A29F0905B2980E060E040E050E0BE
:100B500026E099EDC92E99E2D92E0E94458E10C04B
:100B6000813091F40115110541F48FEF89838A8357
:100B700082E089878E010F5F1F4FC8010E94334EAC
:100B800010925B2910925A2980E090E029960FB6C6
:100B9000F894DEBF0FBECDBFCF91DF911F910F91B3
:100BA000FF90EF90DF90CF9008950F931F93DF9306
:100BB000CF9300D000D0CDB7DEB78C01CE01019627
:100BC0000E94CB11F80120813181428153818981BA
:100BD0009A81AB81BC81281B390B4A0B5B0BB90195
:100BE000CA010F900F900F900F90CF91DF911F913E
:100BF0000F9108950F931F93DF93CF9300D000D0F0
:100C0000CDB7DEB78C01CE0101960E94CB1160E01A
:100C100070E0F801208131814281538189819A817C
:100C2000AB81BC81281739074A075B0710F461E0E4
:100C300070E0CB010F900F900F900F90CF91DF914C
:100C40001F910F910895CF92DF92EF92FF920F9331
:100C50001F93DF93CF9300D000D0CDB7DEB76C01E8
:100C60007A018B01CE0101960E94CB11F601E4823C
:100C7000F5820683178389819A81AB81BC818E0DB1
:100C80009F1DA01FB11F80839183A283B3830F9008
:100C90000F900F900F90CF91DF911F910F91FF90C8
:100CA000EF90DF90CF900895882321F48DE00E948B
:100CB00009130895813019F48CE00E9409130895F6
:100CC000882321F489E00E9409130895813019F4E2
:100CD00088E00E940913089584E00E94091385E0CA
:100CE0000E94091386E00E94091387E00E940913FD
:100CF00088E00E94091389E00E9409138AE00E949B
:100D000009138BE00E9409138CE00E9409138DE007
:100D10000E9409138EE00E9409138FE00E940913BC
:100D200080E10E94091381E10E9409130895AF92A6
:100D3000BF92CF92DF92EF92FF920F931F935A01CF
:100D40006B01813031F480E120E030E00DE918E8FA
:100D500005C081E120E030E006E918E8EE24FF2438
:100D60000E9415148823B9F0A114B104C104D10460
:100D700091F000D000D08AE298E0EDB7FEB7928300
:100D800081838EEE91E0948383830E94FCBB0F905D
:100D90000F900F900F901F910F91FF90EF90DF90A9
:100DA000CF90BF90AF900895AF92BF92CF92DF9255
:100DB000EF92FF920F931F935A016B01813031F430
:100DC0008EE020E030E00CEA18E805C08FE020E07B
:100DD00030E005EA18E8EE24FF240E941514882369
:100DE000B9F0A114B104C104D10491F000D000D035
:100DF0008AE298E0EDB7FEB79283818388ED91E0B7
:100E0000948383830E94FCBB0F900F900F900F90F0
:100E10001F910F91FF90EF90DF90CF90BF90AF9018
:100E20000895AF92BF92CF92DF92EF92FF920F930D
:100E30001F935A016B01813031F48CE020E030E0E7
:100E40000BEB18E805C08DE020E030E004EB18E87B
:100E5000EE24FF240E9415148823B9F0A114B104D4
:100E6000C104D10491F000D000D08AE298E0EDB73F
:100E7000FEB79283818381EC91E0948383830E9407
:100E8000FCBB0F900F900F900F901F910F91FF9050
:100E9000EF90DF90CF90BF90AF900895AF92BF9248
:100EA000CF92DF92EF92FF920F931F93282F5A0158
:100EB0006B01E82FF0E0411551056105710551F412
:100EC000EE0FFF1FE955FA4D808191815C01CC2422
:100ED000DD2406C0EE0FFF1FE955FA4D5183408314
:100EE000213041F48AE0B601A50120E030E001EDB7
:100EF00018E807C08BE0B601A50120E030E003EC64
:100F000018E8EE24FF240E9415148823B9F0A114D8
:100F1000B104C104D10491F000D000D08AE298E07D
:100F2000EDB7FEB7928381838AEA91E0948383834D
:100F30000E94FCBB0F900F900F900F901F910F918C
:100F4000FF90EF90DF90CF90BF90AF900895AF9259
:100F5000BF92CF92DF92EF92FF920F931F935A01AD
:100F60006B01813031F488E020E030E006EE18E8D3
:100F700005C089E020E030E00FED18E8EE24FF2402
:100F80000E9415148823B9F0A114B104C104D1043E
:100F900091F000D000D08AE298E0EDB7FEB79283DE
:100FA00081838DE891E0948383830E94FCBB0F9042
:100FB0000F900F900F901F910F91FF90EF90DF9087
:100FC000CF90BF90AF900895AF92BF92CF92DF9233
:100FD000EF92FF920F931F93282F5A016B01E82F76
:100FE000F0E0411551056105710551F4EE0FFF1F49
:100FF000E555FA4D808191815C01CC24DD2406C049
:10100000EE0FFF1FE555FA4DB182A082213041F469
:1010100086E0B601A50120E030E00CEF18E807C03B
:1010200087E0B601A50120E030E00EEE18E8EE24DE
:10103000FF240E9415148823B9F0A114B104C1043F
:10104000D10491F000D000D08AE298E0EDB7FEB76D
:101050009283818387E791E0948383830E94FCBB22
:101060000F900F900F900F901F910F91FF90EF90A6
:10107000DF90CF90BF90AF900895AF92BF92CF9284
:10108000DF92EF92FF920F931F93282F5A016B016B
:10109000E82FF0E0411551056105710551F4EE0F9F
:1010A000FF1FE155FA4D808191815C01CC24DD2444
:1010B00006C0EE0FFF1FE155FA4DB182A08221302C
:1010C00041F484E0B601A50120E030E008E119E830
:1010D00007C085E0B601A50120E030E00AE019E88C
:1010E000EE24FF240E9415148823B9F0A114B10442
:1010F000C104D10491F000D000D08AE298E0EDB7AD
:10110000FEB7928381838AE591E0948383830E9472
:10111000FCBB0F900F900F900F901F910F91FF90BD
:10112000EF90DF90CF90BF90AF9008951092592923
:101130000E94A0600E94C168089581E080935929AF
:101140000E94A0600E94C1680895109259290E94CF
:1011500097610E94C168089581E0809359290E9497
:1011600097610E94C1680895109259290E941C62DB
:101170000E94C168089581E0809359290E941C62F1
:101180000E94C16808951092592980E040E050E023
:1011900060E070E00E944E870E9427660E94C1684E
:1011A000089581E08093592940E050E060E070E0CC
:1011B0000E944E870E9427660E94C168089510927F
:1011C00059290E945E630E94C168089581E080935E
:1011D00059290E945E630E94C1680895109259299E
:1011E00080E040E050E060E070E00E94E4870E9410
:1011F000387F0E94C168089581E08093592940E0BA
:1012000050E060E070E00E94E4870E94387F0E9416
:10121000C16808951092592980E040E050E060E0F4
:1012200070E00E943D880E94E36B0E94C1680895AF
:1012300081E08093592940E050E060E070E00E9436
:101240003D880E94E36B0E94C16808950F931F932D
:10125000DF93CF93CDB7DEB762970FB6F894DEBFBA
:101260000FBECDBF9A8B898BFB0181E080935929FA
:101270008A898093563189898093573182E080939F
:101280007329808180936B29818180936C298EEFF3
:1012900090E89A8389831C821B821E821D82188695
:1012A0001F821A8619861C861B861E861D86188A32
:1012B0001F86CE01019660E420E030E040E050E07F
:1012C00001E010E00E943C6562960FB6F894DEBF24
:1012D0000FBECDBFCF91DF911F910F910895CF9297
:1012E000DF92EF92FF920F93DF93CF93CDB7DEB7EC
:1012F00029970FB6F894DEBF0FBECDBFAC01FE013B
:10130000319689E0DF011D928A95E9F786E08987A9
:10131000109259294115510581F020E030E0BF01BC
:10132000FB01E20FF31FDA01A20FB31F8C91808340
:101330002F5F3F4F2630310599F786E0898788E592
:1013400098E00E94A06868E077E080E090E041E0EB
:1013500021E000E0BFE3EB2EB8E0FB2E6E01089425
:10136000C11CD11C0E94C25F80E040E251EA67E0EC
:1013700070E00E943D8829960FB6F894DEBF0FBE3C
:10138000CDBFCF91DF910F91FF90EF90DF90CF9085
:101390000895CF92DF92EF92FF920F936C0101E0DC
:1013A000009359298091760390917703892BC1F49A
:1013B00088E498E00E94A0680093592968EE73E0E1
:1013C00080E090E041E021E000E053E4E52E58E0C9
:1013D000F52E0E94C25F88E498E00E9498450DC0F7
:1013E00060E070E080E090E040E021E000E033E485
:1013F000E32E38E0F32E0E94C25F81E040E251EA22
:1014000067E070E00E943D880F91FF90EF90DF90C1
:10141000CF90089583EB95E29093562980935529B8
:101420000E946C860E949C450895FC0120E09081FA
:101430008181808391832E5F32962031C1F7089598
:10144000992787FD90950E9490BA8A3314F08753AC
:10145000089580530895FF920F931F938C01FC0110
:1014600080810E94208AF82EF29480EFF822F80101
:1014700081810E94208A8F0D1F910F91FF90089506
:10148000992787FD90950E9488BA8833A1F1893306
:1014900084F4843341F185333CF4823301F18333A6
:1014A00004F58133D1F417C0863309F187330CF585
:1014B0001CC0833641F184363CF4813601F182361A
:1014C00004F5893351F419C0853609F18536ECF0FD
:1014D000863619F41EC081E0089580E0089582E008
:1014E000089583E0089584E0089585E0089586E0F6
:1014F000089587E0089588E0089589E008958AE0D6
:1015000008958BE008958CE008958DE008958EE0B5
:1015100008958FE00895EF92FF921F93CF93DF938A
:101520007C01EC0110E001C01F5F8881992787FDD5
:1015300090950E946CBA892B19F4C0E0D0E022C0CB
:101540002196143089F7F9CFF70180810E94408AF3
:1015500090E0143029F4982F88279295907F0CC042
:10156000133019F4982F882707C0123029F424E08B
:10157000880F991F2A95E1F7C80FD91F11500894B9
:10158000E11CF11C112301F7CE01DF91CF911F91D6
:10159000FF90EF9008955F926F927F928F929F924B
:1015A000AF92BF92CF92DF92EF92FF920F931F9371
:1015B000DF93CF9300D000D00F92CDB7DEB74C01B0
:1015C0006B018C019C01A8E0EA2EFF24F8E05F2E5D
:1015D0005E010894A11CB11CE5E06E2E712C6C0E0E
:1015E0007D1E02C00F5F1F4FF80140814A3311F08A
:1015F0004423C1F7C801821B930B059714F080E0C8
:101600005EC0F80182918F010F5F1F4F8A3319F07E
:10161000D501F9012FC0442319F0F40190E00EC068
:10162000EF2DF0E0EE0FFF1FEC0DFD1D118210827B
:10163000F39440C08A3309F49F5F319680818823F8
:10164000C9F7252D291B922F8F2D0AC0E82FF0E016
:10165000EE0FFF1FEC0DFD1D1182108291508F5F68
:101660009923A1F7F20EE21A0F5F1F4F98011FC0D6
:101670008D9331969E2F921B80818A3319F0A61587
:10168000B705B1F7F501E90FF11D1082C5010E9400
:101690008B8AEF2DF0E0EE0FFF1FEC0DFD1D918307
:1016A000808398012F5F3F4FF394EA948901EE20E5
:1016B00009F09ACF80E0F8E0FF1609F481E00F907E
:1016C0000F900F900F900F90CF91DF911F910F917E
:1016D000FF90EF90DF90CF90BF90AF909F908F9052
:1016E0007F906F905F900895AF92BF92CF92DF92FC
:1016F000EF92FF920F931F93CF93DF938C01EB0137
:101700006115710509F46BC0EE24FF2438E6C32E81
:1017100038E0D32E20E3A22E9AE3B92E8881998156
:10172000009779F5EE2069F540E06F2D70E001C07B
:101730004F5F242F30E0F901EE0FFF1FEC0FFD1F6C
:1017400080819181892B29F4260F371F283031059C
:101750007CF3413039F4D801AD928D01F394229697
:1017600040E030C08F2D90E0840F911D089709F460
:101770004150842F90E0880F991FC80FD91FF40E95
:1017800021C00E94995500D000D000D0EDB7FEB71F
:101790003196ADB7BEB712961C930E931197D382B4
:1017A000C282958384830E946DBC080F191F229604
:1017B000F3944E2DEDB7FEB736960FB6F894FEBFF4
:1017C0000FBEEDBFF8E0FF1641F0D801BD928D01CC
:1017D000B7E0BF1510F0E42EA1CFF8011082DF9121
:1017E000CF911F910F91FF90EF90DF90CF90BF901E
:1017F000AF900895AF92BF92CF92DF92EF92FF9297
:101800000F931F93DF93CF9300D000D000D0CDB7BC
:10181000DEB77C0100E010E05E010894A11CB11C61
:101820004BE6C42E48E0D42E00D000D000D0EDB757
:10183000FEB73196ADB7BEB71296BC92AE92119775
:10184000D382C282D701A00FB11F8C9184831582ED
:101850000E946DBC0F5F1F4F8DB79EB706960FB6E7
:10186000F8949EBF0FBE8DBF00311105E9F6269694
:101870000FB6F894DEBF0FBECDBFCF91DF911F91A1
:101880000F91FF90EF90DF90CF90BF90AF900895B1
:101890001F93CF93DF939C01EB01142F80915A2962
:1018A00090915B29892B19F02FEF3FEF13C089ED41
:1018B00099E2B901AE010E94DFBA10935929D09381
:1018C0005B29C0935A2981E00E9435560E94C16865
:1018D00020E030E0C901DF91CF911F910895DC0134
:1018E0009C9111968C9111979F5F983728F090E00A
:1018F00003C06B9A639A08959817D9F38C91FD01F0
:10190000E80FF11D62839C930895DC0111969C9170
:101910001197FD01E90FF11D22818C918C9198178F
:1019200011F42FEF07C0892F8F5F883708F080E010
:1019300011968C93822F0895FC019081818120E083
:10194000981321E0822F0895FC018081282F30E038
:101950008181281B310937FF02C028583F4F822F51
:10196000089510924A3780914A37809349371092F0
:10197000C4378091C4378093C33788E98093C1000E
:1019800086E08093C2001092C50083E08093C4007B
:101990001092632608951092C1000895682F7894DC
:1019A00083EC97E30E946F8C8091C10085FD21C07C
:1019B0008091C00085FFFCCF9091C437E92FF0E003
:1019C000ED53F84C22818091C3378091C33798172B
:1019D00011F42FEF07C0E92FEF5FE83708F0E0E0E0
:1019E000E093C4372093C6008091C1008062809349
:1019F000C1000895833A29F0843A41F08B3179F49B
:101A00000AC08BE10E94CE8C81E009C08BE10E946C
:101A1000CE8C82E004C08BE10E94CE8C83E00E94D9
:101A2000CE8C0895EF92FF921F93CF93DF93182FE0
:101A3000EB017A0183EA0E94CE8C8C2F0E94FA8CF3
:101A40008D2F0E94FA8C812F0E94FA8C06C0F7011C
:101A500081917F010E94FA8C21972097C1F784EA37
:101A60000E94CE8CDF91CF911F91FF90EF9008954F
:101A7000CF93DF93EC0103C00E94CE8C2196888126
:101A80008823D1F7DF91CF91089580914937282F8E
:101A900030E080914A37281B310937FF02C02858AF
:101AA0003F4F822F089580914937282F30E0809151
:101AB0004A37281B310937FF02C028583F4F822F71
:101AC00008958091C337282F30E08091C437281BB8
:101AD000310937FF02C028583F4F822F0895909157
:101AE000C437E92FF0E0ED53F84C22818091C337E1
:101AF0008091C337981711F42FEF07C0E92FEF5FDC
:101B0000E83708F0E0E0E093C437822F0895789436
:101B100080914937282F30E080914A37281B3109BE
:101B200037FF02C028583F4F222391F390914A3744
:101B3000E92FF0E0E75BF84C2281809149378091F2
:101B40004937981711F42FEF07C0E92FEF5FE837F7
:101B500008F0E0E0E0934A37822F0895682F89E487
:101B600097E30E946F8C1092372608951F920F9270
:101B70000FB60F920BB60F9211242F933F934F93F2
:101B80005F936F937F938F939F93AF93BF93EF93E5
:101B9000FF936091C60089E497E30E946F8C1092D6
:101BA0003726FF91EF91BF91AF919F918F917F91D8
:101BB0006F915F914F913F912F910F900BBE0F90BE
:101BC0000FBE0F901F9018951F920F920FB60F9295
:101BD0000BB60F9211242F938F939F93EF93FF9344
:101BE0009091C3378091C4379817C9F09091C4374A
:101BF000E92FF0E0ED53F84C22818091C3378091BA
:101C0000C337981711F42FEF07C0E92FEF5FE837BC
